:020000040800F2
:100000000006022001020008510F0008D10E00086E
:10001000290F0008D10E0008FD0E00080302000899
:10002000030200080302000803020008CD270008AD
:10003000030200080302000803020008030200088C
:10004000030200080302000803020008030200087C
:10005000030200080302000831390008593900087A
:1000600081390008A9390008D139000803020008C5
:10007000030200080302000803020008030200084C
:10008000030200080302000803020008030200083C
:10009000030200080302000803020008F9390008FF
:1000A000030200080302000803020008030200081C
:1000B000E13A0008030200080302000803020008F6
:1000C00003020008030200080302000803020008FC
:1000D00003020008030200080302000803020008EC
:1000E0005D3A00080302000803020008030200084A
:1000F00003020008030200080302000803020008CC
:1001000003020008030200080302000803020008BB
:1001100003020008030200080302000803020008AB
:10012000030200080302000803020008030200089B
:10013000030200080302000803020008030200088B
:10014000030200080302000803020008812F0008D0
:10015000030200080302000803020008030200086B
:10016000030200080302000803020008030200085B
:10017000030200080302000803020008030200084B
:100180000302000803020008CD3A00080302000839
:10019000030200080302000803020008030200082B
:1001A000030200080302000803020008030200081B
:1001B000030200080302000803020008030200080B
:1001C00003020008030200080302000803020008FB
:1001D00003020008030200080302000803020008EB
:1001E00003020008030200080302000803020008DB
:1001F00003020008030200080302000803020008CB
:1002000002E000F000F8FEE772B63A4880F3088892
:10021000394880F3098839484EF60851CEF200017A
:10022000086040F20000CCF200004EF63471CEF2CD
:1002300000010860BFF34F8FBFF36F8F40F20000E3
:10024000C0F2F0004EF68851CEF200010860BFF314
:100250004F8FBFF36F8F4FF00000E1EE100A4EF6A4
:100260003C71CEF200010860062080F31488BFF3D1
:100270006F8F02F069FB02F00BFB03F0FBF94FF00C
:1002800055301F491B4A91423CBF41F8040BFAE725
:100290001C49194A91423CBF41F8040BFAE71A493C
:1002A0001A4A1B4B9A423EBF51F8040B42F8040B0A
:1002B000F8E700201749184A91423CBF41F8040B67
:1002C000FAE702F023FB03F035FA144C144DAC426C
:1002D00003DA54F8041B8847F9E700F041F8114CA1
:1002E000114DAC4203DA54F8041B8847F9E702F0D9
:1002F0000BBB0000000602200022022000000008C4
:100300000000022000060220083F00080022022010
:1003100068220220682202207834022000020008AD
:100320000002000800020008000200082DE9F04F5A
:100330002DED108AC1F80CD0D0F80CD0BDEC108A8D
:10034000BDE8F08F002383F311882846A0470020E2
:1003500001F048FEFEE701F0C3FD00DFFEE700000C
:1003600038B500F0C1FC40B1174B6FF07F0100229F
:1003700059720E211A729972DA7202F0E7F9054683
:1003800002F01AFA0446D0B9104B9D4219D001333D
:100390009D4241F2883512BF044600250124002009
:1003A00002F0DEF90CB100F059F800F039FD00F070
:1003B000DBFB284600F0E0F800F050F8F9E70025F4
:1003C000EDE70546EBE700BF00220220010007B081
:1003D00008B500F095FBA0F120035842584108BD34
:1003E00007B541F21203022101A8ADF8043000F074
:1003F000A5FB03B05DF804FB202310B583F311883F
:100400001248C3680BB101F073FE0023104A4FF489
:100410007A710E4801F030FE002383F311880D4CF1
:10042000236813B12368013B2360636813B16368D9
:10043000013B6360084B1B7833B9636823B9022022
:1004400000F068FC3223636010BD00BF6822022008
:10045000F9030008842302207C220220F8B5404BD7
:10046000404A1C461968013179D004339342F9D1CE
:100470006268A24273D33C4B9B6803F1006303F5AF
:10048000C0339A426BD2002000F088FB0220374B29
:10049000187000F035FC364B00211A6C19641A6E86
:1004A00019661A6E5A6C59645A6E59665A6E5A69B0
:1004B00042F080025A615A6922F080025A615A69F8
:1004C0001A6942F000521A611A6922F000521A6148
:1004D0001B6972B64FF0E023C3F8084DD4E900045D
:1004E000BFF34F8FBFF36F8F224AC2F88410BFF360
:1004F0004F8F536923F480335361BFF34F8FD2F88A
:10050000803043F6E076C3F3C905C3F34E335B0195
:1005100003EA060C29464CEA81770139C2F8747265
:10052000F9D2203B13F1200FF2D1BFF34F8FBFF36D
:100530006F8FBFF34F8FBFF36F8F536923F4003377
:1005400053610023C2F85032BFF34F8FBFF36F8F58
:10055000202383F31188854680F308882047F8BD5F
:100560000080010820800108002202207C22022055
:100570000038024000ED00E02DE9F04F93B0A94BA8
:100580002022FF2100900AA89D6800F0F3FBA64AF4
:100590001378A3B90121A5481170C360202383F308
:1005A0001188C3680BB101F0A3FD0023A04A4FF4EA
:1005B0007A719E4801F060FD002383F31188009B4F
:1005C0009C4A03B1136000239B49009C98469B46BC
:1005D0001E469A460B705360012000F091FB24B137
:1005E000944B1B68002B00F01682002000F088FA64
:1005F0000390039B002BF2DB012000F077FB039BB1
:10060000213B162BE8D801A252F823F06906000816
:100610009106000825070008D9050008D90500083B
:10062000D9050008B90700088B090008A5080008CB
:10063000070900082F09000855090008D905000816
:1006400067090008D9050008D9090008090700084A
:10065000D90500081D0A00087506000809070008EA
:10066000D9050008070900080220FFF7B1FE00289D
:1006700040F0FB81009B022105A8B8F1000F08BFE4
:100680001C4641F21233ADF8143000F057FAA3E7DC
:100690004FF47A7000F034FA071EEBDB0220FFF70C
:1006A00097FE0028E6D0013F052F00F2E081DFE849
:1006B00007F0030A0D1013360523042105A805933E
:1006C00000F03CFA17E004215648F9E704215B48A2
:1006D000F6E704215A48F3E74FF01C09484609F1B0
:1006E000040900F05DFA0421059005A800F026FA3F
:1006F000B9F12C0FF2D101204FF0000A00FA07F7F0
:1007000047EA0B0B5FFA8BFB00F080FB26B10BF086
:100710000B030B2B08BF0024FFF762FE5CE70421EC
:100720004848CDE7002EA5D00BF00B030B2BA1D131
:100730000220FFF74DFE074600289BD001203E4EC9
:1007400000F02CFA4FF000080220307000F0D8FAC8
:100750005FFA88F9484600F031FA044690B14846FD
:1007600008F1010800F03AFA0028F1D1B846044631
:1007700041F21213022105A83E46ADF8143000F0F4
:10078000DDF929E7012325460220337000F0AEFA97
:10079000244B9B68AB4207D9284600F001FA013090
:1007A00040F068810435F3E70025234BB8463E4608
:1007B0001D70204B5D60A7E7002E3FF45BAF0BF090
:1007C0000B030B2B7FF456AF02201B4B187000F06D
:1007D00097FA322000F094F9B0F10009FFF64AAF21
:1007E00019F003077FF446AF0E4A09EB0503926840
:1007F00093423FF63FAFB9F5807F3FF73BAF124BD7
:10080000B945019322DD4FF47A7000F079F9039035
:10081000039A002AFFF62EAF039A0137019B03F8D3
:10082000012BEDE700220220802302206822022013
:10083000F9030008842302207C22022004220220E3
:10084000082202200C22022080220220C820FFF76A
:10085000BFFD074600283FF40DAF1F2D11D8C5F18D
:1008600020020AAB25F0030084494A45184428BFFA
:100870004A46019200F058FA019AFF217F4800F0A1
:1008800079FA4FEAA903C9F387027C492846019304
:1008900000F078FA064600283FF46AAF019B05EBAA
:1008A000830531E70220FFF793FD00283FF4E2AE15
:1008B00000F0BEF900283FF4DDAE0027B946704BCA
:1008C0009B68BB4218D91F2F11D80A9B01330ED049
:1008D00027F0030312AA134453F8203C059348461B
:1008E000042205A9043700F035FB8146E7E73846C6
:1008F00000F056F90590F2E7CDF81490042105A810
:1009000000F01CF900E70023642104A8049300F020
:100910000BF900287FF4AEAE0220FFF759FD002846
:100920003FF4A8AE049800F06BF90590E6E70023C9
:10093000642104A8049300F0F7F800287FF49AAE2D
:100940000220FFF745FD00283FF494AE049800F024
:1009500067F9EAE70220FFF73BFD00283FF48AAE83
:1009600000F076F9E1E70220FFF732FD00283FF4BE
:1009700081AE05A9142000F071F907460421049006
:1009800004A800F0DBF83946B9E7322000F0B8F8E7
:10099000071EFFF66FAEBB077FF46CAE384A07EB5D
:1009A0000A03926893423FF665AE0220FFF710FDFE
:1009B00000283FF45FAE27F003075744BA453FF4E1
:1009C000A3AE50460AF1040A00F0EAF804210590AB
:1009D00005A800F0B3F8F1E74FF47A70FFF7F8FCE0
:1009E00000283FF447AE00F023F9002844D00A9BCA
:1009F00001330BD008220AA9002000F0C3F9002817
:100A00003AD02022FF210AA800F0B4F9FFF7E8FC51
:100A10001C4801F0EDFA13B0BDE8F08F002E3FF452
:100A200029AE0BF00B030B2B7FF424AE00236421C3
:100A300005A8059300F078F8074600287FF41AAE61
:100A40000220FFF7C5FC814600283FF413AEFFF7F4
:100A5000C7FC41F2883001F0CBFA059800F018FA93
:100A60004E463C4600F0D2F9B6E506464CE64FF05D
:100A7000000AFFE5B8467BE6374679E68022022089
:100A800000220220A0860100F7B50C46184E4FF454
:100A90007A71054602FB01F396F90020501C0BD138
:100AA0001448294601930268176A2246B8478442CF
:100AB000019B03D1002310E0002AF1D096F9002019
:100AC000511C01D0012A0DD10B4829460268166A33
:100AD0002246B047844205D10123084A0120137001
:100AE00003B0F0BD4FF4FA7001F082FA0020F7E78E
:100AF00010220220F8270220D4230220D023022033
:100B0000002307B5024601210DF107008DF80730DB
:100B1000FFF7BAFF20B19DF8070003B05DF804FBB2
:100B20004FF0FF30F9E700000A46042108B5FFF74F
:100B3000ABFF80F00100C0B2404208BD074B0A463F
:100B400030B41978064B53F82140014623682046FB
:100B5000DD69044BAC4630BC604700BFD0230220A7
:100B6000BC3B0008A086010070B50A4E00240A4D67
:100B700001F0DEFC308028683388834208D901F018
:100B8000D1FC2B6804440133B4F5C03F2B60F2D391
:100B900070BD00BFD22302208C23022001F08ABD49
:100BA00000F1006000F5C0300068704700F100609F
:100BB000920000F5C03001F009BD0000054B1A6835
:100BC000054B1B889B1A834202D9104401F0AABC32
:100BD000002070478C230220D223022038B5074D15
:100BE00004462868204401F0A5FC28B92868204460
:100BF000BDE8384001F0B6BC38BD00BF8C230220F0
:100C000010F0030309D1B0F5846F04D200F1005055
:100C1000A0F571200368184670470023FBE7000029
:100C200000F10050A0F57120D0F8200470470000BA
:100C3000064991F8243033B100230822086A81F86C
:100C40002430FFF7B3BF0120704700BF902302207C
:100C5000014B1868704700BF002004E0204B02469B
:100C6000F0B518681F4BC0F30B06000C1F885D68B9
:100C7000BE4293F9084022D09F89BE4221D01F8BEB
:100C8000BE4206D102240C2505FB04335D6893F9AE
:100C90000840B0F5805F16D041F20103984208BFCA
:100CA0005A24013A013D0B460A4493420DD215F9EC
:100CB000016F581C5EB1034600F8016CF5E7002493
:100CC000E1E70124DFE74124EBE7184605E02C25A6
:100CD00090421D7001D2981C5C70401AF0BD00BF9C
:100CE000002004E01422022000207047022803D1D3
:100CF000024B4FF080629A61704700BF000C0240C7
:100D0000022803D1024B4FF480629A61704700BF02
:100D1000000C0240022804D1024A536983F4806324
:100D200053617047000C0240002310B5934203D07A
:100D3000CC5CC4540133F9E710BD0000013810B594
:100D400010F9013F3BB191F900409C4203D11AB127
:100D50000131013AF4E71AB191F90020981A10BD57
:100D60001046FCE703460246D01A12F9011B00297F
:100D7000FAD1704702440346934202D003F8011BA4
:100D8000FAE770472DE9F8431F4D14460746884699
:100D900095F8242052BBDFF870909CB395F824306E
:100DA0002BB92022FF2148462F62FFF7E3FF95F879
:100DB00024004146C0F1080205EB8000A24228BF92
:100DC0002246D6B29200FFF7AFFF95F82430A41B5D
:100DD00017441E449044E4B2F6B2082E85F824600D
:100DE000DBD1FFF725FF0028D7D108E02B6A03EB02
:100DF00082038342CFD0FFF71BFF0028CBD1002016
:100E0000BDE8F8830120FBE790230220024B1A780B
:100E1000024B1A70704700BFD0230220102202201C
:100E200038B5154C154D204600F0F0FB29462046FC
:100E300000F018FC2D681248EA6ED2F8043843F02E
:100E40000203C2F8043801F0D3F80E49284600F036
:100E500011FDEA6E0C48D2F804380C49A04223F088
:100E60000203C2F804384FF4E1330B6003D0BDE84D
:100E7000384000F02BBB38BDF8270220C83C0008E2
:100E800040420F00D03C0008D4230220B8230220A7
:100E900038B50B4B04461A780A4B53F822500A4BCC
:100EA0009D420CD0094B002118221846FFF762FF23
:100EB000046001462846BDE8384000F007BB38BD55
:100EC000D0230220BC3B0008F8270220B8230220D0
:100ED00000B59BB0EFF3098168226846FFF724FF55
:100EE000EFF30583044B9A6BDA6A9A6A9A6A9A6AF4
:100EF0009A6A9A6A9B6AFEE700ED00E000B59BB033
:100F0000EFF3098168226846FFF70EFFEFF30583D0
:100F1000044B9A6B9A6A9A6A9A6A9A6A9A6A9B6A64
:100F2000FEE700BF00ED00E000B59BB0EFF30981E4
:100F300068226846FFF7F8FEEFF30583034B5A6B10
:100F40009A6A9A6A9A6A9A6A9B6AFEE700ED00E0DA
:100F5000FEE7000030B50A44084D91420DD011F86B
:100F6000013B5840082340F30004013B2C4013F0A0
:100F7000FF0384EA5000F6D1EFE730BD2083B8EDDF
:100F8000026843681143016003B1184770470000CD
:100F9000024A136843F0C0031360704700780040B2
:100FA00013B50E4C204600F085FA04F1140000231E
:100FB0004FF480720A49009400F046F9094B4FF44F
:100FC0008072094904F13800009400F0BFF9074A23
:100FD000074BC4E9172302B010BD00BFD423022081
:100FE00040240220910F0008402502200078004094
:100FF00080F93703037C30B5214C002918BF0C461B
:10100000012B0CD11F4B984209D11F4B1A6C42F097
:1010100080421A641A6E42F080421A661B6E226881
:10102000036EC16D03EB52038466B3FBF2F3626897
:10103000150442BF23F0070503F0070343EA450305
:10104000CB60A36843F040034B60E36843F00103C7
:101050008B6042F4967343F001030B604FF0FF3353
:101060000B62510505D512F0102205D0B2F1805F58
:1010700004D080F8643030BD7F23FAE73F23F8E7DF
:10108000C43B0008D4230220003802402DE9F04779
:10109000C66D05463768F4692107346219D014F02B
:1010A000080118BF8021E20748BF41F02001A307D3
:1010B0004FF0200348BF41F04001600748BF41F4B2
:1010C000807183F31188281DFFF75AFF002383F3F3
:1010D0001188E2050AD5202383F311884FF40071AB
:1010E000281DFFF74DFF002383F311884FF02009DF
:1010F0004FF0000A14F0200838D13B0616D54FF007
:10110000200905F1380A200610D589F311885046C8
:1011100000F050F9002836DA0821281DFFF730FFCB
:1011200027F080033360002383F31188790614D5F8
:10113000620612D5202383F31188D5E913239A423E
:1011400008D12B6C33B127F040071021281DFFF781
:1011500017FF3760002383F31188E30618D5AA6EC2
:101160001369ABB15069BDE8F047184789F311889E
:10117000736A284695F86410194000F0B5F98AF3AF
:101180001188F469B6E7B06288F31188F469BAE7A8
:10119000BDE8F087F8B51546826804460B46AA42BA
:1011A00000D28568A1692669761AB5420BD2184625
:1011B0002A46FFF7B9FDA3692B44A3612846A3681B
:1011C0005B1BA360F8BD0CD9AF1B18463246FFF776
:1011D000ABFD3A46E1683044FFF7A6FDE3683B44C7
:1011E000EBE718462A46FFF79FFDE368E5E70000B6
:1011F00083689342F7B50446154600D28568D4E962
:101200000460361AB5420BD22A46FFF78DFD63699A
:101210002B4463612846A3685B1BA36003B0F0BD49
:101220000DD93246AF1B0191FFF77EFD01993A4679
:10123000E0683144FFF778FDE3683B44E9E72A467C
:10124000FFF772FDE368E4E710B50A440024C361C8
:10125000029B8460C16002610362C0E90000C0E9D2
:10126000051110BD08B5D0E90532934201D182685D
:1012700082B98268013282605A1C42611970002171
:10128000D0E904329A4224BFC368436100F0CCFE27
:10129000002008BD4FF0FF30FBE7000070B52023B1
:1012A00004460E4683F31188A568A5B1A368A26918
:1012B000013BA360531CA36115782269934224BFAC
:1012C000E368A361E3690BB120469847002383F3E9
:1012D0001188284607E03146204600F095FE002898
:1012E000E2DA85F3118870BD2DE9F74F04460E460A
:1012F00017469846D0F81C904FF0200A8AF31188C0
:101300004FF0000B154665B12A4631462046FFF7DF
:1013100041FF034660B94146204600F075FE0028B3
:10132000F1D0002383F31188781B03B0BDE8F08F60
:10133000B9F1000F03D001902046C847019B8BF301
:101340001188ED1A1E448AF31188DCE7C160C3617D
:10135000009B82600362C0E905111144C0E90000EE
:1013600001617047F8B504460D461646202383F305
:101370001188A768A7B1A368013BA36063695A1CE1
:1013800062611D70D4E904329A4224BFE36863614C
:10139000E3690BB120469847002080F3118807E0ED
:1013A0003146204600F030FE0028E2DA87F311884B
:1013B000F8BD0000D0E9052310B59A4201D182683A
:1013C0007AB982680021013282605A1C82611C78DD
:1013D00003699A4224BFC368836100F025FE20465A
:1013E00010BD4FF0FF30FBE72DE9F74F04460E46E6
:1013F00017469846D0F81C904FF0200A8AF31188BF
:101400004FF0000B154665B12A4631462046FFF7DE
:10141000EFFE034660B94146204600F0F5FD002886
:10142000F1D0002383F31188781B03B0BDE8F08F5F
:10143000B9F1000F03D001902046C847019B8BF300
:101440001188ED1A1E448AF31188DCE702684368AC
:101450001143016003B11847704700001430FFF7D3
:1014600043BF00004FF0FF331430FFF73DBF0000D3
:101470003830FFF7B9BF00004FF0FF333830FFF7C7
:10148000B3BF00001430FFF709BF00004FF0FF3179
:101490001430FFF703BF00003830FFF763BF0000D0
:1014A0004FF0FF323830FFF75DBF0000002070477B
:1014B000FFF776BD044B036000234360C0E90233AD
:1014C00001230374704700BFDC3B000810B52023E4
:1014D000044683F31188FFF78DFD02232374002354
:1014E00083F3118810BD000038B5C36904460D466A
:1014F0001BB904210844FFF7A9FF294604F1140091
:10150000FFF7B0FE002806DA201D4FF48061BDE829
:101510003840FFF79BBF38BD026843681143016044
:1015200003B118477047000013B5446BD4F8A438D2
:101530001A681178042915D1217C022912D1197950
:10154000012312898B4013420CD101A904F14C00F4
:1015500001F096FFD4F8A4480246019B2179206847
:1015600000F0D4F902B010BD143001F019BF000032
:101570004FF0FF33143001F013BF00004C3001F086
:10158000EBBF00004FF0FF334C3001F0E5BF00002F
:10159000143001F0E7BE00004FF0FF31143001F0CD
:1015A000E1BE00004C3001F0B7BF00004FF0FF3249
:1015B0004C3001F0B1BF000000207047D0F8A438D3
:1015C0001A6810B511780446042917D1017C022944
:1015D00014D15979012352898B4013420ED1143012
:1015E00001F07AFE024648B1D4F8A4484FF4807363
:1015F00061792068BDE8104000F076B910BD0000A8
:10160000406BFFF7DBBF0000704700007FB5124B57
:1016100001250426044603600023057400F18402BA
:1016200043602946C0E902330C4B02901430019309
:101630004FF48073009601F02BFE094B04F29442A4
:10164000294604F14C000294CDE900634FF4807305
:1016500001F0F2FE04B070BD043C00080116000861
:10166000291500080B68202282F311880A7903EB00
:10167000820210624A790D3243F822008A7912B14F
:1016800003EB820318620223C0F8A418037400233A
:1016900083F311887047000038B5037F044613B107
:1016A00090F85430ABB90125201D0221FFF734FF1B
:1016B00004F114006FF00101257700F0C1FC04F182
:1016C0004C0084F854506FF00101BDE8384000F040
:1016D000B7BC38BD10B5012104460430FFF71CFF2C
:1016E0000023237784F8543010BD000038B5044639
:1016F0000025143001F0E4FD04F14C00257701F0E1
:10170000B3FE201D84F854500121FFF705FF204649
:10171000BDE83840FFF752BF90F85C3003F060033B
:10172000202B06D190F85D200023212A03D81F2A00
:1017300006D800207047222AFBD1C0E9143303E009
:10174000034A02650722426583650120704700BF96
:1017500038220220D0F8A43837B51A680446117828
:1017600004291AD1017C022917D119790123128980
:101770008B40134211D100F14C05284601F034FF93
:1017800058B101A9284601F07BFED4F8A4480246CE
:10179000019B2179206800F0B9F803B030BD00004A
:1017A00000EB8103F0B51E6A85B004460D46FEB11C
:1017B000202383F3118804EB8507301D0821FFF7F0
:1017C000ABFEFB6806F14C005B691B681BB1019026
:1017D00001F064FE019803A901F052FE024648B1EF
:1017E000039B2946204600F091F8002383F31188DB
:1017F00005B0F0BDFB685A691268002AF5D01B8A53
:10180000013B1340F1D104F15C02EAE70D3138B538
:1018100050F82140DCB1202383F31188D4F8A428A8
:101820001368527903EB8203DB689B695D6845B1FD
:1018300004216018FFF770FE294604F1140001F03E
:1018400055FD2046FFF7BAFE002383F3118838BD0B
:101850007047000001F0EEB801232822002110B5E6
:10186000044600F8243BFFF785FA0023C4E901335E
:1018700010BD000038B50446202383F311880025ED
:101880004160C0E90355C0E90555C0E9075501F0BD
:10189000E1F80223237085F3118838BD70B500EBA1
:1018A0008103054650690E461446DA6018B11022CD
:1018B0000021FFF75FFAA06918B110220021FFF79D
:1018C00059FA31462846BDE8704001F08DB9000054
:1018D000826802F0011282600022C0E90422C0E99D
:1018E0000622026201F00CBAF0B4012500EB81047B
:1018F00047898D40E4683D43A46945812360002306
:10190000A2606360F0BC01F027BA0000F0B40125CA
:1019100000EB810407898D40E4683D4364690581DB
:1019200023600023A2606360F0BC01F0A1BA000054
:1019300070B502230025044603704566056280F8F1
:101940004C50C0E90255C0E90455C0E9065501F004
:10195000E7F863681B6823B129462046BDE870405C
:10196000184770BD037880F868300523037043681A
:101970001B6810B504460BB1042198470023A360EF
:1019800010BD000090F86820436802701B680BB11E
:10199000052118477047000070B590F84C30044698
:1019A00013B1002380F84C3004F15C02204601F0B2
:1019B000C9F963689B68B3B994F85C3013F06005AB
:1019C00035D00021204601F02FFC0021204601F0F7
:1019D00021FC63681B6813B1062120469847062343
:1019E00084F84C3070BD204698470028E4D0B4F805
:1019F0006230626D9A4288BF636594F95C30656DB0
:101A0000002B4FF0200380F20381002D00F0F280C4
:101A1000092284F84C2083F3118800212046D4E960
:101A20001423FFF773FF002383F31188DAE794F898
:101A30005D2003F07F0343EA022340F20232934227
:101A400000F0C58021D8B3F5807F48D00DD8012B98
:101A50003FD0022B00F09380002BB2D104F164023E
:101A6000226502226265A365C1E7B3F5817F00F0BC
:101A70009B80B3F5407FA4D194F85E30012BA0D1B8
:101A8000B4F8643043F0020332E0B3F5006F4DD098
:101A900017D8B3F5A06F31D0A3F5C063012B90D850
:101AA0006368204694F85E205E6894F85F10B4F88E
:101AB0006030B047002884D04368236503686365BD
:101AC0001AE0B3F5106F36D040F6024293427FF42D
:101AD00078AF5C4B2365022363650023C3E794F86A
:101AE0005E30012B7FF46DAFB4F8643023F0020355
:101AF000A4F86430C4E91455A56578E7B4F85C30FF
:101B0000B3F5A06F0ED194F85E30204684F86630AD
:101B100001F05EF863681B6813B101212046984705
:101B2000032323700023C4E914339CE704F1670303
:101B300023650123C3E72378042B10D1202383F3EB
:101B400011882046FFF7C4FE85F3118803216368DE
:101B500084F8675021701B680BB12046984794F8B1
:101B60005E30002BDED084F8673004232370636876
:101B70001B68002BD6D0022120469847D2E794F864
:101B8000603020461D0603F00F010AD501F0CCF8A5
:101B9000012804D002287FF414AF2B4B9AE72B4B7B
:101BA00098E701F0B3F8F3E794F85E30002B7FF488
:101BB00008AF94F8603013F00F01B3D01A06204636
:101BC00002D501F045FBADE701F038FBAAE794F838
:101BD0005E30002B7FF4F5AE94F8603013F00F0107
:101BE000A0D01B06204602D501F01EFB9AE701F0AB
:101BF00011FB97E7142284F84C2083F311882B46BD
:101C00002A4629462046FFF76FFE85F31188E9E64C
:101C10005DB1152284F84C2083F311880021204601
:101C2000D4E91423FFF760FEFDE60B2284F84C2074
:101C300083F311882B462A4629462046FFF766FE85
:101C4000E3E700BF343C00082C3C0008303C0008AF
:101C500038B590F84C300446002B3ED0063BDAB243
:101C60000F2A34D80F2B32D8DFE803F03731310890
:101C7000223231313131313131313737456DB0F8C0
:101C800062309D4214D2C3681B8AB5FBF3F203FB9A
:101C900012556DB9202383F311882B462A46294615
:101CA000FFF734FE85F311880A2384F84C300EE0E8
:101CB000142384F84C30202383F31188002320461A
:101CC0001A461946FFF710FE002383F3118838BD2A
:101CD000836D03B198470023E7E70021204601F018
:101CE000A3FA0021204601F095FA63681B6813B13E
:101CF0000621204698470623D7E7000010B590F844
:101D00004C300446142B29D017D8062B05D001D807
:101D10001BB110BD093B022BFBD80021204601F06E
:101D200083FA0021204601F075FA63681B6813B13D
:101D3000062120469847062319E0152BE9D10B23ED
:101D400080F84C30202383F3118800231A4619466B
:101D5000FFF7DCFD002383F31188DAE7C3689B6992
:101D60005B68002BD5D1836D03B19847002384F8BD
:101D70004C30CEE7024B0022C3E900339A60704733
:101D800040260220002382680374054B1B68996873
:101D90009142FBD25A6803604260106058607047FD
:101DA0004026022008B5202383F31188037C032BEF
:101DB00005D0042B0DD02BB983F3118808BD4369DE
:101DC00000221A604FF0FF334361FFF7DBFF00236F
:101DD000F2E7D0E9003213605A60F3E7002382682B
:101DE0000374054B1B6899689142FBD85A680360DD
:101DF000426010605860704740260220054B196908
:101E000008741868026853601A601861012303742B
:101E1000FEF78CBA402602204B1C30B5044687B032
:101E20000A4D10D02B6901A8094A00F025F9204677
:101E3000FFF7E4FF049B13B101A800F059F92B69E7
:101E4000586907B030BDFFF7D9FFF8E740260220F8
:101E5000A51D000838B50C4D044641612B69816809
:101E60009A68914203D8BDE83840FFF78BBF184607
:101E7000FFF7B4FF01232C61014623742046BDE81F
:101E80003840FEF753BA00BF40260220044B1A68C0
:101E90001B6990689B68984294BF0020012070479E
:101EA0004026022010B5084C236820691A68546047
:101EB0002260012223611A74FFF790FF0146206916
:101EC000BDE81040FEF732BA4026022008B5FFF701
:101ED000DDFF18B1BDE80840FFF7E4BF08BD000012
:101EE000FFF7E0BFFEE7000010B50C4CFFF742FF24
:101EF00000F0B4F880220A49204600F03BF80123A4
:101F000044F8180C037400F071FC002383F311886B
:101F100062B60448BDE8104000F04CB868260220C4
:101F2000383C0008483C000800F01CB9EFF3118071
:101F300020B9EFF30583202282F311887047000057
:101F400010B530B9EFF30584C4F3080414B180F37D
:101F5000118810BDFFF7BAFF84F31188F9E700007C
:101F6000034A516853685B1A9842FBD8704700BF18
:101F7000001000E082600222028270478368A3F1B1
:101F80007C0243F80C2C026943F83C2C426943F86C
:101F9000382C074A43F81C2CC268A3F1180043F8F8
:101FA000102C022203F8082C002203F8072C70479B
:101FB0004503000810B5202383F31188FFF7DEFFE7
:101FC00000210446FFF746FF002383F311882046D3
:101FD00010BD0000024B1B6958610F20FFF70EBFB8
:101FE00040260220202383F31188FFF7F3BF00006F
:101FF00008B50146202383F311880820FFF70CFF62
:10200000002383F3118808BD49B1064B42681B6960
:1020100018605A60136043600420FFF7FDBE4FF064
:10202000FF307047402602200368984206D01A68A5
:102030000260506018465961FFF7A4BE7047000067
:1020400038B504460D462068844200D138BD036887
:1020500023605C604561FFF795FEF4E7054B4FF0A8
:10206000FF3103F11402C3E905220022C3E907127C
:10207000704700BF4026022070B51C4E05460C4636
:10208000C0E9032301F0E2FA334653F8142F9A42D1
:102090000DD130620A2C2CBF00190A302A60C5E924
:1020A0000124C6E90555BDE8704001F0BDBA316AAA
:1020B000431AE31838BF1C469368A34202D9081993
:1020C00001F0C0FA73699A6894420CD85A68AC60FF
:1020D0002B606A6015609A685D60121B9A604FF011
:1020E000FF33F36170BDA41A1B68ECE740260220A1
:1020F00038B51B4C636998420DD08168D0E9003235
:1021000013605A600022C2609A680A449A604FF0D5
:10211000FF33E36138BD03682246002142F8143FD3
:1021200093425A60C16003D1BDE8384001F084BADF
:102130009A688168256A0A449A6001F087FA63699F
:10214000411B9A688A42E5D9AB181D1A206A092DED
:1021500098BF01F10A02BDE83840104401F072BA9C
:10216000402602202DE9F041184C002704F1140606
:10217000656901F06BFA236AAA68C11A8A4215D808
:102180001344D5F80C802362D5E9003213605A60FD
:102190006369EF60B34201D101F04EFA87F3118811
:1021A0002869C047202383F31188E1E76169B142C0
:1021B00009D013441B1ABDE8F0410A2B2CBFC018EC
:1021C0000A3001F03FBABDE8F08100BF402602208E
:1021D00000207047FEE70000704700004FF0FF301E
:1021E0007047000002290CD0032904D001290748B8
:1021F00018BF00207047032A05D8054800EBC2002D
:102200007047044870470020704700BF2C3D00080D
:1022100048220220E03C000870B59AB00546084606
:10222000144601A900F0C2F801A8FEF79BFD431C6B
:102230000022C6B25B001046C5E9003423700323B8
:10224000023404F8013C01ABD1B202348E4201D811
:102250001AB070BD13F8011B013204F8010C04F828
:10226000021CF1E708B5202383F311880348FFF728
:1022700071FA002383F3118808BD00BFF8270220FC
:1022800090F85C3003F01F02012A07D190F85D201E
:102290000B2A03D10023C0E9143315E003F06003D7
:1022A000202B08D1B0F860302BB990F85D20212A9E
:1022B00003D81F2A04D8FFF72FBA222AEBD0FAE757
:1022C000034A02650722426583650120704700BF0B
:1022D0003F22022007B5052917D8DFE801F01916BB
:1022E00003191920202383F31188104A012101903A
:1022F000FFF7D4FA019802210D4AFFF7CFFA0D48F3
:10230000FFF7F4F9002383F3118803B05DF804FBB1
:10231000202383F311880748FFF7BEF9F2E7202353
:1023200083F311880348FFF7D5F9EBE7803C0008F9
:10233000A43C0008F827022038B50C4D0C4C2A4666
:102340000C4904F10800FFF767FF05F1CA0204F128
:1023500010000949FFF760FF05F5CA7204F1180083
:102360000649BDE83840FFF757BF00BFD030022014
:1023700048220220603C00086A3C0008753C0008C6
:1023800070B5044608460D46FEF7ECFCC6B2204682
:10239000013403780BB9184670BD32462946FEF762
:1023A000CDFC0028F3D10120F6E700002DE9F0472D
:1023B00005460C46FEF7D6FC2B49C6B22846FFF769
:1023C000DFFF08B10736F6B228492846FFF7D8FFE5
:1023D00008B11036F6B2632E0BD8DFF88C80DFF828
:1023E0008C90234FDFF894A02E7846B92670BDE874
:1023F000F08729462046BDE8F04701F0C1BB252EF5
:102400002ED1072241462846FEF798FC70B9194B99
:10241000224603F10C0153F8040B8B4242F8040BE3
:10242000F9D11B8807350E341380DDE708224946B1
:102430002846FEF783FC98B9A21C0F4B197802328C
:102440000909C95D02F8041C13F8011B01F00F0112
:102450005345C95D02F8031CF0D118340835C3E7B1
:10246000013504F8016BBFE74C3D0008753C0008DE
:10247000633D0008543D000820F4F01F2CF4F01FC9
:10248000BFF34F8F024AD368DB03FCD4704700BF11
:10249000003C024008B5074B1B7853B9FFF7F0FF2B
:1024A000054B1A69002A04DA044A5A6002F188329C
:1024B0005A6008BD2E330220003C024023016745CC
:1024C00008B5054B1B7833B9FFF7DAFF034A1369E8
:1024D00043F00043136108BD2E330220003C02404C
:1024E0000B28F0B516D80C4C0C4923787BB90E4656
:1024F0000B4D0C234FF00062013B55F8047B46F86E
:10250000042B13F0FF033A44F6D10123237051F852
:102510002000F0BD0020FCE76033022030330220B1
:10252000743D0008014B53F820007047743D0008CB
:102530000C2070470B2810B5044601D9002010BDAF
:10254000FFF7CEFF064B53F824301844C21A0BB9DC
:102550000120F4E712680132F0D1043BF6E700BF36
:10256000743D00080B2838B5044628D8FFF7DEFC78
:102570000546FFF785FF2046FFF78CFF114AF3233E
:10258000D360E300DBB243F4007343F00203136152
:10259000136943F480331361FFF772FFFFF7A0FF65
:1025A000094B53F8241000F0E9F82846FFF788FF9C
:1025B000FFF7C6FC2046BDE83840FFF7BBBF002050
:1025C00038BD00BF003C0240743D000812F001031A
:1025D0002DE9F04105460E4614464BD18218B2F162
:1025E000026F61D8314B1B6813F001035CD0FFF719
:1025F0009DFC2F4FFFF74EFFF323314640F2012899
:10260000FB60FFF73DFF032C18D824F001046D1A7E
:10261000274E40F201180C44A14205EB0107336933
:102620002AD123F001033361FFF74AFFFFF788FC4B
:102630000120BDE8F081043C0435E4E7AB07E4D1B8
:102640003B6923F440733B613B6943EA08033B6108
:1026500051F8046B2E60BFF34F8FFFF711FF2B680B
:102660009E42E8D03B6923F001033B61FFF728FF5E
:10267000FFF766FC0020DCE723F440733361336925
:1026800043EA080333610B883B80BFF34F8FFFF7AA
:10269000F7FE3F88BFB231F8023BBB42BCD0336982
:1026A00023F001033361E1E71846C2E70038024036
:1026B000003C0240084908B50B7828B11BB9FFF768
:1026C000E9FE01230B7008BD002BFCD00870BDE8AB
:1026D0000840FFF7F5BE00BF2E3302200244074B2F
:1026E000D2B210B5904200D110BD441C00B253F8D4
:1026F000200041F8040BE0B2F4E700BF502800408E
:102700000F4B30B51C6F240407D41C6F44F40074C5
:102710001C671C6F44F400441C670A4C0244236885
:10272000D2B243F480732360074B904200D130BD96
:10273000441C51F8045B00B243F82050E0B2F4E7C7
:1027400000380240007000405028004007B50122C8
:1027500001A90020FFF7C2FF019803B05DF804FB58
:1027600013B50446FFF7F2FFA04205D0012201A9EC
:1027700000200194FFF7C4FF02B010BD0144BFF375
:102780004F8F064B884204D3BFF34F8FBFF36F8F39
:102790007047C3F85C022030F4E700BF00ED00E0B2
:1027A000034B1A681AB9034AD2F874281A607047A2
:1027B000643302200030024008B5FFF7F1FF024BFE
:1027C0001868C0F3407008BD64330220EFF309833A
:1027D000054968334A6B22F001024A6383F3098892
:1027E000002383F31188704700EF00E0202080F37E
:1027F000118862B60D4B0E4AD96821F4E0610904D4
:10280000090C0A430B49DA60D3F8FC2042F08072CD
:10281000C3F8FC20084AC2F8B01F116841F001015A
:1028200011601022DA7783F82200704700ED00E093
:102830000003FA0555CEACC5001000E0202310B50A
:1028400083F311880E4B5B6813F4006314D0F1EE30
:10285000103AEFF309844FF08073683CE361094B51
:10286000DB6B236684F30988FFF710FB10B1064B7E
:10287000A36110BD054BFBE783F31188F9E700BFA7
:1028800000ED00E000EF00E0570300085A030008E5
:1028900070B5BFF34F8FBFF36F8F1A4A0021C2F894
:1028A0005012BFF34F8FBFF36F8F536943F4003360
:1028B0005361BFF34F8FBFF36F8FC2F88410BFF324
:1028C0004F8FD2F8803043F6E074C3F3C900C3F3EE
:1028D0004E335B0103EA0406014646EA817501397D
:1028E000C2F86052F9D2203B13F1200FF2D1BFF3AE
:1028F0004F8F536943F480335361BFF34F8FBFF35E
:102900006F8F70BD00ED00E0FEE700000A4B0B4842
:102910000B4A90420BD30B4BC11EDA1C121A22F049
:1029200003028B4238BF00220021FEF723BA53F87E
:10293000041B40F8041BECE7703F000878340220C9
:1029400078340220783402207047000070B5D0E956
:102950001B4300224FF0FF359E6804EB42135101E8
:10296000D3F80009002805DAD3F8000940F08040C8
:10297000C3F80009D3F8000B002805DAD3F8000BE0
:1029800040F08040C3F8000B013263189642C3F850
:102990000859C3F8085BE0D24FF00113C4F81C38A3
:1029A00070BD00001D4B03EB8002D2F80CC02DE976
:1029B000F043DCF81420461CDD6ED2F800E005EB95
:1029C000063605EB4018516871450AD30122D5F847
:1029D000343802FA00F023EA0000C5F83408BDE8F4
:1029E000F083AEEB0103BCF81040A34228BF23469E
:1029F000D8F81849A4B2B3EB840FF0D89468A4F1C6
:102A0000040959F8047F3760A4EB09071F44042F19
:102A1000F7D81C440B4494605360D4E76833022019
:102A2000890141F02001016103699B06FCD4122059
:102A3000FFF796BA10B5054C2046FEF70DFF4FF094
:102A4000A043E366024B236710BD00BF683302203A
:102A5000C83D000870B503780546012B50D12A4BBC
:102A6000C46E98421BD1294B0E2143205A6B42F071
:102A700080025A635A6D42F080025A655A6D5A6953
:102A800042F080025A615A6922F080025A615B6901
:102A900000F0E8FB1E4BE3601E4BC4F80038002337
:102AA000EE6EC4F8003EC02323604FF40413A3630A
:102AB0003369002BFCDA01230C203361FFF750FA55
:102AC0003369DB07FCD41220FFF74AFA3369002B85
:102AD000FCDA00262846A660FFF738FF6B68C4F8CA
:102AE0001068DB68C4F81468C4F81C684BB90A4B5A
:102AF000A3614FF0FF336361A36843F00103A36058
:102B000070BD064BF4E700BF683302200038024076
:102B10004014004003002002003C30C0083C30C09C
:102B2000F8B5C46E054600214FF000662046FFF759
:102B300077FF296F00234FF001128F684FF0FF30AD
:102B4000C4F83438C4F81C2804EB431201339F4204
:102B5000C2F80069C2F8006BC2F80809C2F8080B95
:102B6000F2D20B68EA6E6B67636210231361166919
:102B700016F01006FBD11220FFF7F2F9D4F8003856
:102B800023F4FE63C4F80038A36943F4402343F000
:102B90001003A3610923C4F81038C4F814380A4B91
:102BA000EB604FF0C043C4F8103B084BC4F8003B47
:102BB000C4F81069C4F800396B6F03F1100243F4D4
:102BC00080136A67A362F8BDA43D0008408000102E
:102BD000C26E90F86610D2F8003823F4FE6343EA20
:102BE0000113C2F8003870472DE9F84300EB810368
:102BF000C56E0C468046DA680FFA81F948011668FE
:102C000006F00306731E022B05EB41134FF0000183
:102C100094BFB604384EC3F8101B4FF0010104F105
:102C2000100398BF06F1805601FA03F3916998BF2B
:102C300006F5004600293AD0578A04F15801374377
:102C400049016F50D5F81C180B430021C5F81C38FA
:102C50002B180127C3F81019A7405369611E9BB3B5
:102C6000138A928B9B08012A88BF5343D8F874209B
:102C7000981842EA034301F140022146C8F8740063
:102C8000284605EB82025360FFF7CAFE08EB890075
:102C9000C3681B8A43EA845348341E4364012E519F
:102CA000D5F81C381F43C5F81C78BDE8F88305EB40
:102CB0004917D7F8001B21F40041C7F8001BD5F8CD
:102CC0001C1821EA0303C0E704F13F030B4A28461E
:102CD000214605EB83035A60FFF7A2FE05EB49107E
:102CE000D0F8003923F40043C0F80039D5F81C3877
:102CF00023EA0707D7E700BF0080001000040002A6
:102D0000026F12684267FFF721BE00005831C36EA0
:102D100049015B5813F4004004D013F4001F0CBFAA
:102D200002200120704700004831C36E49015B5802
:102D300013F4004004D013F4001F0CBF0220012044
:102D40007047000000EB8101CB68196A0B681360C3
:102D50004B6853607047000000EB810330B5DD68BD
:102D6000AA691368D36019B9402B84BF402313604C
:102D70006B8A1468C26E1C4402EB4110013C09B21C
:102D8000B4FBF3F46343033323F0030343EAC44384
:102D900043F0C043C0F8103B2B6803F00303012B42
:102DA0000ED1D2F8083802EB411013F4807FD0F82E
:102DB000003B14BF43F0805343F00053C0F8003B86
:102DC00002EB4112D2F8003B43F00443C2F8003B4F
:102DD00030BD00002DE9F041244D0446EE6E06EBB7
:102DE0004013D3F8087B3807C3F8087B0AD5D6F818
:102DF0001438190706D505EB840321462846DB68FD
:102E00005B689847FA071FD5D6F81438DB071BD53F
:102E100005EB8403D968CCB98B69488A5A68B2FB40
:102E2000F0F600FB16228AB91868DA6890420DD2D3
:102E3000121AC3E90024202383F311880B4821468A
:102E4000FFF78AFF84F31188BDE8F081012303FABC
:102E500004F26B8923EA02036B81CB68002BF3D069
:102E600021460248BDE8F041184700BF6833022000
:102E700000EB81034A0170B5DD68C36E6C6926689A
:102E8000E66056BB1A444FF40020C2F810092A68C5
:102E900002F00302012A0AB20ED1D3F8080803EBAC
:102EA000421410F4807FD4F8000914BF40F0805021
:102EB00040F00050C4F8000903EB4212D2F80009B8
:102EC00040F00440C2F800090122D3F8340802FAA5
:102ED00001F10143C3F8341870BD19B9402E84BF05
:102EE0004020206020681A442E8A8419013CB4FBDB
:102EF000F6F440EAC44040F00050C6E7F8B5044696
:102F00001E48C56E05EB4413D3F80869F107C3F8F2
:102F1000086917D5D5F81038DA0713D500EB840304
:102F2000D9684B691F68DA68974218D2D21B00270C
:102F30001A605F60202383F311882146FFF798FF12
:102F400087F31188330617D50123D5F83428A34019
:102F5000134211D02046BDE8F840FFF723BD0123FE
:102F600003FA04F2038923EA020303818B68002B2E
:102F7000E8D021469847E5E7F8BD00BF6833022056
:102F80002DE9F74FA24CE66E7569B3691D4015F443
:102F90008058756107D02046FEF7CAFC03B0BDE833
:102FA000F04FFFF74BBC002D12DAD6F8003E9F071A
:102FB00005D0D6F8003E23F00303C6F8003ED6F84D
:102FC0000438934823F00103C6F80438FEF7DAFC0E
:102FD000280505D58E48FFF7B9FC8D48FEF7C2FCE1
:102FE000A9040CD5D6F8083813F0060FF36823F4BB
:102FF00070530CBF43F4105343F4A053F3602A07FB
:1030000004D56368DB680BB181489847EB0200F197
:103010008A80AF0227D5D4F86C9000274FF0010AC0
:10302000DFF8ECB109EB4712D2F8003B03F4402380
:10303000B3F5802F11D1D2F8003B002B0DDA628955
:103040000AFA07F322EA0303638104EB8703DB68D0
:10305000DB6813B13946584698470137236FFFB2F2
:103060009B689F42DED9E80618D5E76E3A6AC2F33C
:103070000A1002F00F0302F4F012B2F5802F00F0F4
:103080009C80B2F5402F09D104EB8303002207F5A1
:103090008057DB681B6A904240F082802B03D6F891
:1030A00018481DD5E70302D50020FFF793FEA603BD
:1030B00002D50120FFF78EFE600302D50220FFF744
:1030C00089FE210302D50320FFF784FEE20202D528
:1030D0000420FFF77FFEA30202D50520FFF77AFE4A
:1030E0006F037FF55BAFE60702D50020FFF706FF11
:1030F000A50702D50120FFF701FF600702D50220D6
:10310000FFF7FCFE210702D50320FFF7F7FEE206DA
:1031100002D50420FFF7F2FEA3067FF53FAF05209E
:10312000FFF7ECFE3AE7E36E00274FF0010ADFF805
:10313000E0B00193236F5FFA87F99B6899453FF6EA
:1031400068AF019B03EB4913D3F8002902F4402236
:10315000B2F5802F22D1D3F80029002A1EDAD3F845
:10316000002942F09042C3F80029D3F80029002A30
:10317000FBDB4946E06EFFF753FC22890AFA09F3AC
:1031800022EA0303238104EB8903DB689B6813B104
:103190004946584698474846FFF704FC0137C9E7B7
:1031A000910701D1D7F80080072A02F101029CBFE4
:1031B00003F8018B4FEA18286DE7023307F58057B3
:1031C00004EB83025268D2F818C0DCF80820DCE96E
:1031D000001CA1EB0C0C002188420AD104EB8304F3
:1031E00063689B699A6802449A605A6802445A600C
:1031F00054E711F0030F01D1D7F800808C4501F19D
:10320000010184BF02F8018B4FEA1828E4E700BFF0
:1032100068330220C36E03EB4111D1F8003B43F445
:103220000013C1F8003B7047C36E03EB4111D1F8A6
:10323000003943F40013C1F800397047C36E03EB43
:103240004111D1F8003B23F40013C1F8003B704753
:10325000C36E03EB4111D1F8003923F40013C1F818
:1032600000397047090100F16043012203F5614311
:10327000C9B283F8001300F01F039A4043099B0072
:1032800003F1604303F56143C3F880211A6070477E
:1032900030B50433039C0172002104FB0325C16097
:1032A000C0E90653049B0363059BC0E90000C0E925
:1032B0000422C0E90842C0E90A11436330BD00009E
:1032C0000022416AC260C0E90411C0E90A226FF01D
:1032D0000101FEF7B5BE0000D0E90432934201D1EE
:1032E000C2680AB9181D7047002070470369196049
:1032F0000021C2680132C260C269134482699342EC
:10330000036124BF436A0361FEF78EBE38B50446ED
:103310000D46E3683BB162690020131D1268A36289
:103320001344E36207E0237A33B929462046FEF7C7
:103330006BFE0028EDDA38BD6FF00100FBE70000FE
:10334000C368C269013BC360436913448269934205
:10335000436124BF436A436100238362036B03B16B
:103360001847704770B52023044683F31188866A96
:103370003EB9FFF7CBFF054618B186F31188284602
:1033800070BDA36AE26A13F8015B9342A36202D3A1
:103390002046FFF7D5FF002383F31188EFE70000F5
:1033A0002DE9F84F04460E46174698464FF020097F
:1033B00089F311880025AA46D4F828B0BBF1000F84
:1033C00009D141462046FFF7A1FF20B18BF31188B8
:1033D0002846BDE8F88FD4E90A12A7EB050B521A6C
:1033E000934528BF9346BBF1400F1BD9334601F1EB
:1033F000400251F8040B914243F8040BF9D1A36A3F
:10340000403640354033A362D4E90A239A4202D3BE
:103410002046FFF795FF8AF31188BD42D8D289F381
:103420001188C9E730465A46FDF77EFCA36A5E4420
:103430005D445B44A362E7E710B5029C043301726C
:1034400004FB0321C460C0E906130023C0E90A336A
:10345000039B0363049BC0E90000C0E90422C0E9A8
:103460000842436310BD0000026A6FF00101C260B0
:10347000426AC0E904220022C0E90A22FEF7E0BD48
:10348000D0E904239A4201D1C26822B9184650F803
:10349000043B0B607047002070470000C3680021A8
:1034A000C2690133C3604369134482699342436133
:1034B00024BF436A4361FEF7B7BD000038B5044638
:1034C0000D46E3683BB1236900201A1DA262E26940
:1034D0001344E36207E0237A33B929462046FEF716
:1034E00093FD0028EDDA38BD6FF00100FBE7000026
:1034F00003691960C268013AC260C26913448269F3
:103500009342036124BF436A036100238362036B18
:1035100003B118477047000070B520230D460446DC
:10352000114683F31188866A2EB9FFF7C7FF10B1E1
:1035300086F3118870BDA36A1D70A36AE26A013325
:103540009342A36204D3E16920460439FFF7D0FF18
:10355000002080F31188EDE72DE9F84F04460D4671
:10356000904699464FF0200A8AF311880026B34608
:10357000A76A4FB949462046FFF7A0FF20B187F35D
:1035800011883046BDE8F88FD4E90A073A1AA8EB4B
:103590000607974228BF1746402F1BD905F1400365
:1035A00055F8042B9D4240F8042BF9D1A36A40360C
:1035B0004033A362D4E90A239A4204D3E169204646
:1035C0000439FFF795FF8BF311884645D9D28AF36A
:1035D0001188CDE729463A46FDF7A6FBA36A3D448C
:1035E0003E443B44A362E5E7D0E904239A4217D165
:1035F000C3689BB1836A8BB1043B9B1A0ED01360E6
:10360000C368013BC360C3691A4483699A4202617B
:1036100024BF436A03610023836201231846704775
:103620000023FBE700F094B84FF08043002258637A
:103630001A610222DA6070474FF080430022DA609C
:10364000704700004FF08043586370474FF080434D
:10365000586A70474B6843608B688360CB68C3606F
:103660000B6943614B6903628B6943620B680360BA
:103670007047000008B52C4B40F2FF712B481A69C7
:103680000A431A611A6922F4FF6222F007021A61E2
:103690001A691A6B0A431A631A6D0A431A65244A97
:1036A0001B6D1146FFF7D6FF00F5806002F11C018B
:1036B000FFF7D0FF00F5806002F13801FFF7CAFF85
:1036C00000F5806002F15401FFF7C4FF00F580604F
:1036D00002F17001FFF7BEFF00F5806002F18C017E
:1036E000FFF7B8FF00F5806002F1A801FFF7B2FF15
:1036F00000F5806002F1C401FFF7ACFF00F58060C7
:1037000002F1E001FFF7A6FF00F5806002F1FC0185
:10371000FFF7A0FF02F58C7100F58060FFF79AFFBC
:10372000BDE8084000F08AB80038024000000240BE
:10373000D43D000808B500F003FAFEF7D5FBFFF70B
:103740002FF8BDE80840FEF7F7BD00007047000005
:103750000F4B1A6C42F001021A641A6E42F0010219
:103760001A660C4A1B6E936843F0010393604FF096
:1037700080436B229A624FF0FF32DA6200229A6134
:103780005A63DA605A6001225A611A60704700BFBA
:1037900000380240002004E04FF0804208B5116973
:1037A000D3680B40D9B29B076FEA0101116107D5BD
:1037B000202383F31188FEF7B7FB002383F31188DE
:1037C00008BD00001B4B4FF0FF3000211A696FEA63
:1037D00042526FEA52521A611A69C2F30A021A611E
:1037E0001A695A6958615A6959615A691A6A62F0C4
:1037F00080521A621A6A02F080521A621A6A5A6A6F
:1038000058625A6A59625A6A0B4A106840F48070CA
:103810001060186F00F44070B0F5007F03D04FF4D3
:10382000803018671967536823F40073536000F001
:103830005FB900BF0038024000700040364B4FF4C3
:103840004041364A1A64364A11601A6842F0010251
:103850001A601A689207FCD59A6822F003029A60EF
:103860002D4B9A6812F00C02FBD1196801F0F90196
:1038700019609A601A6842F480321A601A689003DC
:10388000FCD55A6F42F001025A67234B5A6F9107D9
:10389000FCD5244A5A601A6842F080721A60204BA4
:1038A0005A685204FCD51A6842F480321A605A6889
:1038B000D003FCD51A6842F400321A60184A5368E3
:1038C0009903FCD5144B1A689201FCD5164A9A60EC
:1038D00040F20112C3F88C200022C3F8902040F27D
:1038E0000733124A1360136803F00F03072BFAD152
:1038F000094B9A6842F002029A609A6802F00C0240
:10390000082AFAD15A6C42F480425A645A6E42F440
:1039100080425A665B6E7047003802400004001017
:1039200000700040086C400900948838003C024058
:10393000074A08B5536903F00103536123B1054AEF
:1039400013680BB150689847BDE80840FEF776BF92
:10395000003C0140F8330220074A08B5536903F0E0
:103960000203536123B1054A93680BB1D0689847AD
:10397000BDE80840FEF762BF003C0140F83302207A
:10398000074A08B5536903F00403536123B1054A9C
:1039900013690BB150699847BDE80840FEF74EBF68
:1039A000003C0140F8330220074A08B5536903F090
:1039B0000803536123B1054A93690BB1D069984755
:1039C000BDE80840FEF73ABF003C0140F833022052
:1039D000074A08B5536903F01003536123B1054A40
:1039E000136A0BB1506A9847BDE80840FEF726BF3E
:1039F000003C0140F8330220164B10B55C6904F41A
:103A000078725A61A30604D5134A936A0BB1D06A3F
:103A10009847600604D5104A136B0BB1506B98475A
:103A2000210604D50C4A936B0BB1D06B9847E20585
:103A300004D5094A136C0BB1506C9847A30504D503
:103A4000054A936C0BB1D06C9847BDE81040FEF767
:103A5000F5BE00BF003C0140F8330220194B10B501
:103A60005C6904F47C425A61620504D5164A136D00
:103A70000BB1506D9847230504D5134A936D0BB1D4
:103A8000D06D9847E00404D50F4A136E0BB1506E09
:103A90009847A10404D50C4A936E0BB1D06E984799
:103AA000620404D5084A136F0BB1506F9847230482
:103AB00004D5054A936F0BB1D06F9847BDE810400D
:103AC000FEF7BCBE003C0140F833022008B50348B5
:103AD000FDF7DCFABDE80840FEF7B0BED4230220B3
:103AE00008B5FFF759FEBDE80840FEF7A7BE000085
:103AF000062108B50846FFF7B5FB06210720FFF7AA
:103B0000B1FB06210820FFF7ADFB06210920FFF7D6
:103B1000A9FB06210A20FFF7A5FB06211720FFF7C6
:103B2000A1FB06212820FFF79DFB07211C20FFF7A2
:103B300099FB0C215220BDE80840FFF793BB000021
:103B400008B5FFF73FFE00F00DF8FDF7B1FCFDF7FB
:103B500081FEFDF759FDFFF7F9FDBDE80840FFF7CD
:103B600061BD00000023054A19460133102BC2E94C
:103B7000001102F10802F8D1704700BFF8330220AB
:103B8000034611F8012B03F8012B002AF9D17047E5
:103B900053544D3332463F3F3F3F3F3F0053544D18
:103BA000333246375B347C355D780053544D3332C5
:103BB00046375B367C375D7800000000F82702202E
:103BC000D423022000960000000000000000000046
:103BD00000000000000000000000000000000000E5
:103BE0007914000865140008A11400088D14000859
:103BF0009914000885140008711400085D14000869
:103C0000AD140008000000008515000871150008BB
:103C1000AD15000899150008A515000891150008B4
:103C20007D15000869150008B9150008000000009E
:103C300001000000000000006D61696E00000000DE
:103C400069646C6500000000403C0008802602208A
:103C5000F827022001000000E51E00080000000017
:103C60004172647550696C6F740025424F41524433
:103C7000252D424C002553455249414C250000005A
:103C80000200000000000000A11700080D18000845
:103C900040004000A0300220B030022002000000AE
:103CA00000000000030000000000000051180008A0
:103CB0000000000010000000C030022000000000E2
:103CC0000100000000000000683302200101020032
:103CD000D5220008E521000881220008652200089D
:103CE00043000000E83C000809024300020100C054
:103CF0003209040000010202010005240010010540
:103D000024010001042402020524060001070582A3
:103D1000030800FF09040100020A00000007050172
:103D20000240000007058102400000001200000070
:103D3000343D0008120110010200004009124157F1
:103D400000020102030100000403090425424F415F
:103D5000524425004D6174656B463736352D5769E1
:103D60006E670030313233343536373839414243AB
:103D700044454600008000000080000000800000F4
:103D800000800000000002000000040000000400A9
:103D90000000040000000400000004000000040013
:103DA000000004000000000099190008511C0008E0
:103DB000FD1C000840004000E0330220E0330220F8
:103DC00001000000F03302208000000040010000EC
:103DD000050000000000802A00000000AAAAAAAA8C
:103DE00000000024FFFF00000000000000A00A0007
:103DF0000000000100000000AAAAAAAA0000000119
:103E0000FFFF0000000000000000000000010000B3
:103E100000000000AAAAAAAA00010000FFFF0000FB
:103E20000000000000000000004010000000000042
:103E3000AAAAAAAA00400000FFFB000000000000A0
:103E4000000000000081420000000000AAAAAAAA07
:103E500000404100EFFF000000000080080000006B
:103E60000000000000000000AAAAAAAA00000000AA
:103E7000FFFF000000000000000000000000000044
:103E800000000000AAAAAAAA00000000FFFF00008C
:103E90000000000000000000000000000000000022
:103EA000AAAAAAAA00000000FFFF0000000000006C
:103EB000000000000000000000000000AAAAAAAA5A
:103EC00000000000FFFF00000000000000000000F4
:103ED00000000000000000000000000000000000E2
:103EE00000000000000000000000000000000000D2
:103EF00000000000000000000000000000000000C2
:103F000000000000000000008F0000000000000022
:103F100000801E0000000000FF0000000000000004
:103F2000903B00083F000000490400009D3B000852
:103F30003F00000051040000AB3B00083F000000C0
:103F40000096000000000800960000000008000035
:103F500004000000483D00080000000000000000D0
:103F60000000000000000000000000000000000051
:103F7000FFFFFFFFFFFFFFFFFFFFFFFFFFFFFFFF51
:103F8000FFFFFFFFFFFFFFFFFFFFFFFFFFFFFFFF41
:103F9000FFFFFFFFFFFFFFFFFFFFFFFFFFFFFFFF31
:020000040801F1
:1080000000060220AD8C010891520E086182010821
:1080100019520E0811520E0815520E08AF8C0108A5
:10802000AF8C0108AF8C0108AF8C01082D4B1308F1
:10803000AF8C0108AF8C0108AF8C0108AF8C010830
:10804000AF8C0108AF8C0108AF8C0108AF8C010820
:10805000AF8C0108AF8C0108255813084D58130840
:10806000755813089D581308C558130875F212085F
:108070009DF21208C9F21208F5F2120821F3120853
:1080800049F3120875F31208F9F11208AF8C0108D0
:10809000AF8C0108AF8C0108AF8C0108ED581308B4
:1080A000615A1308755A1308895A13089D5A130800
:1080B000A15A1308B55A1308C95A13088DFA1208A1
:1080C000BDFA1208EDFA12081DFB1208AF8C010868
:1080D000AF8C0108C1591308D5591308E959130881
:1080E00051591308AF8C0108AF8C0108F15A1308DD
:1080F000015B1308155B1308195B1308A1F3120841
:10810000AF8C010805FE1208DD5A1308AF8C010878
:10811000FD591308115A1308AF8C0108AF8C0108E0
:10812000CDF31208F5F3120821F412084DF41208E9
:1081300079F41208AF8C0108AF8C0108AF8C0108EC
:10814000AF8C0108AF8C0108AF8C010835531308C0
:10815000A1F41208CDF41208F9F41208255A1308F4
:10816000AF8C0108AF8C0108AF8C0108AF8C0108FF
:10817000AF8C0108AF8C0108AF8C0108AF8C0108EF
:10818000AF8C0108AF8C0108395A13084D5A1308F7
:10819000AF8C0108AF8C0108AF8C0108AF8C0108CF
:1081A000AF8C0108AF8C0108AF8C0108AF8C0108BF
:1081B000AF8C0108AF8C0108AF8C0108AF8C0108AF
:1081C000AF8C0108AF8C0108AF8C0108AF8C01089F
:1081D000AF8C0108AF8C0108AF8C0108AF8C01088F
:1081E000AF8C0108AF8C0108AF8C0108AF8C01087F
:1081F000AF8C0108AF8C0108AF8C0108AF8C01086F
:1082000071F901088D030408E9F90508C557080844
:10821000195E080875EB0808215A0908E961090880
:108220002965090819DF0908FD0D0A084D410B08E9
:108230005DA10B08B5AE0B08B1440E0895490E08B8
:10824000CD640E08814C1108A1E1110875081208CF
:108250002D141208D5461208A54D12080000000082
:10826000EFF30383EFF30982EFF30881DFF814D013
:108270002DE9FE4F684600F0F1FFBDE8FE4F8D4648
:1082800070470000C4320220F1EE101AA0EC200A60
:1082900001607047A0EC108A704700BF81F0004178
:1082A00002E000BF83F0004330B54FEA41044FEADB
:1082B000430594EA050F08BF90EA020F1FBF54EA76
:1082C000000C55EA020C7FEA645C7FEA655C00F012
:1082D000E2804FEA5454D4EB5555B8BF6D420CDDE3
:1082E0002C4480EA020281EA030382EA000083EA66
:1082F000010180EA020281EA0303362D88BF30BD06
:1083000011F0004F4FEA01314FF4801C4CEA11315B
:1083100002D0404261EB410113F0004F4FEA0333BA
:108320004CEA133302D0524263EB430394EA050F45
:1083300000F0A780A4F10104D5F1200E0DDB02FAB4
:108340000EFC22FA05F2801841F1000103FA0EF248
:10835000801843FA05F359410EE0A5F120050EF10E
:10836000200E012A03FA0EFC28BF4CF0020C43FA3F
:1083700005F3C01851EBE37101F0004507D54FF04C
:10838000000EDCF1000C7EEB00006EEB0101B1F59C
:10839000801F1BD3B1F5001F0CD349085FEA3000E2
:1083A0004FEA3C0C04F101044FEA445212F5800FED
:1083B00080F09A80BCF1004F08BF5FEA500C50F18A
:1083C000000041EB045141EA050130BD5FEA4C0C6D
:1083D000404141EB0101013C28BFB1F5801FE9D2CA
:1083E00091F0000F04BF01460020B1FA81F308BFED
:1083F0002033A3F10B03B3F120020CDA0C3208DDB9
:1084000002F1140CC2F10C0201FA0CF021FA02F193
:108410000CE002F11402D8BFC2F1200C01FA02F103
:1084200020FA0CFCDCBF41EA0C019040E41AA2BF28
:1084300001EB0451294330BD6FEA04041F3C1CDAF0
:108440000C340EDC04F11404C4F1200220FA04F010
:1084500001FA02F340EA030021FA04F345EA0301BA
:1084600030BDC4F10C04C4F1200220FA02F001FA7C
:1084700004F340EA0300294630BD21FA04F02946FE
:1084800030BD94F0000F83F4801306BF81F4801197
:108490000134013D4EE77FEA645C18BF7FEA655C0A
:1084A00029D094EA050F08BF90EA020F05D054EADC
:1084B000000C04BF1946104630BD91EA030F1EBFE1
:1084C0000021002030BD5FEA545C05D140004941E5
:1084D00028BF41F0004130BD14F580043CBF01F5D8
:1084E000801130BD01F0004545F0FE4141F47001BE
:1084F0004FF0000030BD7FEA645C1ABF1946104699
:108500007FEA655C1CBF0B46024650EA013406BF99
:1085100052EA033591EA030F41F4002130BD00BF58
:1085200090F0000F04BF0021704730B54FF4806415
:1085300004F132044FF000054FF0000150E700BF96
:1085400090F0000F04BF0021704730B54FF48064F5
:1085500004F1320410F0004548BF40424FF00001E2
:108560003EE700BF42004FEAE2014FEA31014FEA25
:1085700002701FBF12F07F4393F07F4F81F0605174
:10858000704732F07F4208BF704793F07F4F04BFBF
:1085900041F40021704730B54FF4607401F000459C
:1085A00021F000411CE700BF50EA010208BF7047FC
:1085B00030B54FF000050AE050EA010208BF7047ED
:1085C00030B511F0004502D5404261EB41014FF456
:1085D000806404F132045FEA915C3FF4D8AE4FF05E
:1085E00003025FEADC0C18BF03325FEADC0C18BF41
:1085F000033202EBDC02C2F1200300FA03FC20FA92
:1086000002F001FA03FE40EA0E0021FA02F11444DE
:10861000BDE600BF80F0004002E000BF81F00041F5
:1086200042001FBF5FEA410392EA030F7FEA226C18
:108630007FEA236C6AD04FEA1262D2EB1363C1BFA8
:10864000D218414048404140B8BF5B42192B88BF17
:10865000704710F0004F40F4000020F07F4018BF3A
:10866000404211F0004F41F4000121F07F4118BF5A
:10867000494292EA030F3FD0A2F1010241FA03FC02
:1086800010EB0C00C3F1200301FA03F100F00043EA
:1086900002D5494260EB4000B0F5000F13D3B0F1B2
:1086A000807F06D340084FEA310102F10102FE2A21
:1086B00051D2B1F1004F40EBC25008BF20F0010091
:1086C00040EA03007047490040EB0000013A28BF30
:1086D000B0F5000FEDD2B0FA80FCACF1080CB2EBB3
:1086E0000C0200FA0CF0AABF00EBC2505242184331
:1086F000BCBFD0401843704792F0000F81F40001D6
:1087000006BF80F400000132013BB5E74FEA4103A8
:108710007FEA226C18BF7FEA236C21D092EA030F14
:1087200004D092F0000F08BF0846704790EA010F8E
:108730001CBF0020704712F07F4F04D1400028BFBB
:1087400040F00040704712F100723CBF00F500009D
:10875000704700F0004343F0FE4040F400007047D3
:108760007FEA226216BF08467FEA2363014642027F
:1087700006BF5FEA412390EA010F40F48000704792
:108780004FF0000304E000BF10F0004348BF404238
:108790005FEA000C08BF704743F0964301464FF074
:1087A00000001CE050EA010208BF70474FF00003D0
:1087B0000AE000BF50EA010208BF704711F0004311
:1087C00002D5404261EB41015FEA010C02BF8446E1
:1087D0000146002043F0B64308BFA3F18053A3F540
:1087E0000003BCFA8CF2083AA3EBC25310DB01FA87
:1087F00002FC634400FA02FCC2F12002BCF1004F0B
:1088000020FA02F243EB020008BF20F0010070479B
:1088100002F1200201FA02FCC2F1200250EA4C00EF
:1088200021FA02F243EB020008BF20EADC70704735
:108830007BB972B90029BEBF00204FF0004106E0AD
:1088400008BF00281CBF6FF000414FF0FF3000F060
:108850002BBAADF1080C6DE904CE002909DB002B21
:108860001ADB00F0B9F8DDF804E0DDE9022304B01A
:108870007047404261EB4101002B1BDB00F0ACF87C
:10888000DDF804E0DDE9022304B0404261EB410180
:10889000524263EB43037047524263EB430300F0E1
:1088A0009BF8DDF804E0DDE9022304B0404261EB0F
:1088B00041017047524263EB430300F08DF8DDF84D
:1088C00004E0DDE9022304B0524263EB4303704746
:1088D00053B94AB9002908BF00281CBF4FF0FF3127
:1088E0004FF0FF3000F0E0B9ADF1080C6DE904CEB7
:1088F00000F072F8DDF804E0DDE9022304B070470F
:10890000430803F05533C01A830803F0333300F0F3
:108910003330184400EB101000F00F3000EB002053
:1089200000EB0040000E704708B502460B4643ECD2
:10893000172BB5EEC07BF1EE10FA03D4BDE808406A
:1089400000F02AB8B1EE477B51EC170B00F024F889
:10895000404261EB410108BD9FED0B6B07EE900AB1
:108960009FED0B5BB7EEE77A27EE066BBCEEC66BAE
:10897000B8EE464BA4EE457BFCEEC77B16EE101A14
:1089800017EE900A704700BF000000000000F03DA5
:10899000000000000000F0419FED0B6B41EC170B55
:1089A0009FED0B5B27EE066BBCEEC66BB8EE464B3D
:1089B000A4EE457BFCEEC77B16EE101A17EE900A6C
:1089C000704700BFAFF30080000000000000F03DE2
:1089D000000000000000F0412DE9F047089D04462A
:1089E0008E46002B4DD18A42944669D9B2FA82F262
:1089F00052B101FA02F3C2F1200120FA01F10CFA9E
:108A000002FC41EA030E94404FEA1C48210CBEFBD5
:108A1000F8F61FFA8CF708FB16E341EA034306FB5E
:108A200007F199420AD91CEB030306F1FF3080F0ED
:108A30001F81994240F21C81023E63445B1AA4B23A
:108A4000B3FBF8F008FB103344EA034400FB07F7DC
:108A5000A7420AD91CEB040400F1FF3380F00A811D
:108A6000A74240F207816444023840EA0640E41B12
:108A700000261DB1D4400023C5E900433146BDE8BE
:108A8000F0878B4209D9002D00F0EF800026C5E960
:108A9000000130463146BDE8F087B3FA83F6002E78
:108AA0004AD18B4202D3824200F2F980841A61EBF0
:108AB000030301209E46002DE0D0C5E9004EDDE70E
:108AC00002B9FFDEB2FA82F2002A40F09280A1EBF6
:108AD0000C014FEA1C471FFA8CFE0126200CB1FB4B
:108AE000F7F307FB131140EA01410EFB03F0884244
:108AF00008D91CEB010103F1FF3802D2884200F2D1
:108B0000CB804346091AA4B2B1FBF7F007FB101162
:108B100044EA01440EFB00FEA64508D91CEB040400
:108B200000F1FF3102D2A64500F2BB800846A4EB5B
:108B30000E0440EA03409CE7C6F12007B34022FA46
:108B400007FC4CEA030C20FA07F401FA06F31C4375
:108B5000F9404FEA1C4900FA06F3B1FBF9F8200C82
:108B60001FFA8CFE09FB181140EA014108FB0EF0C8
:108B7000884202FA06F20BD91CEB010108F1FF3A18
:108B800080F08880884240F28580A8F10208614424
:108B9000091AA4B2B1FBF9F009FB101144EA014132
:108BA00000FB0EFE8E4508D91CEB010100F1FF34DD
:108BB0006CD28E456AD90238614440EA0840A0FB75
:108BC0000294A1EB0E01A142C846A64656D353D04B
:108BD0005DB1B3EB080261EB0E0101FA07F722FA6F
:108BE00006F3F1401F43C5E9007100263146BDE898
:108BF000F087C2F12003D8400CFA02FC21FA03F3FB
:108C0000914001434FEA1C471FFA8CFEB3FBF7F07B
:108C100007FB10360B0C43EA064300FB0EF69E42A0
:108C200004FA02F408D91CEB030300F1FF382FD239
:108C30009E422DD9023863449B1B89B2B3FBF7F6E1
:108C400007FB163341EA034106FB0EF38B4208D9BA
:108C50001CEB010106F1FF3816D28B4214D9023EFB
:108C60006144C91A46EA004638E72E46284605E719
:108C70000646E3E61846F8E64B45A9D2B9EB0208EA
:108C800064EB0C0E0138A3E74646EAE7204694E77A
:108C90004046D1E7D0467BE7023B614432E73046AD
:108CA00009E76444023842E7704700BF02E000F081
:108CB00000F8FEE772B6374880F30888364880F33C
:108CC000098836483649086040F20000CCF20000BE
:108CD0004EF63471CEF200010860BFF34F8FBFF340
:108CE0006F8F40F20000C0F2F0004EF68851CEF2D5
:108CF00000010860BFF34F8FBFF36F8F4FF000008C
:108D0000E1EE100A4EF63C71CEF20001086006203A
:108D100080F31488BFF36F8F1BF16AFF1AF1C4FE52
:108D20004FF055301F491B4A91423CBF41F8040B9C
:108D3000FAE71D49184A91423CBF41F8040BFAE793
:108D40001A491B4A1B4B9A423EBF51F8040B42F88A
:108D5000040BF8E700201849184A91423CBF41F83B
:108D6000040BFAE71BF182FF1AF1FEFE144C154DBD
:108D7000AC4203DA54F8041B8847F9E702F054FACE
:108D8000114C124DAC4203DA54F8041B8847F9E742
:108D90001BF16ABF000602200022022000800108A9
:108DA00008ED00E00000022000060220886317089A
:108DB00000220220CC300220D03002205CC40320EC
:108DC000008201085C8201085C8201085C82010863
:108DD0002DE9F04F2DED108AC1F80CD0D0F80CD051
:108DE000BDEC108ABDE8F08F002383F3118828467C
:108DF000A04700201AF1C8FBFEE71AF127FA00DFAE
:108E0000FEE7000070B54FF0FF0C4CF4E06C1CEA7C
:108E100011541DBF1CEA135594EA0C0F95EA0C0F70
:108E200000F0DEF82C4481EA030621EA4C5123EAE3
:108E30004C5350EA013518BF52EA033541F4801112
:108E400043F4801338D0A0FB02CE4FF00005E1FBC5
:108E500002E506F00042E0FB03E54FF00006E1FB0F
:108E600003569CF0000F18BF4EF0010EA4F1FF0452
:108E7000B6F5007F64F5407404D25FEA4E0E6D4192
:108E800046EB060642EAC62141EA55514FEAC520A3
:108E900040EA5E504FEACE2EB4F1FD0C88BFBCF51F
:108EA000E06F1ED8BEF1004F08BF5FEA500E50F1D0
:108EB000000041EB045170BD06F0004646EA010196
:108EC00040EA020081EA0301B4EB5C04C2BFD4EBC8
:108ED0000C0541EA045170BD41F480114FF0000EC1
:108EE000013C00F3AB8014F1360FDEBF002001F02F
:108EF000004170BDC4F10004203C35DA0C341BDCA9
:108F000004F11404C4F1200500FA05F320FA04F07A
:108F100001FA05F240EA020001F0004221F00041AE
:108F200010EBD37021FA04F642EB06015EEA430E21
:108F300008BF20EAD37070BDC4F10C04C4F1200551
:108F400000FA04F320FA05F001FA04F240EA020004
:108F500001F0004110EBD37041F100015EEA430ED5
:108F600008BF20EAD37070BDC4F1200500FA05F2F5
:108F70004EEA020E20FA04F301FA05F243EA020374
:108F800021FA04F001F0004121FA04F220EA020083
:108F900000EBD3705EEA430E08BF20EAD37070BDC9
:108FA00094F0000F0FD101F00046400041EB0101A9
:108FB00011F4801F08BF013CF7D041EA060195F08B
:108FC000000F18BF704703F00046520043EB030345
:108FD00013F4801F08BF013DF7D043EA0603704732
:108FE00094EA0C0F0CEA135518BF95EA0C0F0CD03D
:108FF00050EA410618BF52EA4306D1D181EA030183
:1090000001F000414FF0000070BD50EA410606BF7C
:109010001046194652EA430619D094EA0C0F02D1C1
:1090200050EA013613D195EA0C0F05D152EA033606
:109030001CBF104619460AD181EA030101F0004124
:1090400041F0FE4141F470014FF0000070BD41F06D
:10905000FE4141F4780170BD4FEA410212F5001261
:1090600015D211D56FF47873B3EB625212D94FEA6F
:10907000C12343F0004343EA505311F0004F23FA59
:1090800002F018BF404270474FF00000704750EAAE
:10909000013005D111F0004008BF6FF0004070476B
:1090A0004FF00000704700BF4FEA4102B2F1E043C9
:1090B00024BFB3F5001CDCF1FE5C0DD901F0004CBF
:1090C0004FEAC0024CEA5070B2F1004F40EB83000F
:1090D00008BF20F00100704711F0804F21D113F13B
:1090E0003872BCBF01F00040704741F480114FEA74
:1090F0005252C2F11802C2F1200C10FA0CF320FAFD
:1091000002F018BF40F001004FEAC1234FEAD32319
:1091100003FA0CFC40EA0C0023FA02F34FEA430383
:10912000CCE77FEA625307D150EA01331EBF4FF00C
:10913000FE4040F44000704701F0004040F0FE4027
:1091400040F40000704700BF01F0FF01102A2BDB44
:1091500010F0070F08D010F8013B013A8B422DD0D8
:1091600010F0070F42B3F6D1F0B441EA012141EA11
:10917000014122F007047FF000070023F0E80256C7
:10918000083C85EA010586EA010685FA47F5A3FA57
:1091900087F586FA47F6A5FA87F68EB9EED1F0BCC8
:1091A00001F0FF0102F0070232B110F8013B013A71
:1091B00083EA010313B1F8D10020704701387047EA
:1091C000002D06BF35460338073815F0010F07D1CB
:1091D000013015F4807F02BF013015F4C03F01302B
:1091E000F0BC0138704700BFEC46A0E8F05F4FF0DC
:1091F00000007047B0E8F05FE546080008BF0120B6
:10920000704700BF10F8012B11F8013B012A28BF5D
:109210009A42F7D0D01A7047034613F8012B002A60
:10922000FBD1181A0138704710B5044620461CB10E
:1092300054F80C3B013300D110BD0822012100F08D
:1092400067FB54F80C0C54F8082C14F8041C121A80
:10925000B2FBF1F200F05CFBE8E70000C26AD0E983
:10926000003112F0040F2DE9F04118BF0B46A6B0F3
:109270000021594C042601270291CDE90003D006B4
:109280004CBF03F1200203F168020392DA690399EB
:10929000D2099B6902F004021B880A4303F47F434E
:1092A00003924FF0E022A3F53E41D2F8882D02F45C
:1092B000A002B2F5A00F04BF012202924B424B4123
:1092C0000493464D03A82C6000F020FA04220121EB
:1092D000434800F01DFB0422012102A800F018FB06
:1092E00010220121019800F013FB00982022012197
:1092F0000C3000F00DFB019804220121103000F029
:1093000007FB0422012103A800F002FB01980C22B4
:109310000121143000F0FCFA0C220121009800F029
:10932000F7FA029BDA071FD5009BDB6ADB064ED4F7
:1093300015A8FEF7AFFFDDF804C00DF1140E0CF117
:1093400020030CF160081868083353F8041C7246B7
:10935000434503C29646F6D1DCF86030259384225B
:10936000012105A800F0D4FA00F0B6F8FFF75CFF81
:109370004FF0E023D3F8003D03F47023B3F5402F02
:109380000ED0184B05A88DF81C60059314338DF88A
:10939000287006934FF0FF33CDE90833FFF744FF01
:1093A0002B68A34206D0104B0422012105A8059387
:1093B00000F0AEFA00F020FA002882D0049B1BB126
:1093C000019A93690233936126B0BDE8F08105A844
:1093D000FEF75AFFC3E700BFED55CEACD0300220F8
:1093E0006CE9130828ED00E0ACCE55ED08B525205A
:1093F00018F17AF90F4B5A6A42F010025A625A6A0F
:1094000022F010025A625A6A5A6C42F010025A64F0
:109410005A6E42F010025A6675225B6E064BDA6095
:109420004FF0FF321A620D221A600122034B1A70AC
:1094300008BD00BF0038024000100140FC3202208D
:1094400037B50E4D2A78202A15D10D4C0D482368CA
:109450000D49184401921AF1A9FD23680021019ACF
:10946000203309482970236020F134FE03B0BDE8A1
:1094700030401BF125BB03B030BD00BFC432022019
:10948000EC32022060721708C6320220014B1868C5
:10949000704700BFFCFF1F08014B0248C01A70470D
:1094A00060721708000020080048704760721708B3
:1094B00007490022074B5B1A9A4201D301207047EB
:1094C00051F8040B013001D10432F5E70020704758
:1094D00060721708000020085E4B2DE9F74F1A68EC
:1094E00002255D4B02F56A58DFF894911A7808F16D
:1094F00018085A4F5A4C9044DFF888A119F1C8FD5A
:10950000A9EB070B06460EB14E2D49D9A9EB070270
:10951000B2EB080700F192804E2D00F28F80DFF849
:1095200068C16B1C4F4E0C21DBB2ACEB06006943EB
:10953000B84273DD60184FF0010C665090463E440F
:1095400080F808C04660B2EB080213D44F2B11D04C
:10955000454E19464548AB1C351ADBB295424FF0D3
:109560000C0505FB01F163DD65180126024460501E
:109570002E726A600C2201215343E21811724FF0DF
:10958000FF31E15051603A4B1B782BB1394B1B68CE
:109590002360394B1B686360314803B0BDE8F08F2E
:1095A000336AF06953450ABF344BF31AA3EB0A033D
:1095B00080B101931AF1CAFE019B58B12A460C21D1
:1095C00001354A430121EDB2A0180172F169A150A1
:1095D0000D3141600C200121984400FB05FCD84569
:1095E00004EB0C0244F80C6006F13C0C1172C2F85A
:1095F00004C005EB010205F10205D2B2EDB200FB99
:1096000002F204EB02000172316AA1501944416078
:1096100014D2304619F14CFD064674E767184FF036
:10962000010E8044665087F808E0C7F804C08AE756
:10963000621801256050157256609BE74F2D01D8C6
:109640002B4697E7012384F8BC334FF0FF33C4E97E
:10965000ED3398E7EC320220C43202206072170822
:1096600004220220D03002200000082060C4032021
:1096700000220220F0320220E832022000220220E2
:1096800000002008000602205CC403200C4B1B785D
:1096900010B50BB9FFF7AAFE00230A490A48CA69A8
:1096A0009206FCD54A6A1C5CD2B2944205D10133C1
:1096B000DBB20E2BF3D1002010BD0023EFE700BF7B
:1096C000FC3202200010014070E9130838B5084B45
:1096D00004461B780BB9FFF789FEE4B2054DAC6276
:1096E000EB695B0600D538BD1BF1EAF9F8E700BF6E
:1096F000FC3202200010014010B5441E14F8010F86
:1097000000B910BDFFF7E2FFF8E7000070B502688E
:109710000446EFF30581D9205369C9B2CBF07EFD31
:10972000294B1B78A3B1294B94E8030083E803007D
:109730002748FFF7E1FF6368B3B12648FFF7DCFF76
:109740002548FFF7D9FFFFF7A1FF2448FFF7D4FF13
:10975000234D2B783BB124681CB120461AF1F6FD4D
:1097600020B900232B7070BD1E48E7E720461E4E2F
:109770001AF10AFE00F2145084421FD220461AF158
:1097800003FE30602046194E1AF124FE04F5E05322
:10979000834217D920461AF11DFE30600023144A77
:1097A0001360144A1370FFF783FE0028D9D01BF111
:1097B00087F90120BDE870401AF16CBCA4F2145383
:1097C0003360DFE73360E9E7C5320220F43202207C
:1097D00080E9130885E9130896E913083C24150865
:1097E0000022022090E91308F0320220E832022021
:1097F000EC320220C4320220284B1A7870B542B1F4
:109800002748FFF779FF274B5868003818BF012019
:1098100070BD254A107800283CD0244E244C336873
:109820002448254D1A1D21782D1A0A44AA4205D331
:10983000224A4FF0FF31D161202222702278D2B12A
:1098400003F120018D4205D81F2A9FBF1B4AD36117
:10985000202222702022194918441AF1A7FB3268ED
:10986000237800211548134420222170336020F111
:1098700031FC1BF125F933689D4207D90F4920229D
:109880000F48CB611AF192FB1BF11AF900201AF173
:1098900001FCB8E701221A70BAE700BFC532022006
:1098A000DCE91308F432022000220220EC3202200C
:1098B000C43202206072170800002008C63202205D
:1098C000E0FF1F082DE9F84307460E460024DFF8A5
:1098D0003890DFF83880B44201D1BDE8F88324B174
:1098E000230702D14846FFF707FF3D5D01342B09EE
:1098F00005F00F0518F80300FFF7E8FE18F805005B
:10990000FFF7E4FEE7E700BF3C241508ECE9130885
:10991000474B1B782DE9F74F07460E4690465BB143
:10992000022925D0042938D0012902D11146FFF798
:10993000C9FF4048FFF7E0FE3F4B1B78002B4ED09D
:109940003E4A00253E4BA2EB030938E037F81430BD
:10995000ADF8043024B1620702D12846FFF7CCFEEF
:109960000134022101A8FFF7ADFFA045EED1E0E7E9
:109970000024304DF9E757F82430019324B1A307B0
:1099800002D12846FFF7B8FE042101340DEB010097
:10999000FFF798FFA045EED1CBE70024254DF9E76E
:1099A000FFF74EFD022E1DD0042E2CD0012E06D125
:1099B0002378795D5A1C2270224AD1540135A8457A
:1099C0000DD0214B214C1B682278043313444B45A6
:1099D000E6D31C4B4FF0FF32DA612023237003B033
:1099E000BDE8F08F2378DFF85CA05A1C22703A782B
:1099F0000AF80320FFF724FD23785A1C2270002266
:109A00000AF80320DAE74FF0000ADFF838B02278CE
:109A10003B78511C23FA0AF30AF1080A21700BF86B
:109A20000230FFF70DFDBAF1200FF0D1C6E700BFFD
:109A3000C53202203C241508002202200000200824
:109A400060721708C6320220EC320220C4320220B3
:109A5000036800221B68184710B5036804465B685A
:109A6000984708B194F84D0010BD0000684B2DE9EF
:109A7000F04103F5004490B006460F4694F9A42B3C
:109A8000002A00F0C28094F8EC5B35B9614AB5F069
:109A900069FD284610B0BDE8F081B3F9A4201AB9D9
:109AA000B3F8A220A3F8A420B3F8A430632B05D800
:109AB0000025594A39463046B5F054FD00212E2282
:109AC00004A8039120F106FBD4F8040B03AA322169
:109AD00003681B689847804630B9454603AB4F4A38
:109AE00039463046B5F03EFDB4F8E03A41F658321A
:109AF000A3F57A739BB2934206D90025484B3A46A8
:109B000020213046B5F024FB94F9243D002B6BDD79
:109B100094F9DC3C002B5BDD0025424B3A462021CA
:109B20003046B5F015FB322303AA3F49D4F8100B99
:109B3000C2F02CF9804640B903AB45463A46202195
:109B400000933046394BB5F003FB322303AA384962
:109B5000D4F80C0BBFF020F8804640B903AB454663
:109B60003A46202100933046304BB5F0F1FA2021DF
:109B70003046B5F0E5FAC8B104F536639FED2D7AAD
:109B8000D3ED007AF0EEE77AF4EEC77AF1EE10FA50
:109B90000CD594F9243D002B02DD94F8883D2BB9B7
:109BA0000025254A39463046B5F0DCFC94F9243DC1
:109BB000002B7FF76EAF94F9D13B002B3FF469AFD8
:109BC0001E4B3A46202130460025B5F0C1FA60E729
:109BD00094F8888DB8F1000F06D14546184B3A46E7
:109BE00020213046B5F0B4FA94F9DC3C002B9ADD24
:109BF00094F80D8DB8F1000F95D1124B3A46202103
:109C000030464546B5F0A4FA8DE7012541E700BF8F
:109C10001033022000EA130822EA130849EA130865
:109C200054EA130866EA1308D7EA1308DBEA1308B4
:109C3000EDEA130800000034F1EA13080BEB1308F7
:109C40008CEA1308B2EA130838B50446B5F05CFA9A
:109C5000114B93F8C01C114B002908BF01461D6829
:109C6000EB6A1A6818461268904777F0DDF8EB6ADD
:109C700093F89C1076F0ACF894F860305BB1CBF0C0
:109C800039FBEB6AD3F8A030C01AB0F5FA6F24BFE5
:109C9000002384F8603038BD10B302200C3302205A
:109CA00008B5FFF7D1FF054B05481B68DB6A93F841
:109CB0009C10BDE8084013F08DBA00BF0C330220A1
:109CC000E8BD022070B50E46054684F06BFB84F0BB
:109CD0002DFB10B90124204670BD0A4B93F90E3BB1
:109CE000012BF7D184F05EFB437A002BF2D184F094
:109CF00059FB847A002CEDD1034A31462846B5F051
:109D000031FCE8E71063022024EB1308034BD3F87F
:109D1000783B0BB9B5F08CB9012070471063022075
:109D20002DE9F0472DED028BC47F90B007468846A1
:109D30008CB990F90430002B00F00481824B1D682F
:109D4000A86A03685B6B9847044650B97F4A41464E
:109D50003846B5F007FC204610B0BDEC028BBDE8DC
:109D6000F087BB684BB93B68414638469B6B10B0E7
:109D7000BDEC028BBDE8F0471847E86AFFF76CFEC0
:109D800004460028E7D14146714E3846B6F092FCB1
:109D9000414605463846B5F02BFD06F5326206F61B
:109DA0001C33284092ED007AD3ED007AC5B2B4EEB0
:109DB000E77AF1EE10FA09D596F9183B032B05D096
:109DC0002546644A41463846B5F0CCFB624BB0EEBE
:109DD000088A93ED007AB4EEC87AF1EE10FA09D54C
:109DE000B7EEC77A00255D4A414638468DED007BC7
:109DF000B5F0B8FB06F6C42393ED007AB4EEC87A4A
:109E0000F1EE10FA09D5B7EEC77A0025544A41465B
:109E100038468DED007BB5F0A5FB06F6C823F8EEBD
:109E2000087A93ED007AB4EEE77AF1EE10FA09DDE4
:109E3000B7EEC77A00254B4A414638468DED007B88
:109E4000B5F090FBB6F9AC3A042B07DC05220025EF
:109E5000414638460092444AB5F084FBDFF8289129
:109E6000D9F8280F84F092FB80B196F90E3B6BB1C4
:109E7000D9F8283FB6F9102BB3F90E309A4205DA1B
:109E800000253A4A41463846B5F06CFB4146384613
:109E9000DFF8F8A0FFF716FF414606463846FFF701
:109EA000E5FD9AF84933002B45D1354000EA050419
:109EB0004FF480612E4801F081F978B1D9F8283F3C
:109EC000B3F90C30A3F2E24292B2B2F5FA7F05D9AF
:109ED0000024284A41463846B5F044FB9AF86C3ACB
:109EE00053B1254844F01EFF054628B92C46234AA5
:109EF00041463846B5F036FB002103AE2E2204A8B9
:109F0000039120F1E7F832463221DAF834030BF0FE
:109F1000F9FA054600287FF41EAFDAF834032C4620
:109F200003689B689847164A0346414638460096A0
:109F3000B5F018FB0FE7134A414638460024B5F048
:109F400011FBB5E7012406E70C33022034EB1308BC
:109F5000106302204BEB1308D06D02206EEB130848
:109F60008EEB1308B0EB1308D2EB1308F1EB1308D8
:109F7000103302202CEC130874AD022054EC1308AB
:109F8000F66A150817EC13081073022010A30220BC
:109F900070B505460E46FFF795FE04463146284645
:109FA000B6F0E2FA2040C0B270BD0000F0B591B04A
:109FB00005460E46B5F0D2FC0446D8B1102128461D
:109FC000B5F0BEF8B0B1002103AF2E2204A8039172
:109FD00020F180F81EF02EFC32233A4601211DF0BC
:109FE00081FE044630B9054B3246102128460097C1
:109FF000B5F0AEF8204611B0F0BD00BFF34F160823
:10A0000070B505460E46B1B990F910408CB11648AE
:10A0100016F058F8B0EEC00ADFED147AB4EEE70A95
:10A02000F1EE10FA07D43446114A01212846B5F062
:10A0300099FA204670BDAB689BB10E4B1B68D86A7D
:10A04000FFF70AFD044630B181F05EFE0A4A0421A2
:10A050007AF0FAFAEDE731462846BDE87040B5F0EF
:10A060006FBF0124E5E700BF103302200000003479
:10A0700068EC13080C3302207AEC130838B5044658
:10A08000B6F0FAFB0546A8B10B4807F091FE38B1CF
:10A090000A490B481DF0AEFF10B1074801F060F807
:10A0A0002046FFF7FDFD01230649204684F8603075
:10A0B000B6F0ACFA284638BD1033022064BC02204A
:10A0C000085202209CEC1308F8B505460E461746C8
:10A0D000C2B1232901D0012914D824480AF0A8FCD0
:10A0E000044668B100242046F8BD95F91030022BD3
:10A0F00008D081F009FE1E4A06217AF0A5FAF2E79F
:10A10000002EF2D03A4631462846B6F06DFC0446A1
:10A110000028E7D0174E06F17803D6F834239A4288
:10A1200003D006F6642044F09BFAD6F83403124FAD
:10A1300003689B6B9847D7F8283B86F8380A012BB1
:10A1400007D184F02FF9542185F0BEFB08B9C7F878
:10A15000280B2846FFF7A4FD4FF0FF330749284698
:10A16000C6F86C33B6F052FABDE700BF10330220D8
:10A17000ACEC130810A3022010B30220C4EC1308A7
:10A180002DE9F04FDFF85091074688462DED028B00
:10A1900093B0B5F081F899F9E34A0546CCB9BD21F1
:10A1A000464844F0E7FB38B12546454B42464FF45C
:10A1B00080413846B4F0CCFFBC21404844F0DAFB83
:10A1C00038B100253F4B42464FF480413846B4F049
:10A1D000BFFF3D4C94F8EC3B002B68D0A4F58053B6
:10A1E0001C22002104A8B3F8983AA4F29C5AA4F5C2
:10A1F000004B0126A4F5405403931FF16BFF06A802
:10A2000025F0DEFB039B9E4251D20DA825F0D8FB22
:10A210000BAA3146504644F073FA002847D0BDF8E7
:10A220002E10584609F0F6FC80B3BDF81230102B02
:10A230002CD106A90DA825F06BFFDFED247AB7EE2F
:10A24000C08B94ED140A2248B4EEE70AF1EE10FA3E
:10A25000BCBF09F52B6393ED000A20EE000A11F054
:10A26000E3F8F6EE087A20EE270AB4EEC08AF1EEA3
:10A2700010FA0BD5B7EEC00A0025164B42464FF434
:10A28000804138468DED000BB4F062FF0DF12C0CCF
:10A290000DF1100E0136BCE80F00AEE80F009CE88F
:10A2A0000700B6B2AEE803008EF80020AAE7284601
:10A2B00013B0BDEC028BBDE8F08F00BF74AD02207F
:10A2C000D8EC130804ED130810B30220000000348A
:10A2D000E8BD022037ED130810630220002070470C
:10A2E000014800F00DBE00BF1033022003685B6818
:10A2F0001847000019F0A2BC8EF0E2BE83F090BFB8
:10A3000007F05ABB39F048BC75F0E4BE0AF0D6BC81
:10A3100073F0E0BC0FF05ABC17F03CBA04F07CB804
:10A3200072F06AB822F000BF87F0D8BE87F0E6BAB4
:10A3300017F094BA67F058B88FF01ABA15F042BF08
:10A3400022F09CB991F032BA83F06CBC81F096B9DE
:10A3500009F03EBE06F084BA0EF076BE0FF092BB56
:10A3600017F010B817F034BB15F05ABD17F04AB902
:10A3700001F0ECBC00F2EC6026F014BD0AF0E2B98A
:10A38000B02290F8F43202FB030390F8892393F88B
:10A39000D13012B1012B28BF0123184670470000AD
:10A3A00090F814310BB190F8413118467047000015
:10A3B000034808603121117008221A60704700BFFD
:10A3C00094F21308F8B5044600F50A4004F5F75571
:10A3D0006430FFF739FC0021183528461EF09EF93D
:10A3E0008021204617F08CFD18B13BF097FB38F028
:10A3F0000FFF04F56B539FED337A04F5804604F5A7
:10A400000D40D3ED007A06F63C77203067EE877A70
:10A41000FDEEE77A17EE903AC6F8383F04F56B5335
:10A4200008331B683B6017F06FFFD8B9D6F8383F88
:10A4300007EE903A04F5F753F8EEE77A93ED997A40
:10A4400067EE877AFDEEE77A17EE902AC6F8382F86
:10A45000D3ED987A97ED007AF0EEE77A67EE877A97
:10A46000C7ED007A04F5085104F5F24605F545708C
:10A47000303141F0ABFB94ED467AD6ED167AE7EE3B
:10A48000007AB7EEE70AC6ED167A3CF065F9B7EE4A
:10A49000C00B04F50A4086ED160AD83010F0C4F857
:10A4A00004F50A400021E430BBF018FA4FF4001123
:10A4B000204617F025FD20B12846BDE8F8401CF0E5
:10A4C000F1B8F8BD0000C842FFF77CBFF8B500F551
:10A4D000E0470546D7F8340305F50A440368D83445
:10A4E0009B6B98470646204612F038FE97F897393E
:10A4F000002818BF00262BB926B105F59F40603013
:10A50000BBF050F9204612F0C9FA18B92046FFF7FF
:10A5100047FF20B12046BDE8F84013F07FB8F8BDF2
:10A52000FFF7D4BF38B54FF48011044617F0E8FCAC
:10A53000054620B90121204617F0E2FC054602211C
:10A54000204617F0DDFC48B115B9204603F086FE21
:10A5500004F5F75018301BF0A3FF01E0002DF7D1F0
:10A560004FF48051204617F0CBFC30B104F5094080
:10A57000BDE83840E03087F027BF38BDFFF7D2BFD5
:10A5800038B504464FF4801117F0BAFC0121054696
:10A59000204617F0B5FC18B115B9204603F05EFE51
:10A5A0001021204617F0ACFC88B1204603F04CFF88
:10A5B0004FF48001204617F0A3FC18B93BF0AEFA27
:10A5C00038F022FF04F5BB501030A6F04DFB2021DF
:10A5D000204617F095FC28B1204604F005F82046E7
:10A5E00004F022F94FF40051204617F089FC10B115
:10A5F000204604F0FFF88021204617F081FC28B1A6
:10A600003BF08CFABDE8384038F026BE38BD00007B
:10A61000FFF7B6BF00F5E04300F50840D3F8581344
:10A62000B830B7F013BE0000FFF7F4BF10B5044612
:10A6300026F0C0FC90F925308BB190F8443373B10B
:10A6400094F914375BB1064B1B68DB6A93F89C30B6
:10A650002BB904F2EC60BDE8104026F0AFB910BD94
:10A660000C330220FFF7E2BF464B1B682DE9F04197
:10A67000DB6A044693F89C30002B00F0818000F5E3
:10A68000005393F80132002B7AD00AF0D1F9002858
:10A6900076D004F5475504F54056043596F81A135C
:10A6A00028461BF03BFA00286AD004F5907738461C
:10A6B000FFF766FE022863D994F814244FF0B0081F
:10A6C000F1EE007A08FB024292ED837AB4EEE77A6B
:10A6D000F1EE10FA54D496F81A1328461BF0D8FC61
:10A6E000B6F9AC3A07EE903AB8EEE77AB4EEC07A33
:10A6F000F1EE10FA0CDD94F81434F8EE677A08FBEA
:10A70000034393ED837AF4EEC77AF1EE10FA37DC67
:10A7100004F50051D1F8F03083EAE372A2EBE37262
:10A7200004F58043D3F8380F824229DC06F6C422B0
:10A73000D1ED3D7A9FED146AD2ED006AF8EEE77A2A
:10A7400066EE866AF4EEE67AF1EE10FA18DC03F6AD
:10A750003C7393ED007A27EE067AF4EEC77AF1EEB9
:10A7600010FA0DD494F81414B023B6F9AE2A284682
:10A7700003FB0171BDE8F04101F582711AF0B2BF2F
:10A78000BDE8F0810C3302200000C842FFF76CBF27
:10A790002DE9F04190F8143400F590762C4D0446E4
:10A7A00000EB031330462F68D3F8C481FFF7E8FDB0
:10A7B000474514D0022814D904F5E047C5F80080B5
:10A7C00097F86433012B15D817D104F50045D5F857
:10A7D0005C39E3B9D5F86039CBB905230BE0022821
:10A7E00010D804F5E04393F864235AB1052283F8A6
:10A7F000642307E0013B87F8643304F50C503430E0
:10A800001FF0E4F92046BDE8F0410EF07FBE114B89
:10A810001B68D86A03685B68984780460028ECD1BB
:10A82000B02394F81414204603FB016105F6441686
:10A8300005F66415DC3107F02BFB55F8243C0FCBF3
:10A8400086E80F0085E80F0087F86483D5E700BF2E
:10A85000003302200C330220FFF79ABF00F50043BB
:10A8600070B593F8EC3B054600F58054DBB100F57C
:10A870000D40203018F04CF828B104F58054012325
:10A8800084F8013270BD05F50A46D836304612F01C
:10A8900005F918B104F580540023F1E73046FFF7BD
:10A8A0007FFD0028F6D105F5E04393F89729002AAB
:10A8B000F0D1D3F8403A042BDFD105F5054004F57B
:10A8C00080547830C4F010FE84F80102DAE700000A
:10A8D00010B500F5E0442346D4F8342378339A4287
:10A8E00008D000F5E4431C339A421CBF4FF0FF33FD
:10A8F000C4F8503904F51463074A1A6004F6441387
:10A90000064A1A60FFF7AAFFD4F834030368BDE8CB
:10A9100010401B69184700BF0000C8420000C8C2B1
:10A92000FFF7D6BFF7B500F5E04604460D46D6F86A
:10A93000403A8B423FD00B1F00F50547594207F1C3
:10A940007807594138460191C4F094FC0199384682
:10A95000C4F090FC042D02D1184899F0B9FFD6F844
:10A96000403A012B18D1032D16D104F50A4064306A
:10A97000B4F0D4FB40B120460AF05AF820B104F5F7
:10A980009840543099F09EFF2046C6F8405A03B0D4
:10A99000BDE8F04003F092BE072DF5D1D6F860294E
:10A9A00004F5AE4064230521143092FBF3F3044A0E
:10A9B00079F04AFEE8E703B0F0BD00BF647F0220F3
:10A9C000CCED130870B500F5E0450446D5F8340326
:10A9D00003689B6B9847A0B195F8383A8BB92B4622
:10A9E000D5F8342378339A424ED104F50A46D83646
:10A9F000304611F07BFA60B995F890397BB90121A6
:10AA000008E004F50A45D835284612F047F8002832
:10AA100040D002212046BDE87040FFF783BFB5F863
:10AA2000A23A152B29D104F5004393F87C1511F0B7
:10AA3000010120D1D5F8402A072A1CD093F91E37EE
:10AA40000BB90421E6E7204615F03CFBDFED127A56
:10AA5000B4EEE70AF1EE10FAF3DB04F505407830C6
:10AA6000C4F06EFC0028ECD004F5AE400B4A062181
:10AA7000143079F0E9FD0721CCE73046FFF790FC70
:10AA80000028C6D10321C5E704F5E4431C339A42EC
:10AA9000F8D170BD2846F1E70000B442F0ED13088C
:10AAA00038B5304C054604F17803D4F834239A4283
:10AAB0002DED028BB0EE408A03D00020BDEC028B5E
:10AAC00038BD294811F012FA40B105F50A40BDEC35
:10AAD000028BD830BDE8384012F00EBBD4F8403AB3
:10AAE000042B35D194F8653333B12049A1F56F605B
:10AAF00044F0D8FE0028E1D11D4D95F8EC3B5BB148
:10AB000005F6D82011F0F2F90028D6D105F6D820A4
:10AB100011F0ACF90028D0D1F0EEC87A9FED157A8B
:10AB2000F4EEC77AF1EE10FA09D49FED130A28EE7D
:10AB3000008ABDEEC88A18EE103AC4F860390F4892
:10AB4000C4F0FEFB0028B8D0002384F89339B5E7A1
:10AB5000B4F8A21AA4F5E04009F05CF80028C1D1CD
:10AB6000ABE700BF10A30220E8BD022064BC0220B6
:10AB700010B30220000000340000C84288B8022050
:10AB800000F5E04313B5D3F8403A0446042B16D140
:10AB900001A906F0D5FD18B19DED010A02B010BD66
:10ABA000204606F0FDF820468DED010A06F0C4F9B6
:10ABB000DDED017A37EEC00A8DED010AECE700F514
:10ABC0000944D4F890300193E6E700002DE9F04104
:10ABD00000F5AA6504462DED028B28468AB020F0C8
:10ABE000F3FA04F5F750002307A9183007930893E8
:10ABF00009931DF021FC002800F095809DED090AC5
:10AC000004F5E045DFED5F7A04F5F94005F51763DB
:10AC100020EE270ADFED5C7A303093ED007AA7EE64
:10AC2000270A83ED000A91F0D1FA2046FFF7CAFE09
:10AC3000204608F0E9FE002870D1D5F834030368F7
:10AC40009B6B9847064604F50A40D83012F086FA06
:10AC500095F89739002818BF0026002B5ED1002EEA
:10AC60005CD095F8383A002B58D1D5F8403A042BEF
:10AC700070D09FED468A204606F080F904F5004228
:10AC800004F5E143C2F84C0E2433D5F8341399424D
:10AC90001CD192F8D839CBB904F58043B3F9043FFD
:10ACA000002B04DC3A49D1F84C1CC9060ED5D2F869
:10ACB00040690A33D2F848197668891B64267343C1
:10ACC0008142ACBF5B181B18C2F84C3ED5F8403A25
:10ACD0002046D2F84C1E04F56D56D5F86823059130
:10ACE0000492039318F01CFE07462046B5F97683BC
:10ACF000FFF746FF05F65C2504F59F40F0EE400A9D
:10AD00000599B0EE480A6030CDE90078DDE90332FC
:10AD1000D6ED021A95ED001ABAF0F2F90AB0BDECC0
:10AD2000028BBDE8F08104F59070FFF729FB022843
:10AD30000AD9B02294F8143402FB034393F840225A
:10AD400012B193ED8B0A5BE7284620F0D9F8B1EEFB
:10AD5000400A55E704F5094604F5094704F5094199
:10AD60005436643744313A46304625F00DF9002810
:10AD70003FF47FAF3946304625F0CAF9B7EEC08BB5
:10AD800079E700BFCDCC4C3ECDCC4C3F000000005D
:10AD900010730220FFF71ABF2DE9F04100F5E243DE
:10ADA00000F5E04704460E463433D7F834239A4280
:10ADB00025D000F50A4808F1D808404611F06EFE8B
:10ADC0000546B0B1404610F0F7FA78B104F50044FA
:10ADD000D4F8140B03689B689847DFED0A7A20EEDD
:10ADE000270A86ED000A2846BDE8F0819FED060A95
:10ADF000F7E707F6781701253B683360F3E700258E
:10AE0000F1E700BF0AD7233C00000000F8B500F5C9
:10AE1000E04200F5E24304460E463433D2F83423D0
:10AE20009A4230D000F50A47D837384611F036FE3E
:10AE30000546A8B1384610F0BFFA70B104F50044D9
:10AE4000D4F8140B0368DB68984707EE900AF8EE15
:10AE5000E77AC6ED007A2846F8BDDFED0C7AF8E710
:10AE600004F5A0440125D4F87C0903681B699847C0
:10AE700007EE900A9FED067AF8EEE77A67EE877A9A
:10AE8000C6ED007AE7E70025E5E700BF0000000017
:10AE90000AD7233CF8B500F5E04200F5E24304464A
:10AEA0000E463433D2F834239A4224D000F50A47B0
:10AEB000D837384611F0F2FD054688B1384610F013
:10AEC0007BFA50B104F50044D4F8143B1869BFF084
:10AED00045FE86ED000A2846F8BD9FED080AF8E712
:10AEE00004F5A0440125D4F87C0903685B69984700
:10AEF00086ED000AEFE70025EDE700BF0000000047
:10AF000030B585B005466C460FC984E80F0040F2A5
:10AF100079322146284606F0BBFC0C4B03F1F802BF
:10AF2000D3F8343393420ED19DF8001011F0040190
:10AF300002D1204624F00EFE0548214606F0F4FE1C
:10AF4000012005B030BD0020FBE700BF10A30220A8
:10AF50001033022038B500F5E04304460D46D3F81F
:10AF6000340303685B6898470F2803D8092805D87D
:10AF700000200AE01338C0B20228F9D804F50940CD
:10AF800064300FC885E80F00012038BD2DE9F0417D
:10AF900000F509480E460446154608F16408304697
:10AFA000414624F03FFE18B900273846BDE8F0813D
:10AFB0004146304624F042FE07460028F4D0304691
:10AFC00024F02EFD0646284624F02AFD8642EBD1C9
:10AFD00004F5094695E80F00643604F5E04586E877
:10AFE0000F0040F2B1324146204606F051FC04F514
:10AFF000E343D5F8342328339A4204D004F5E344DC
:10B000000834A242D1D1CAF075F9C5F8A401CCE741
:10B0100070B500F50A4504460E46D835284611F0AD
:10B020003DFD68B104F5004496E8030004F549636A
:10B0300083E80300CAF05EF9C4F8980C012070BDE3
:10B04000284611F011FD0028F9D0EBE710B50446B1
:10B0500000F50A402DED028BD830B0EE408A11F099
:10B0600053FB40B904F5E04204F5E343D2F834233E
:10B0700028339A420AD104F5004404F6AC4383ED28
:10B08000008ACAF037F9C4F8B00C0120BDEC028B7D
:10B0900010BD000030B500F509450446443504F5FF
:10B0A000E0440FC985E80F00012084F8940930BD01
:10B0B00010B50446064811F027FB40B904F5E044FA
:10B0C000D4F834030368BDE810409B6C184710BDEA
:10B0D000E8BD022010B50446064810F06FFF40B9E5
:10B0E00004F5E044D4F834030368BDE81040DB6C99
:10B0F000184710BDE8BD022070B5044600F50A40AF
:10B100000E461546D83010F0A7FA50B104F50044A9
:10B11000D4F89C3D9B682B60D4F89C3D5B68336001
:10B1200070BD04F5F753D3F8202218332A60D3F802
:10B130000432336004F58043D3F84C3C9B05EFD4D4
:10B1400004F56D54D5ED007A9FED047AD4ED026AD2
:10B15000E6EEC77AC5ED007AE2E700BF35FA8E3C2D
:10B1600038B50D4D04460D4829461DF07BF804F511
:10B17000E04305F13C0183F8650304F5F75018300E
:10B180001CF0E2FE04F50940D0ED247AF1EE677A76
:10B19000C0ED247A38BD00BF64BC022008520220F2
:10B1A00010B5044600F590702EF03AFF2046BDE839
:10B1B0001040FFF7D5BF0000FFF7F2BF00F5804059
:10B1C000D0F84C3C194214BF012000207047000009
:10B1D00000F58043DFED087A00F5984093F8481FAA
:10B1E00003F66473743093ED000A01F0010120EE60
:10B1F000270AC8F091B900BF0000C842FFF7E8BFB6
:10B2000000F5E04310B50446D3F8340303689B6DA2
:10B210009847014604F5E440BDE810407430C8F09A
:10B220006DBD0000FFF7ECBF38B5054B0A4601467F
:10B230001C68236820461D68024BA847002038BDC3
:10B240000C33022010330220F8B504462DED028B9A
:10B25000036804F5004504F54056D3F8BC30984720
:10B2600095F81908B6F9AC3A30B903EB830202EB52
:10B2700082029200A5F80A28B6F9AE1A58B907EE6C
:10B28000901A9FED717A05F5E662F8EEE77A67EEBF
:10B29000877AC2ED397A04F58042D2F84C2C120636
:10B2A00014D5CA1A0B4404F5F75002EBD27203EB23
:10B2B000D373183052105B1000EE902A00EE103A53
:10B2C000F8EEE00AB8EEC00A1CF080FBB6F8DE2A01
:10B2D00004F50A465D4B64365D4F1A7085F088FDB3
:10B2E00085F0BEF800213046FEF71AFD0123B87143
:10B2F0003046FB71B3F008FF28B93046B5F09AF933
:10B30000B0FA80F0400938710421204616F0F8FDAB
:10B3100020B104F5F940503072F08EFD3046B3F0A4
:10B32000F3FED8B994F8143441F2883204EB0313D5
:10B33000D3F8C461D5F8DC39F31A93420ED904F579
:10B340009070FFF71DF8022808D92046C5F8DC697F
:10B3500006F02EFD05F5AF6300221A60B4F9A430A3
:10B360001BB9B4F8A230A4F8A430B4F8A430B7EEF6
:10B37000008ADFED388A07EE903AF8EEE77A88EE39
:10B38000270AD4ED2B7AF0EEE77AF4EEE87AF1EEC4
:10B3900010FA09D5B4F9A23007EE903AF8EEE77A40
:10B3A00088EE277A84ED2B7AD4ED2B0A3BF086F8D1
:10B3B00070BB73F08DFE40F27D124FF4801173F07C
:10B3C0003FFE71F0CFF870F037FD95F8EC3BB0EE32
:10B3D000408A23B1D5F80C0B03681B6F984704F51E
:10B3E000A540B0EE480A1C30A2F00EF904F5A840C2
:10B3F000B0EE480A0430A2F007F904F5AA40B0EE16
:10B40000480A4430BDEC028BBDE8F840A2F0FCB81D
:10B41000D4ED2B7A94ED460AF0EEE77AF4EEE87A72
:10B42000F1EE10FA09D5B4F9A23007EE903AF8EE31
:10B43000E77A88EE277A84ED2B7AD4ED2B0A3BF05D
:10B440003DF80028B5D0BCE7E5CFF83F9C270220A7
:10B450000DC2022000000034FFF7F6BE70B500F503
:10B460000046044696F91C37002B2ADD09F0E0FA65
:10B4700038BB04F50A4564352846B5F0DBF800B35F
:10B480002846B3F041FEE0B1C9F034FF04F5E043D3
:10B490004FF47A72D3F88039C01A96F91C375343A7
:10B4A00098420ED301221C212846FEF70DFE40B122
:10B4B00004F5AE40034A06211430BDE8704079F02F
:10B4C000C3B870BD10EE130800B52DED028B9FEDD3
:10B4D0000B8A83B0D0ED517A383067EE887AC0EDB0
:10B4E000437A0190A2F04EF920EE080A019803B0C9
:10B4F000BDEC028B5DF804EBA2F0BABA52B87E3F05
:10B5000000B52DED028B9FED0B8A83B0D0ED527A02
:10B510003C3067EE887AC0ED437A0190A2F032F9B0
:10B5200020EE080A019803B0BDEC028B5DF804EB35
:10B53000A2F09EBA52B87E3F30B5044600F5F750EF
:10B540002DED048B83B0183001A91CF03BFF0028BF
:10B5500000F0B98004F5F245DDED017A95ED1A7A37
:10B560006835B4EEE77AF1EE10FA07D504F50A4033
:10B570006430B3F0D3FD08B1019B2B6004F5405259
:10B5800004F56C55B6EE009ADFED606AB2F9AC3A9C
:10B59000182095ED007A052BB8BF052307EE903AE9
:10B5A000B2F9AE3AF8EEE78A07EE903AF8EEE77AAB
:10B5B00077EEA77AC7EE270ADFED557A68EEA77A0D
:10B5C00087EE271AF0EE007AF4EE490AF1EE10FA4F
:10B5D00079FE200AB4EE671AF1EE10FA48BFB0EE19
:10B5E000671ADDED017AF4EEE67AF1EE10FACCBFDF
:10B5F00087EE270AB0EE410A3BF0C6F804F50A4090
:10B60000B0EE408AD83011F049FA38B904F5004359
:10B6100093F8EC2BD2B393F8193CBBB304F50A4072
:10B620006430B3F07BFD88B328EE892A9DED011AC2
:10B63000B4EEC21AF1EE10FA28D5D5ED000ADFED0E
:10B64000351AC0EE820A9FED340A3AF0B3FF04F5D2
:10B65000A4406430B4EE408AF0EE408AF1EE10FA75
:10B6600048BFF0EE488AFFF72FFF04F5A74004F526
:10B67000AA444830B0EE688AFFF742FFD4ED647AFE
:10B680009FED267A67EE877AC4ED647A24481BF032
:10B690000FFD90B940212348FFF790FD68B1224B80
:10B6A000D3F8403A012B08D1F7EE007AB4EEE78ADE
:10B6B000F1EE10FA58BFB0EE678AB0EE480A03B058
:10B6C000BDEC048B30BD04F50A40B7EE008A64304F
:10B6D000B3F024FD0028D9D0462084F077FCB4EEE6
:10B6E000C80ADFED127AF1EE10FA30FE080A87EE92
:10B6F000800A1BF173FE2F209FED0D1ADFED0D0A5E
:10B700003BF042F8B0EE408AC0E700BF17B7D1382F
:10B710003333333F000000006F12833A52B87E3F4C
:10B72000085202201033022010A3022000003442ED
:10B730008FC2D53F9A99193FF8B5044682F032FE80
:10B740000368DB689847054610B900252846F8BD10
:10B75000204604F5E04608F0E3FF04F5E343D6F89D
:10B760003423074644339A4205D104F5004393F845
:10B77000B83C022BE9D804F50A40D83011F0AEFBF2
:10B780000028E2D1D6F8340303689B6B984758B978
:10B7900096F84833002BD9D004F5405494F9185B3F
:10B7A000023D18BF0125D1E7084BD3F834030368E5
:10B7B0005B6B98470028EBD004F5405494F9553B57
:10B7C000002BC2D0032BC0D03D46BFE710A3022000
:10B7D000F0B5044600F5E04700F50A4004F5A4453D
:10B7E000D83064352DED028B83B097EDE18A11F0EE
:10B7F0008BFA002841D104F50046D6F80C0B0368FB
:10B800009B689847D6F8AC3D5B0220D5D6F80C3B38
:10B8100093ED437AD3ED097A67EE877A9FED2F7A1D
:10B82000F4EEC77AF1EE10FA11DB04F5A044F7EE5E
:10B83000006A94ED9A7A67EE877A86EEA77AB4EE7C
:10B84000667AF1EE10FA36FE877A84EDE57ADFED5E
:10B85000247AF0EE480A90ED280A284620EE270ABE
:10B86000B5F0FCFD28468DED010AFFF72DFE9DED9C
:10B87000010A03B0BDEC028BF0BD04F5DF43D7F83D
:10B88000342308339A4226D104F58043D3F8203F6D
:10B89000B3F90860003E18BF012604F50054D7F83C
:10B8A000543AD4F8F0401C1B97F8503A3BB14FF48F
:10B8B00000610C48FFF782FC80F00100C3B2B0EEDB
:10B8C000480A32462146284603B0BDEC028BBDE84B
:10B8D000F040B5F0C7BD0026DFE700BF0000003430
:10B8E000E02E65421033022010B5044608F0B8FA85
:10B8F00098B104F5E042D2F8543A03F58C41503146
:10B90000C2F8541A04F50051D1F8F0100029BEBF56
:10B91000A3F58C43503BC2F8543A2046FFF758FF3A
:10B920000420BDE8104084F03DBB00002DE9F04745
:10B9300000F50A44054600F5E047D83405F5A7466A
:10B940002DED048B2046D7EDE18A483611F0DCF965
:10B95000002845D105F50044D4F80C0B0368DB68DA
:10B960009847D4F8AC3D5B0222D5D4F80C3B93ED5C
:10B97000447AD3ED0B7A67EE877A9FED557AF4EE31
:10B98000C77AF1EE10FA13DB05F5A045F7EE006A71
:10B9900095EDF37A05F2FC4567EE877A86EEA77A95
:10B9A000B4EE667AF1EE10FA36FE877A85ED007A0B
:10B9B00090ED280AF0EE680ADFED467A304620EE78
:10B9C000270AB5F099F9B0EE408A3046FFF798FDA6
:10B9D000BDEEC80ABDEC048BB8EEC00ABDE8F08726
:10B9E000204605F540540FF015FD9FED3B9A04F6F7
:10B9F000483304F52F648146462093ED008AD7F83A
:10BA0000583A28EE098ABDEEC88A18EE102A1A4460
:10BA100008EE102A84F0DAFAD4ED007A05F5DF4357
:10BA2000B8EEC88AD7F834030833A0EE278A9842C4
:10BA3000FDEEC87A17EE904A47D105F58043D3F85A
:10BA4000243FB3F90880B8F1000818BF4FF001088F
:10BA5000B9F1000F1ED103685B699847D0B9D7F8D8
:10BA6000340303689B6B9847A0B905F50049D9F8E2
:10BA7000443E022B0ED1284614F06AF950B109F267
:10BA8000FC69D9ED007A67EE897AFDEEE77A17EE68
:10BA9000903A1CB205F50055D5F8F430E41A97F841
:10BAA000503A3BB14FF400610C48FFF787FB80F040
:10BAB0000100C3B2B0EE680A424621463046BDECF2
:10BAC000048BBDE8F047B5F0FFB94FF00008BFE7C1
:10BAD00000000034E02E65420000C842103302200E
:10BAE00010B5044618F066F868B100B200EB4000EB
:10BAF000C0EB001300EE103AB8EEC00A1320BDE808
:10BB0000104084F04FBA2046FFF710FFF6E7000020
:10BB100010B51048FFF710FED0B10F4811F014FB1C
:10BB2000B0B10E4C042084F051FAD4F8200F82F00A
:10BB30003DFF042084F036FA132084F047FAD4F84D
:10BB4000240F82F033FF1320BDE8104084F02ABA9E
:10BB500010BD00BF10330220E8BD02201073022088
:10BB600070B52DED028B0446FFF7E6FD002800F0CE
:10BB7000A38004F5E04504F5DF42D5F834334032C4
:10BB8000934200F0998004F5DF427C32934200F04A
:10BB900093806032934200F08F80443A934200F0E9
:10BBA0008B801C32934200F0878004F5E2425032D1
:10BBB000934200F0818004F5E2426C3293427BD0E4
:10BBC00004F5E3420832934276D004F5E34228328A
:10BBD000934271D004F5E342643293426CD004F591
:10BBE0000A40D83011F0B0FA002865D004F5DF43E0
:10BBF000D5F8342324339A425ED0F6EE008A04F559
:10BC00008046D6F8200F82F093FDB4EEE80AF1EEFC
:10BC100010FA3EDDB0EE087AFFEE007AE0EE077A29
:10BC2000B0EE670AD6F8382FD5F8543A07EE902AC6
:10BC30005142B8EEE77A07EE903AF8EEE77AE7EE8F
:10BC4000007AFDEEE77A17EE900AC5F8540A3AF04A
:10BC500065FE04F5E143D5F834234033C5F8540AB2
:10BC60009A4222D0D6F8240F82F062FDB4EEE80AA0
:10BC7000B0EE408AF1EE10FA21DCFEEE007AB4EE6E
:10BC8000E70AF1EE10FA22D5B0EE087AF7EE007A64
:10BC900019E0FEEE007AB4EEE70AF1EE10FAC1D533
:10BCA000B0EE087AF7EE007AB8E74FF480512548F5
:10BCB000FFF784FA0028D5D0BDEC028B70BDB0EE42
:10BCC000087AFFEE007AE8EE077AB0EE678A20463F
:10BCD00008F0C6F808B1B1EE488AB5EEC08AD5F8CA
:10BCE000583A04F56B5406F63C7607EE903A9FED11
:10BCF000166AF1EE10FAD4ED016A96ED007AF8EECC
:10BD0000E77ACCBF28EE268A27EE488A66EE866A56
:10BD100027EE067AE8EE067AFDEEE66ABDEEC77A11
:10BD200016EE902A17EE101AFDEEE77A17EE903A0B
:10BD300017EE900AC5F8583A3AF0F0FDC5F8580ADF
:10BD4000BAE700BF103302200000C842F0B5044635
:10BD500004F500462DED028B83B0C9F0CBFA96F8BE
:10BD6000EC3B074653B1D6F8140C04F5F44204F545
:10BD7000F4410368543258311B6A984704F5E04592
:10BD8000D5F84433FB1AB3F5FA6F03D9D5F8340369
:10BD900009F0D2FB04F5DF43D5F83423C5F844732A
:10BDA0002433654F9A4204D004F5E24334339A4277
:10BDB00005D1D7F8340303681B6898475CE0204638
:10BDC00007F022FE0028F4D005F6AC1304F5A440D9
:10BDD000D5EDE10A93ED000A6430CDED010AB5F02E
:10BDE0003DFB05F51B6304F5A740DDED010AF0EE10
:10BDF000408A483093ED000AB4F07EFFB0EE408AEE
:10BE00000420B0EE680A84F0CDF81320B0EE480AA2
:10BE100084F0C8F804F5A04393F94235002B00F0F4
:10BE2000838005F6C413DFED457A04F5AA4093ED4F
:10BE3000008A95F8C8392C3028EE278A002B70D05C
:10BE400005F6B4150021DDED010A95ED000AB5F007
:10BE500031FF38EE008AB0EE480A152007F6B81711
:10BE600084F0A0F8B0EE480A1A2084F09BF897ED11
:10BE7000000A462084F096F80021204614F022F9AA
:10BE8000B0EEC00ADFED2E7AB4EEE70AF1EE10FA5A
:10BE90004DD506F51966B1EE047AD6ED007AF0EECE
:10BEA000E77AF4EEC77AF1EE10FA40D504F5AA600D
:10BEB0001FF026F8F6EE007AB0EEC00AB4EEE70AFC
:10BEC000F1EE10FA33D504F50B55F0EE087A95ED46
:10BED0000F7A3C35B4EEE77AF1EE10FA27D504F587
:10BEE000A4406430B5F02EFB04F5A7404830B5F00F
:10BEF0009BF804F5AA402C30B5F0E8FFF7EE007A85
:10BF000095ED007AB4EEE77AF1EE10FA0FD504F56C
:10BF1000AD402C3003B0BDEC028BBDE8F040B5F075
:10BF20001FBDB5F0D3FF96E79FED068A93E703B0F8
:10BF3000BDEC028BF0BD00BF10A302200000344214
:10BF4000000000340000000000F5405393F9A33ACC
:10BF5000012BC5BF00F59F40DFED067A9FED060A75
:10BF600090ED410A4FF04600C8BF20EE270A84F04A
:10BF700019B800BF0000C842000000002DE9F041E0
:10BF800000F5E04805462DED028BD8EDE18A13F06F
:10BF9000DDFC0746D8F8340305F5AA4603682C36BD
:10BFA0001B6A984798B14E4CD4F8E039002B0EDD4F
:10BFB000C9F0A0F9D4F8E039C01A40F6B733984276
:10BFC00005D8B4F9D4493046B5F08CFF7AE005F5D0
:10BFD000004305F5405493F8393E43B1B4F9343B7E
:10BFE000002B04DD05F5A04393F9423513BB05F59D
:10BFF000DF45D8F834330835AB426DD00021B0EEC0
:10C00000680A3046B5F0FAFC0546042083F0DEFFEE
:10C0100004F6E8232AB293ED007A07EE902AF8EEB0
:10C02000E77AE0EE077AFDEEE77A17EE904A3C44B5
:10C0300024B2C8E70121284613F080FE9FED297A3B
:10C04000B4F9343BC0EE077A9FED270A08EE103AA8
:10C05000D8F8543AB8EEC88A28EE278A07EE903A04
:10C06000F8EEE77A67EE807A9FED200A27EE800AE5
:10C070001AF12CFFB4F9AC3ADFED1D7AF0EE680A44
:10C080000021304620EE270A07EE903A08F5266395
:10C09000F8EEE77A93ED007AB4EEE77AF1EE10FA73
:10C0A00058BFF0EE477A80EE277ADFED127AB0EED5
:10C0B000480AA7EE270AB5F0FDFDBDEEC00A10EE56
:10C0C000103A1CB2204641F294120B49BDEC028B8F
:10C0D000BDE8F0413AF032BC391E18BF01218EE7AD
:10C0E00010A3022000A08C450AD7233C35FA8E3CD1
:10C0F0000AE81C41E02E65426CEEFFFF38B500F502
:10C10000A0430546D3F87C090368DB6898470146DD
:10C1100005F5AD402C30B5F005FC04B22846FFF71C
:10C120000BFB70B107EE904A05F58045B8EEE70AC3
:10C13000D5F82C0F82F03AFCBDEEC00A10EE103A92
:10C140001CB2204641F294120249BDE838403AF050
:10C15000F5BB00BF6CEEFFFF38B5B02290F8143489
:10C16000F7EE007A054602FB030300F5E04493ED89
:10C17000837AB4EEE77AF1EE10FA1DD5002113F0C0
:10C18000A1FFB0EEC00ADFED417AB4EEE70AF1EEAE
:10C1900010FA11D5D4F8403A012B0DD0072B0BD053
:10C1A000002304F65814284604F8043C00232360B6
:10C1B000BDE8384013F0CABBC9F09CF8D4F85C392C
:10C1C000C4F85C09C31A2846B3F57A7F84BF0023FC
:10C1D00084F8543913F0BAFBD4F8403A07EE100A49
:10C1E000012B2DD0072B2BD0B8EEC77ADFED286AB4
:10C1F00005F54052C7EE267AB2F9F82A00EE102A69
:10C20000B8EEC00A27EE800ADFED207AB0EEC07AE1
:10C21000B4EEE77AF1EE10FA14D4002384F854391E
:10C2200005F5AD4094F854392C30DBB9B5F058FA27
:10C2300000B241F294121749BDE838403AF07EBB93
:10C240009FED150A94F85429002AE9D1012293425E
:10C2500084F85429E4D0072B1EBF04F6581300229B
:10C260001A60DDE704F65814DFED0C7A94ED007ADD
:10C2700067EEC77A9FED0A7A67EE877AFDEEE77A76
:10C2800017EE901AB5F04EFBD2E700BF0000003465
:10C2900000A08C456CEEFFFF00000000E02E654220
:10C2A0000000C84270B500F50546044678362DED0D
:10C2B000028B304682B0C2F029FF0546E8B904F58A
:10C2C0008043D3F8203FB3F9083083B904F509431C
:10C2D000D3ED247A04F56B53F0EEE77A93ED0D7A03
:10C2E000F4EEC77AF1EE10FA4CBF01250025304676
:10C2F000C2F026FF002808BF00253046C2F006FF26
:10C3000050BB04F5E043D3F8503901331ED01DBBB8
:10C310009FED1C8A2046FFF731FE07EE900AB8EE2B
:10C32000E70A8DED010AFDB9152083F03BFE9DED76
:10C33000010A1A2083F036FE04F50B40603002B08B
:10C34000BDEC028BBDE8704004F060B9002DDFD079
:10C350002046FFF701FF02E02046FFF7CFFE07EE81
:10C36000900AB8EEE78AD5E71A2084F06BF99DEDC4
:10C37000010A08B9B0EE480A152083F013FEB0EEAA
:10C38000480AD6E70000000000F56B53DFED157A90
:10C390009FED156A10B5D3ED016A00F580430446A0
:10C3A00003F63C7203F57E6366EEA76A04F5E0448B
:10C3B00092ED007A27EE277AD3ED2A7AFDEEE66A2F
:10C3C00067EE867ABDEEC77A16EE902AFDEEE77A22
:10C3D00017EE101A17EE900A3AF0A0FAC4F8580AAD
:10C3E00010BD00BF0000C842A00CB34510B5044604
:10C3F00015F08CFD031E2CDB04F5405191F9A32AA6
:10C400009A4226DD04F5E040D0F8404A022C20D0C4
:10C4100001F6FC21D31ADFED0F6A07EE102AD1EDE9
:10C42000007AB8EEC77A66EEE76A07EE903AD0F87F
:10C43000583AF8EEE77A87EE876A07EE903AF8EE18
:10C44000E77AE6EE867AFDEEE77A17EE903AC0F8E4
:10C45000583A10BD0000C84270B500F5E0469FEDA7
:10C46000590A9FED597A04462DED028BD6F8543ABD
:10C47000B7EE008A07EE903AF8EEE77A67EE807A38
:10C480009FED520AF0EEE76AF4EE476AF1EE10FA19
:10C4900077FE277A27EE800A19F1A6FE3AF07CF89B
:10C4A000C8EE007A06F65C23C3ED007A04F500437B
:10C4B00093F8EC2BB2B1D3F8140C04F59E41036849
:10C4C00038315B6A984768B104F58044D6F8540A5D
:10C4D000D4F8382F51423AF021FAC6F8540ABDEC8C
:10C4E000028B70BD04F5405595F9D43A002BF6D077
:10C4F000204607F0B5FC0028F1D104F50D402030AE
:10C5000015F002FF0028EAD1B5F9AC3A06F526622B
:10C51000012BD2ED006AB8BF012307EE903AF8EE86
:10C52000E77A86EEA77AB4EEC87AF1EE10FA15D85B
:10C5300004F5804440F6C4122549D6F8540A3AF06E
:10C54000EDF940F6C413C6F8540AD4F8382F9A42CD
:10C55000D4BFC4F8382FC4F8383FC0E706F65C23D0
:10C56000D3ED007AF4EEC77AF1EE10FAB7DD88EE7B
:10C57000070A04F5804420EE000A1AF165FEDFED9B
:10C58000157A40F6C413D6F8540A20EE270ADFEDD8
:10C59000127A20EE270AFDEEC07A17EE905A9D42DD
:10C5A000B8BF1D462A4669423AF0B8F9C6F8540A9F
:10C5B000D4F8383FAB42D4BFC4F8383FC4F8385F32
:10C5C0008DE700BF0AD7233C0000AA4235FA8E3C13
:10C5D0003CF6FFFFE02E65420000C84200F5A04394
:10C5E00010B50446D3F87C0903681B68984704F526
:10C5F0008043D3F8382F51423AF090F904F5E043E4
:10C60000C3F8540A2046BDE81040FFF725BF0000DC
:10C6100070470000704700000120704708207047F5
:10C6200001207047014B93F8E00A70471063022025
:10C63000034B93F9440A003818BF0120704700BF2C
:10C6400010730220014B93F9E20A70471063022035
:10C65000064B13B5D3F834030831CB680468009354
:10C66000646C0EC9A04702B010BD00BF10A3022029
:10C67000084B82B09FED087AD3EDDA7AF8EEE77ACC
:10C6800067EE877AFCEEE77ACDED017A9DF804003B
:10C6900002B0704710A30220CDCC4C3D7047000083
:10C6A00038B5254DD5F8340303685B6898471928D9
:10C6B0003BD8DFE800F00D38360D0D363636363A09
:10C6C0003838383838383A36363636383A0D383819
:10C6D00040241A4B93F80D2712B193F80C370BB97D
:10C6E00044F01004164BD5F834239A42A3F11C03EE
:10C6F00003D09A4218BF44F01004124991F9551B17
:10C70000A9B19A4215D0032902D10F4B9A4201D107
:10C7100044F040040D48B2F0F7FC50B144F08004FE
:10C7200007E01024D5E71824D3E70124D1E79A4283
:10C73000F0D144F0010038BD10A302201083022084
:10C7400044A402201063022088A3022074BD0220AA
:10C7500008B5044808F06CF900280CBF012002203D
:10C7600008BD00BF10330220F0B52DED028B8BB059
:10C7700005461CF05FF84FF480710446D0F804724F
:10C7800090ED828AD0F80C621F48FEF717FD60B961
:10C790001E4BB7EEC87A93ED006A9FED195BB7EEBA
:10C7A000C66AA6EE457BB7EEC78B19480EF054FF5C
:10C7B00030B1184BD3F89C3D5F6893ED028ADE6878
:10C7C0002D7CC8F097FDD4F81823D4F81C33D4F886
:10C7D00014130892272209931C23039028460791DB
:10C7E0001E2104978DED058A0696CDE9003203AA35
:10C7F00078F0DAFF0BB0BDEC028BF0BDAFF3008038
:10C80000000000A046DF913F10330220586E022046
:10C81000E8BD022010B3022038B5C5780B460446A7
:10C820003522352D4FF00001184628BF35251DF162
:10C8300051FC04F10C012A46BDE838401DF100BC52
:10C8400008B5024815F062FB00B208BD10330220A3
:10C850007FB500230393049305931BF0EBFF00F5D2
:10C860005A7003AB07C883E8070018463FF0B4FDD1
:10C87000F1EE047A20EE270ADFED087AB4EEE70A3B
:10C88000F1EE10FA58BFB0EE670AFCEEC07ACDEDBB
:10C89000017A9DF8040007B05DF804FB00007F43B7
:10C8A00037B50D4640F2EF22124804F0F1FF2C7824
:10C8B00014F004040AD0032269680F4823F086F8B4
:10C8C0000C4803B0BDE8304004F0C8B801AA2146C6
:10C8D000284623F04FF90028F2D0DDED017A2246F8
:10C8E0009FED067A67EE877AFDEEE77A17EE901AEB
:10C8F000E3E700BF1033022074BC02200000C842EE
:10C900000148C6F06BB900BF847F0220012310B537
:10C91000044C84F80F377AF081FC002384F80F3739
:10C9200010BD00BF1083022070B5144605460E46A8
:10C9300007481146B6F0F4F921460648C5F084FED2
:10C94000224631462846BDE870407EF02FBD00BF2C
:10C9500070BB0220808102202DE9F041214F4FF071
:10C9600000080C4615464FF47A7306462DED028BEF
:10C970009FED1D8A82B0B0EE480ACDE90028B1F9DA
:10C980000220D7F8201F7FF063F80123B0EE480A99
:10C99000B4F90020D7F8241F3046CDE900534FF4F6
:10C9A0007A737FF055F84346B4F904203046D7F83F
:10C9B000281F9FED0E0ACDE900587FF049F8B0EE30
:10C9C000480A4FF47A73B4F90620D7F82C1F304682
:10C9D000CDE900587FF03CF802B0BDEC028BBDE819
:10C9E000F08100BF107302200000FA4400007A4476
:10C9F000074B10B540F24D3493F9D02C40F24D1353
:10CA0000002A08BF1C467AF051FA204310BD00BF2F
:10CA100010A302201FB51BF00DFF0446684622F04C
:10CA2000CFFF694620461BF01DFC17480EF014FE90
:10CA3000E8B1164B03F5A872D3F83413914220D015
:10CA400003F58053DDED017AD3F8103BF8EEE77A79
:10CA500093ED0F7A77EE877A9FED0D7A67EE877AFE
:10CA6000FDEEE77A17EE903A18B204B010BD019CC3
:10CA7000084804F0E7F8231807EE903AF8EEE77A52
:10CA8000EAE70020F1E700BFE8BD022010A3022082
:10CA90000AD7233C1033022007B51BF0CBFED0EDA4
:10CAA000DA0A90EDDB0AF1EE600AB1EE400A1AF103
:10CAB00033FCDFED097A20EE270A39F0B3FDF6EEFC
:10CAC000007A20EE270AFCEEC07ACDED017A9DF8BF
:10CAD000040003B05DF804FBE02E654210B5044687
:10CAE00023F062FC204610BD08B51B482DED028BDB
:10CAF0000EF0B2FDB2EE048AF8B117480EF05CFCFD
:10CB0000C0B1164BD3F8140B03689B689847DFED50
:10CB1000147AB4EEE70AF1EE10FA58BFB0EE670AE5
:10CB2000C0EE087AFCEEE77ABDEC028B17EE903A85
:10CB300098B208BD9FED0B0AF2E70B4BDFED087AC8
:10CB400093ED007AB4EEE77AF1EE10FA58BFB0EE4A
:10CB5000677AC7EE087AE5E7E8BD022010B3022045
:10CB600000FF7F470000000088AC0220002310B5C2
:10CB70000A4C84F893397BF059F904F17803D4F81E
:10CB800034239A4208D194F8683A2BB904F6642009
:10CB9000BDE8104042F070BD10BD00BF10A30220E0
:10CBA00013B5124C94F81A1304F5E27018F0B6FF9E
:10CBB00078B194F81A1304F5E27019F025FA40B12F
:10CBC00094F81A1304F5E27002B0BDE8104019F0B1
:10CBD0005FBA1BF02FFE01A91BF0F4FB18B19DED0D
:10CBE000010A02B010BD9FED020AFAE710630220AD
:10CBF00000000000044B93F8EC0B20B1D3F8140CA8
:10CC000003681B6B1847704710B3022008B5084B28
:10CC1000D3F8302C002A03DCBDE808407AF0BEB817
:10CC200003F5356076F0D4FE90ED000A08BD00BF34
:10CC300010730220114808B500F58C73D0F8342326
:10CC40009A4214D0B0F94C339BB990F81D3983B98E
:10CC500090F849336BB990F8293A63B9A0F5E040F0
:10CC600007F0E6FE00280CBF0320042008BD0220C8
:10CC7000FCE70520FAE70620F8E700BF10A3022032
:10CC8000224B10B503F59A72D3F8343390B00446B2
:10CC9000934238D000231E48029322F081FE0146C1
:10CCA00018B902AA1A4822F0C7FE247CC8F022FB59
:10CCB000184B5721DDED027AD3F86C29D3F870397F
:10CCC000F8EEE77A9FED147A0593002367EE877AF2
:10CCD0000793089309930A930B930C930D930E9368
:10CCE0004FF6F853CDED067AADF83C300023CDE990
:10CCF00003028DF83E30962233232046CDE90032E0
:10CD000003AA78F051FD10B010BD00BF10A302209F
:10CD100074BC022010B302200AD7233CF0B58DB0BA
:10CD20000446C8F0E7FA184AD2F8103CC31A642B3C
:10CD300028D8D2F80C3B0290D3F88C10D3F890206E
:10CD4000D3F88460D3F88850D3F8DC70D3F894E03B
:10CD5000D3F898C0D3F89C3006921622099300238A
:10CD6000059153218DF82C302523207CCDF81CE033
:10CD7000CDF820C00A9703960495CDE9003202AAA7
:10CD800078F012FD0DB0F0BD10B302201FB51348AE
:10CD90000EF062FCA0B1124B9FED120AD3F80C0BFF
:10CDA0006C303EF097FEDFED107A21EE271AFCEE94
:10CDB000C17A17EE900AC0F3470005B05DF804FB96
:10CDC0000A4BD3F87C0903681B69984739F0AAFC21
:10CDD000C82390FBF3F0C0B2EFE700BFE8BD02202C
:10CDE00010B302209F0CB3450AD7233C10830220C6
:10CDF00010B57AF055FA044678B9094800F178037D
:10CE0000D0F8342380F893499A4206D190F8683AD2
:10CE10001BB900F6642042F02FFC204610BD00BF75
:10CE200010A302202DE9F043904E044606F59A73B4
:10CE3000D6F834239A422DED088B91B000F0E980AA
:10CE40008B48DFED8C8A0EF007FCDFED8B9A9FEDAF
:10CE50008B9A00286DD086480EF0AEFA002868D074
:10CE600006F580589FED860AD8F80C0B6C303EF022
:10CE700031FE08F6E420B0EE60AACDED070AB0EE70
:10CE8000418A8DED081AF0EE40AA8DED060AB8F041
:10CE900079FDD8F8103B014604A893EDDE7B93EDB5
:10CEA000DC6BB7EEC77BB7EEC66B8DED057A8DED0B
:10CEB000046A3EF0FFFA09A88DED090AB0EE680A8F
:10CEC000CDED0A0A3EF006FB28EE288A02A894F867
:10CED0001090CDED030A6AEEA8AABDEEC88A8DEDCA
:10CEE000020A2AEE28AA18EE103A1DB23EF066FB9E
:10CEF000DFED647A02A820EE270ABDEEC00A10EE2C
:10CF0000103A1FB23EF0A4FBB4EEE90AD6F834237F
:10CF1000F1EE10FA58BFB0EE690ABCEEC00A10EE8E
:10CF2000103A9CB206F5A8739A4277D1DFED568A83
:10CF30007AE0D6F8543ADFF8549107EE903AD6F8F2
:10CF4000583AD9F87C79B8EEE7BA07EE903A3B68E0
:10CF50003846F8EEE7AA94F810809B682BEE28BAC2
:10CF6000984707EE900A38466AEEA8AAF8EEE77AE4
:10CF700067EEA87AFDEEE77A17EE903A1DB23B68AD
:10CF80001B69984707EE900AA9F5A040F8EEE77AEA
:10CF900067EEA87AFDEEE77A17EE903ADFED367A83
:10CFA0001CB206F6781393ED00AAB4EEE9AAF1EEEE
:10CFB00010FA58BFB0EE67AA03F044FE3B6808EED3
:10CFC000100AD6EDDC7A38465B6927EE899A9847D5
:10CFD000BCEECAAAB721B8EEC88A09AA40468DEDB0
:10CFE00009BA1AEE103ACDED0AAA68EE288A8DED3C
:10CFF0000C9AADF83C301A238DED0D0ACDED0B8A5D
:10D00000ADF83850ADF83A40CDE900313E2178F026
:10D01000CBFB11B0BDEC088BBDE8F083D8F8103B1A
:10D02000D3ED0F7A67EEA88AD8F8143BD6EDDC7AF8
:10D03000186927EE899ABDF091FDB7221A233E2187
:10D040004846CDED09AA8DED0AAACDED0B8A8DEDEE
:10D050000C9A8DED0D0AADF83850ADF83A70ADF878
:10D060003C40CDE9003209AAD1E700BF10A302205D
:10D07000E8BD02200AD7233C00FF7F470000C842DA
:10D080009F0CB345E02E6542000000001083022093
:10D0900001480EF0A3B900BFE8BD022008B5034B5C
:10D0A000D3F8340303685B68984708BD10A30220D7
:10D0B00030B587B005461BF0BDFB04462D7CC8F09B
:10D0C00011F9D4F884220021D4F888320492CD22B8
:10D0D0000593102302902846039142F60C31CDE9C6
:10D0E000003202AA78F060FB07B030BD30B52DEDFC
:10D0F000028B89B005461BF09DFB00F55A7302AC0C
:10D100002D7C93E8070084E80700DDED020A9DED21
:10D11000030AF1EE600AB1EE400A1AF1FDF820466A
:10D12000B0EE408A3FF058F9049B0122DFED0A7A05
:10D13000A82107930C2328EE278A28468DED060A9E
:10D14000CDE9003205AA8DED058A78F02DFB09B0F6
:10D15000BDEC028B30BD00BFE02E6542F0B5054648
:10D1600016460C462DED028BB0EE408A8DB000299C
:10D1700030D0007C78F09AFA0746287C79F0B4F930
:10D1800000F121039F4207D2287C0DB0BDEC028B39
:10D19000BDE8F04077F0A8BC636922690893636A30
:10D1A000A069CDF82530236AE16807926222CDF8A4
:10D1B00029302123276805900691C221287C0397F6
:10D1C0008DED048A8DF82460CDE90032192303AA7D
:10D1D00078F0EAFA0DB0BDEC028BF0BD70B5494EA7
:10D1E000044606F59A73D6F834239A4200F08980F3
:10D1F000A6F58045B5F8863BDA0713D542480FF00F
:10D200004DFC002877D006F58053D3F80C0B03684B
:10D210009B68984700F1A00191ED010A0122204688
:10D22000FFF79CFFB5F8863B9B0712D536480FF0F9
:10D2300035FC002861D0354BD3F80C0B0368DB6854
:10D24000984700F1A00191ED010A02222046FFF764
:10D2500085FFB5F8863B580712D52B480FF01EFC0A
:10D2600000284CD0294BD3F80C0B03681B69984756
:10D2700000F1A00191ED010A03222046FFF76EFFA5
:10D28000B5F8863B190708D52149052220460B46EB
:10D29000043993ED000AFFF761FFB5F8863BDA0623
:10D2A00014D5D6F8403A042B10D11BF0C3FA064629
:10D2B0001848C1F069FF96EDC70ADFED177A0146FD
:10D2C0000622204620EE270AFFF748FFB5F8863BE6
:10D2D0009B0616D50C480FF0E1FB90B10B4B204696
:10D2E0000422D3F8101BBDE8704091EDAE0A01F5A1
:10D2F0002D71FFF733BF09498EE70949A3E70949B3
:10D30000B8E770BD10A30220E8BD022010B30220D0
:10D31000F089022088B80220E02E6542A88602200B
:10D3200010880220908902202DE9F04304462DED5B
:10D33000028B89B0007C78F0B9F90546207C79F041
:10D34000D3F8431D9D4207D2207C09B0BDEC028B6F
:10D35000BDE8F04377F0C8BB19F008F8064600288E
:10D360004BD0C7F0C7FF002780469FED268A94F870
:10D370000F5304AB05AA30463D44009303AB01357F
:10D3800005F00105294618F0D7FF88B3059BA8EBE7
:10D390000303B3F5FA6F2BD8207C78F087F9814628
:10D3A000207C79F0A1F8431D207C994523D39DED85
:10D3B000037A1422DDED047A43F2782127EE087A0D
:10D3C0008DF81C5067EE887ABDEEC77AFCEEE77ADE
:10D3D00017EE103AADF8183017EE903AADF81A3053
:10D3E0000523CDE9003206AA78F0DEF984F80F5360
:10D3F0001FB90127BBE777F077FB09B0BDEC028BC3
:10D40000BDE8F0830000C842402938B505463ED04B
:10D4100017D8272924D008D81B2947D024292CD055
:10D420002846BDE838407EF0B7BD2829F8D116213E
:10D4300077F06CFB0446C0B1297C22486FF00AFDEE
:10D4400014E043292ED0532932D04229E8D11021AB
:10D4500077F05CFB044640B12846FFF729FE05E063
:10D46000122177F053FB044610B90024204638BD42
:10D47000297C14486FF014FCF8E70C2177F046FB88
:10D4800004460028F1D02846FFF730FEEEE72621BB
:10D4900077F03CFB04460028E7D0297C0A489FF03F
:10D4A000C9FBE3E7017C0948C1F024FE0124DDE764
:10D4B000052177F02BFB04460028D6D02846FFF73D
:10D4C00033FFD3E7E0AF022040BA022088B8022041
:10D4D00070B504460E462CF0E1FDB02390F8F4122E
:10D4E00003FB01012046DC3104F0D2FC0546C0B14B
:10D4F0003EB11BF09FF990F87C3243F0020380F8B4
:10D500007C3204F5E043D3F8340304F5E1432433DB
:10D51000984204D004F5E3444434A04201D107F01A
:10D5200011FF284670BD000073B5164601910446F0
:10D530001BF080F901991AF05DFD0546C0B13EB1BE
:10D540001BF078F990F87C3243F0020380F87C32CB
:10D5500004F5E043D3F8340304F5E143243398425F
:10D5600004D004F5E3444434A04201D107F0EAFEBC
:10D57000284602B070BD000030B5054685B00C46A7
:10D58000D1E904013AF07CFB40B1684622F018FA78
:10D590006A46214628467EF069F908B9022067E00C
:10D5A00040F24F326946334804F072F9D4ED037A01
:10D5B000F4EE677AF1EE10FA22D6F0EEE77A9FEDFC
:10D5C0002E7AF4EEC77AF1EE10FA54BF012200224F
:10D5D0009DF800306846294962F341038DF8003018
:10D5E00022F064FB0028D9D16946254895F01EFA3F
:10D5F00040B973F019FC0522162173F0C5F9CDE787
:10D600000022E5E7D4ED017AFDEEE77A17EE903AD5
:10D61000DB0706D41B4B03F1F802D3F834339342F3
:10D6200025D119490222134814F052FA9DF800102E
:10D6300011F0040102D1684622F08CFA69460D48C7
:10D6400004F072FB94ED020AB4EE400AF1EE10FA17
:10D650000BD6B5EEC00AF1EE10FA06DD9DF800100B
:10D660000948C1F3400109F075F9002000E00420E9
:10D6700005B030BD103302200000003464BC02202D
:10D68000046A022010A3022008A4022010B52DED88
:10D69000028BD1ED017A8AB091ED008A0446FCEE4E
:10D6A000E77A05AACDED037A9DF80C107EF0C8F854
:10D6B000C8B1DFED0E7A0022059B06A868EE277A36
:10D6C00011460093FDEEE77A17EE903A22F098F9B2
:10D6D0002368204606A9D3F8E830984700200AB00E
:10D6E000BDEC028B10BD0220F9E700BF0000C8426C
:10D6F000F0B54AF2F97207460D462DED028B8B8B81
:10D7000083B0934271D04AF2FA72934200F0B5802E
:10D710004AF2F872934240F0FE80814E06F1F8031F
:10D72000D6F834239A4240F0F880D1ED007AFDEE2D
:10D73000E77A17EE903A0BB1022451E0A6F5804348
:10D7400091ED010AB3F9AE2A07EE902AF8EEE77AD6
:10D75000B4EEE70AF1EE10FAEEDCB3F9AC3A07EEFC
:10D76000903AF8EEE77AB4EEE70AF1EE10FAE3D475
:10D770009FED6C8A06F6EC1720EE088AD7ED000ABA
:10D78000B0EE480A38F09AFE044608B1002427E0BB
:10D7900087ED008AC7F0AEFDC6F8F40906F51F63F1
:10D7A000D5ED027A9FED607AF0EEE77AD7ED006A68
:10D7B000F4EE477A9FED5D7AF1EE10FA48BFF0EE95
:10D7C000477A96EDDA7AB8EEC77AC3ED007AF4EECE
:10D7D000C76AF1EE10FAD9D5F1EE677AC3ED007A97
:10D7E000204603B0BDEC028BF0BD4D4E06F1F803B0
:10D7F000D6F834239A4240F09080FFEE000A91ED73
:10D80000060A38F05BFE002896D1DFED490A95ED57
:10D81000060A38F053FE044600288DD101AA95F877
:10D82000201038467EF00CF8002885D095F820307E
:10D8300006F6F8109FED3B7A06F608263372D5ED12
:10D84000067A019A67EE877AFDEEE77A17EE901A6C
:10D8500022F0BCF8C7F04EFD7060D5ED027A9FED66
:10D86000327AF0EEE77AF4EEC77AF1EE10FA4ABFB8
:10D87000304BC6ED007A3360B2E7294C04F1F8036F
:10D88000D4F834239A4248D191ED010AB5EEC00A8A
:10D89000F1EE10FA3FF550AFDFED277AB4EEE70A6C
:10D8A000F1EE10FABFF648AF38F0D2FED5ED007AAF
:10D8B0009FED228AFDEEE77A20EE088A17EE903A75
:10D8C00013BB01231E4E84F8203A06F110030FCB40
:10D8D00086E80F001B489FF061FF04F614239FEDBC
:10D8E0001A7A83ED008A04F61823D5ED027AF4EE55
:10D8F000C77AF1EE10FA77FE877AC3ED007AC7F0A7
:10D90000F9FCC4F81C0A41E7012B7FF415AF022390
:10D9100084F8203ADEE7032462E7042460E700BFCE
:10D9200010A302200000C8420000003400007A4426
:10D930000000000000007A440000B44335FA8E3C39
:10D9400054BC02208C800220CDCC4C3D37B5124D0A
:10D950000C46D5F8340303681B6A984740B905F1B3
:10D960007803D5F834239A4202D0042003B030BDA6
:10D97000D4ED007AD4ED020AFCEEE77A94ED010AC8
:10D980000648CDED017A9DF8041004F041FF00280F
:10D99000EBD00020EAE700BF10A3022010330220E2
:10D9A0001346242210B50C46184600211CF192FBA8
:10D9B000A27F8277E27FC277072280F82020A28BA5
:10D9C0008283D4ED067AF1EE677AC0ED067A10BD57
:10D9D00010B48C8B162C03D15DF8044BFFF7E0BF1D
:10D9E0005DF8044B7CF026BD08B591F82030072B7C
:10D9F0000ED1094890F8EC3B43B191ED060A00F6D0
:10DA0000D820B1EE400A0EF011FE18B9042008BD6E
:10DA10000220FCE70020FAE710B3022008B5D1EDA0
:10DA2000007A9FED087AF0EEE77A0748F4EEC77ABD
:10DA3000F1EE10FA54BF0121002106F00BFA00208C
:10DA400008BD00BF000000341033022010B5D1ED36
:10DA5000007AFCEEE77A17EE903A9CB2012C02D0E5
:10DA6000022C06D084B9114821468EF01DFB0020FF
:10DA700010BD0F4890F8C43C5B0707D57EF044F911
:10DA80000C4A052176F0E0FD0420F1E790F9B03C66
:10DA90001BB97EF039F9084AF3E7A0F5E0400CF035
:10DAA000C7F8002814BF00200420E1E7C0AF02201F
:10DAB00010A3022070F613088BF613081FB5D1EDE2
:10DAC000017A0B46FCEEE77A1A7CCDED027AD1EDB5
:10DAD000007A017CFCEEE77A01920B48CDED037AE7
:10DAE000D3ED027AFCEEE77A17EE902A92B200921A
:10DAF0009DF80C2093ED030A9DF808300BF04CF9CB
:10DB000005B05DF804FB00BFE8BD022007B5D1ED0C
:10DB1000007A0848FCEEE77ACDED017A9DF8041012
:10DB20000DF058F800280CBF0420002003B05DF869
:10DB300004FB00BFE8BD022073B58B8B05460C4685
:10DB4000C02B54D8B12B10D8162B00F0B28031D88E
:10DB5000112B00F0FC80142B00F0FC80214628469D
:10DB600002B0BDE870407FF0E3BCB23B0E2BF5D8AD
:10DB700001A151F823F000BF9DDC01085DDB010825
:10DB80005DDB01085DDB01085DDB01085DDB010891
:10DB90005DDB01085DDB010887DC01085DDB010856
:10DBA000C9DC010805DD01085DDB0108BDDC0108F9
:10DBB0007BDC0108202BD1D1D1ED007AF5EEC07AC3
:10DBC000F1EE10FA40F3C9809FED657AF4EEC77A62
:10DBD000F1EE10FA00F2C180FCEEE77A614ACDED79
:10DBE000017A9DF80430A2F8723E002024E0B3F5DB
:10DBF000967F00F0928021D8D42B39D008D8D02B32
:10DC000052D0D12BAAD102B0BDE87040FFF756BF69
:10DC1000DF2BA3D1D1ED037A94ED021AFCEEE77A63
:10DC2000D4ED010A94ED000A4F4817EE901A8BF0DC
:10DC300019FC0028D9D1042002B070BD4AF2FA764E
:10DC4000B3420CD84AF2F776B34222D840F6B8363F
:10DC5000B34283D102B0BDE87040FFF757BF4AF22C
:10DC6000FD7083427FF47AAF404803F04DFDBCE77E
:10DC700002B0BDE87040FFF7D1BE214602B0BDE85A
:10DC80007040FFF779BC214602B0BDE87040FFF755
:10DC9000FDBC02B0BDE87040FFF72ABD214602B0CE
:10DCA000BDE87040FFF752BE02B0BDE87040FFF71C
:10DCB000CDBE02B0BDE87040FFF796BE94ED000AFD
:10DCC0002A48FCF7EDFEB4E7294C94F86533002BA5
:10DCD000B1D0284904F6642041F076FD0028AAD08E
:10DCE0000123022204F17801A4F5E04084F89D3A72
:10DCF00013F0EEFE00287FF478AF1D4B002283F86E
:10DD00009D2A98E71A4C94F86533002B93D0194953
:10DD100004F6642041F034FDE0E7D1ED007A9FED98
:10DD2000167AF0EEE77AF4EEC77AF1EE10FA14D52F
:10DD3000D1ED017AF0EEE77AF4EEC77AF1EE10FA5F
:10DD40000BD502220D49094813F0C2FE4DE702220D
:10DD50000B49F8E702220B49F5E702206CE700BF08
:10DD600000007F43107302209C6E022010330220BB
:10DD700010A3022064BC02200000003488A302200B
:10DD8000D0A30220B4A30220F0B5414C8FB00D46C1
:10DD900004F1F803D4F834239A4277D1CE782722BD
:10DDA000002104A8272E28BF27261CF193F905F18E
:10DDB0000C0104A832461CF143F9059B9DF836502E
:10DDC0000093069BED430193EDB2079B8DF836500F
:10DDD00005F087070293089B0393C7F08BFA15F0B1
:10DDE000810F064601D1802F12D168463CF0C6FB58
:10DDF000DFED287AC4F8D86920EE270ADFED267A0D
:10DE000020EE270ABDEEC00A10EE103AC4F8CC3955
:10DE100015F0820F01D1802F12D168463CF0C8FB6B
:10DE2000DFED1C7AC4F8DC6920EE270ADFED1A7AF0
:10DE300020EE270ABDEEC00A10EE103AC4F8D03921
:10DE400015F0840F01D1802F12D168463CF0C0FB41
:10DE5000DFED107AC4F8E06920EE270ADFED0E7AD4
:10DE600020EE270ABDEEC00A10EE103AC4F8D439ED
:10DE70006B060BD5DDED0C7A04F6E4139FED067A04
:10DE8000C4F8E86967EE877AC3ED007A0FB0F0BD99
:10DE900010A30220E02E65420000C84210B590B0E9
:10DEA0001E4C084602A9FEF7B7FC04F1F803D4F8AB
:10DEB00034239A422FD19DF83C30072B2BD104F507
:10DEC00080549FED177ADDED056AD4F8683907EEC6
:10DED000903AF8EEE77AE6EEC77AFDEEE77A17EECB
:10DEE000903AC4F868397DF00FFFD4F84029062134
:10DEF000D4F868395268DFED0B7A9B1A0A4A07EEAC
:10DF0000103AB8EEC77A27EE277AB7EEC77A8DEDCA
:10DF1000007B76F099FB10B010BD00BF10A302206B
:10DF20000000C8420AD7233CA4F613081D4B10B5C5
:10DF300003F1F802D3F83433044696B0934208460E
:10DF40000FD108A9FEF768FC03AA9DF854102046DB
:10DF50007DF076FC38B97DF0D7FE134A042176F0C7
:10DF600073FB16B010BDBDF8503023F004039BB214
:10DF7000002BF6D0DDED0B7A00229FED0C7A04A881
:10DF8000039B114667EE877A0093FDEEE77A17EE62
:10DF9000903A21F035FD236804A92046D3F8E830F3
:10DFA0009847DEE710A30220B8F613080000C84225
:10DFB00030B48D7A04464B7A0A4643EA0523CD7A7B
:10DFC00043EA0543562B1BD008D8522B12D0542BB2
:10DFD00013D02046114630BC7EF02EBB03F1807377
:10DFE000863B23F07F43012BF3D8017C064830BCED
:10DFF0006EF0FCBF30BCFFF7C7BE30BCFFF74EBFB2
:10E0000030BCFFF793BF00BFE0AF02200020704795
:10E01000C8207047012070470020704700207047DB
:10E0200090F8D0308B4286BF00EB8100D0F8D4004E
:10E030000020704790F8D0308B4286BF00EB810003
:10E04000D0F8D4000020704703207047014B93F8AC
:10E05000DE0A70471063022070B504464D4812F086
:10E060002BF818B1636A43F400036362494812F065
:10E0700023F888B1462081F0A9FFDFED477AB4EE9E
:10E08000E70AF1EE10FA07D8A36A43F40003A3628B
:10E09000E36A43F40003E362636A43F4F8436362B0
:10E0A0003E4BD3F8340303685B689847013818285F
:10E0B00015D8DFE800F03D450D4745454545143D81
:10E0C0003D3D3D3D3D14454545453D14473D3D00E5
:10E0D000334A92F80C379BB392F80D279AB3314B21
:10E0E00093F87435012B3FD0022B46D02E4B1D6880
:10E0F000EDB12E4E284696F8121F68F02DF9B0B1FA
:10E10000636A43F480736362A6F5805393F9843B9A
:10E110001BB1A36A43F48073A36296F8121F2846CA
:10E1200068F068F918B1E36A43F48073E36270BD84
:10E13000D4E90A2342F4E04243F4E043A262E362FA
:10E14000012300E00023A16A41F48062A262E26A36
:10E1500042F48060E062002BC1D041F4406142F49F
:10E160004062A162E262BAE7636A43F480036362D9
:10E17000A36A43F48003A362B8E7636A43F48003AD
:10E180006362A36A43F48003A362E36A43F48003F7
:10E19000E362ABE710330220000000B410A30220BA
:10E1A0001083022010B30220D4C202201073022078
:10E1B00013B54FF44470CDE9002122F0EDF8044688
:10E1C00028B1DDE900217EF005FD024B23602046E9
:10E1D00002B010BDBCF81308002070470020704743
:10E1E00000207047002070470020704700207047D3
:10E1F00000207047002070470020704700207047C3
:10E2000000207047002070470020704700207047B2
:10E2100000207047002070470020704700207047A2
:10E220000020704700F56D507047000000487047AF
:10E23000F023140800F5E040D0F8340303685B686D
:10E240001847000000F5E0431846D3F8343378301F
:10E250001B1A584258417047B120704700F5E043FF
:10E26000DFED6B6A2DE9F041D3F8542A03F6582309
:10E2700000F50A4890B007EE902A044608F1D80845
:10E28000B8EEE77AD3ED007A00234046F8EEE77A5D
:10E2900004F5004627EE267A039367EEA67A8DED05
:10E2A000017ACDED027A0DF0D7F9002800F0A880B0
:10E2B000D6F80C3B0CAF08AD84330FCB87E80F00CA
:10E2C00004AF85E80F0087E80F0001A9384603ABCB
:10E2D00002AA3CF097F9D6F89C7D9FED4E0A01A862
:10E2E0003DF0F8FB294638468DED080ACDED090AC8
:10E2F0008DED0A1A18F034FAC6F0FCFFD6F8103C7F
:10E3000004F5AA55C01A083563282DD8D6F80C0B89
:10E3100003689B689847042100F1A002284671F029
:10E3200037FCD6F80C0B0368DB689847052100F131
:10E33000A002284671F02CFCD6F80C0B03681B6970
:10E340009847062100F1A002284671F021FCD6F87A
:10E35000102B2846072102F52D7271F019FC04F5E7
:10E360000D40203015F03EF840460EF097FB90B17E
:10E37000D6F8100BBCF09EF868B1D6F8102B6E21C1
:10E380002846903271F004FCD6F8102B6F212846F5
:10E39000BC3271F0FDFB04F5A74269212846183212
:10E3A00071F0F6FB04F5AA426A21284671F0F0FBF1
:10E3B00004F5A04393F9422542B903F5A763D3EDD1
:10E3C000007AF5EEC07AF1EE10FA05DD04F5AD4203
:10E3D0006B21284671F0DCFB04F5AD442C3420465B
:10E3E000B3F0C2FA28B104F130026D21284671F071
:10E3F000CFFB1AF01FFA19F015FF10B0BDE8F0813D
:10E4000004F5F75001A9183018F072F874E700BF4E
:10E410000AD7233CE02E654210B54FF48011044624
:10E4200013F06EFD10B12046FFF718FF4FF4800186
:10E43000204613F065FD28B137F070FBBDE81040B1
:10E4400034F0E2BF10BD000070B500F5F75590B094
:10E4500000230446183502A9029300230DF1070298
:10E4600028468DF8073019F0B3FF03A9284618F0A5
:10E470006DFE08B92D4B03933022002104A804F54A
:10E48000E0461BF127FEA3238DF8103095238DF86D
:10E490001130C6F037FFD6F8543ACDF813004620B5
:10E4A000ADF81B3004F50053CDF81710D3F8F02069
:10E4B000D3F8F430ADF81D20D6F8582AADF8213045
:10E4C000ADF81F2081F082FD10EE103A1520CDF836
:10E4D000233081F07BFD10EE103A9FED157A28462F
:10E4E000CDF8273004F59F43D3ED417A67EE877A64
:10E4F00017EE903ACDF82B30029BCDF82F309DF8D7
:10E5000007308DF83330039B0D931AF06FF904F543
:10E51000AA50D6F87833302204A908308DED0E0ABF
:10E520000F9371F071FC10B070BD00BF2292CA7FD2
:10E530000000C84210B58AB0044625220021684672
:10E540001BF1C8FDA3238DF8003095238DF8013011
:10E550000A238DF80230C6F0D5FE04F5E043CDF86D
:10E560000710DFED206A03F6EC11CDF8030004F587
:10E57000F34091ED007A03F51F61783027EE267A9B
:10E580000968CDF80F1003F6082117EE102A096864
:10E59000CDF80B20D3F8FC29CDF8171007EE902A00
:10E5A00093F8101AF8EEE77A8DF81B1003F6142191
:10E5B00003F6182367EEA67A1B680968089317EE1E
:10E5C000902A0791CDF8132021F02AFA8DF8240023
:10E5D00004F5AA5025226946083071F015FC0AB0EE
:10E5E00010BD00BF0AD7233C70B58EB0352204465B
:10E5F000002168461BF16EFDA32304F5E04604F5F7
:10E60000A0458DF8003095238DF8013001238DF859
:10E610000230C6F077FE06F67813CDF80300D5F881
:10E620007C091B68CDF80710CDF80B3003681B6917
:10E630009847ADF80F00D5F87C0903689B689847A8
:10E64000ADF811001C4802F0FDFAADF81300D5F842
:10E650007C0903685B699847D5F87C0910EE103A8D
:10E66000CDF8153003689B69984710EE103A04F511
:10E67000AA503522CDF81930D6F870330830CDF8CD
:10E680001D3004F50043D3F86C19CDF82110D3F8F0
:10E690007019CDF82510D3F86819D3F84C3ECDF891
:10E6A00029106946CDF82D30D6F86833CDF83130D1
:10E6B00071F0AAFB0EB070BD1033022030B587B0E8
:10E6C00016220446002168461BF104FDA32304F52D
:10E6D000E0458DF8003095238DF8013002238DF848
:10E6E0000230C6F00FFECDF803002046CDF807102B
:10E6F00006F09EF905F644238DF80B001B68039382
:10E70000134B1B68D86A90F89C308DF81030036862
:10E71000DB69984795F8293A8DF811008DF8123089
:10E7200037F0FCF936F02EF8D5F8403A8DF81300A2
:10E7300004F5AA508DF81430162295F82A3A694645
:10E7400008308DF8153071F05FFB07B030BD00BFA9
:10E750000C33022010B58AB02722044600216846F7
:10E760001BF1B8FCA3238DF8003095238DF8013000
:10E7700009238DF80230C6F0C5FDCDF80300042052
:10E78000CDF8071081F022FC10EE103A1320CDF8DE
:10E790000B3081F01BFC10EE103A4620CDF80F3004
:10E7A00081F014FC10EE103A1520CDF8133081F0F2
:10E7B0000DFC10EE103A0320CDF8173081F016FC56
:10E7C00010EE103A1A20CDF81B3081F0FFFB10EE4E
:10E7D000103A04F5AA5027226946CDF81F3004F5F7
:10E7E000E0430830D3F88433CDF8233071F00CFBCC
:10E7F0000AB010BD13B5044600F5AA5008300190C8
:10E8000070F0B2FD019870F049FE04F58053019854
:10E8100093F978360BB170F06BFF204602B0BDE87B
:10E820001040FFF797BF000038B500F5E04500F550
:10E83000E14304467833D5F834239A421FD1D5F802
:10E840001C3A43B100F59C42082100F5AA501C3245
:10E85000084471F09DF9D5F8FC3901330AD105F669
:10E86000EC15DFED077A95ED007AB4EEE77AF1EE7C
:10E8700010FA04DB2046BDE83840FFF75BBE38BD28
:10E880000000003400F5004330B500F5AA5593F8B8
:10E89000EC2B89B00446083552B11E226946D3F8E4
:10E8A000040BBEF0B9F86A460F49284671F048FCDF
:10E8B00004F5E043D3F8340303685B68984704F534
:10E8C00040530146284693F8B42871F05DFC04F5E6
:10E8D000F75018301AF02AFA04F5907009B0BDE824
:10E8E00030402AF00FBB00BFECF9130800229FED67
:10E8F000020A65F0FBBB00BF0AD7233C324B70B560
:10E90000044640F8043B8AF0FBFC4FF4987504F190
:10E9100078002E4E7FF0AAFB2D4BA36760197FF085
:10E920000FFE66513035B5F5866FF7D104F5866078
:10E9300004F5865582F05AF8264A04F56C6004F511
:10E94000805602F5AA510C35C2F0EAFAFF2322499B
:10E95000284686F8DC3086F8E43065F0BDFF1F4BB2
:10E960001A6812B11E48C6F097FC04F587501D6066
:10E970000C30C3F027FFF1EE043A9FED1A5A04F56C
:10E980008F50F7EE004A9FED180AB0EE454A14305A
:10E99000B0EE633AF0EE632AB2EE042AF0EE451AC6
:10E9A000B0EE451AF0EE450A9EF0DEFD04F59750F4
:10E9B0000830C3F025FC012320460C4986F8893332
:10E9C00065F08AFF204670BDD844022048521408E2
:10E9D0005C521408B06D02209014160828CE022054
:10E9E000F83D14080000000000409C451C4114083C
:10E9F00000F56B510D222DE9F0411C319AB004460F
:10EA00006FF02CFB00222721C14865F0E7FA0421B2
:10EA1000002081F075FF1321012081F071FF462154
:10EA2000022081F06DFF1521032081F069FF81F044
:10EA30007FFC04F5004393F9A43B23B19FEDB50A95
:10EA4000B54866F0DDFA66F039F9B44AB44E4FF0D5
:10EA5000000813880AAF43F004031380002110223A
:10EA600038461BF137FB012305A938468DF83030B5
:10EA70003388ADF8283073680B9365F0B9F9C8B1E5
:10EA80009DF91430002B15DD7FF08CFC9DF81410DF
:10EA9000036801391B68C9B2984758B1051D28465B
:10EAA00065F044F930B9B36806A92846ADF81830C6
:10EAB00066F090FF08F106080C36B8F12A0FCDD1A8
:10EAC00000220DF10B01974806AD64F035FF0646B4
:10EAD00020B365F02BF908BB934B0FCB85E80F00F3
:10EAE00004A9284665F084F9002840F048814FF0D9
:10EAF00004088E4B0FCB87E80F0005A9384665F058
:10EB000077F928B105A865F011F908B148F00108B6
:10EB100003A930468DF80C8066F00AFF844B0FCBBA
:10EB200085E80F0003A9284665F062F9002847D060
:10EB3000002204A9099864F0FFFE064600283FD091
:10EB400065F0F4F8054600283AD19DF80C303946B6
:10EB5000013BDBB2032B94BF764A0346304698BF95
:10EB6000D35C8DF8283066F0E3FE002205A97248D8
:10EB700064F0E2FE064694F09DF978B194F098F9BD
:10EB800090F8302090F8281090F84830114490F810
:10EB900040200A44D34214BF0125002586B13046E7
:10EBA0009DF90C8065F0C2F850B91DB1B8F10005AF
:10EBB00018BF0125394630468DF8285066F0B8FE5A
:10EBC00004F56D50B7EE000A00220121383065F0DF
:10EBD0008DFA04F56C50B7EE000A002202211430C1
:10EBE00065F084FA012304F54751544A00938E20BE
:10EBF0000023043165F0F6F994F94CCBBCF1000F19
:10EC00001AD14F4E3D460FCE0FC50FCE0FC50FCEBA
:10EC10000FC596E80F0085E80F00624604213846CC
:10EC200065F0DCF99FED470A474866F0E9F9B7EE71
:10EC3000000A464866F0E4F9012504F55B5100231B
:10EC4000434A343140F20510009565F0CBF904F5E4
:10EC50006D5002210830FFF749FE04F56A50032188
:10EC60003030FFF743FE04F56A5003213830FFF7D8
:10EC70003DFE04F56D5003210430FFF737FE04F527
:10EC80006D5002210C30FFF731FE04F56B5002216C
:10EC90000430FFF72BFE04F56B5002210830FFF71C
:10ECA00025FE022104F56B50FFF720FE04F5054018
:10ECB0007830C0F033FC27490B68D80711D404F52D
:10ECC0004452254B0D601C321A6004F54C52303210
:10ECD000DA6004F5605208329A6104F5B2521C32CF
:10ECE0005A6204F56E5004221B490125083065F074
:10ECF000CBF904F5AA510023184A0831FD200095EC
:10ED000065F070F9164B1A68D20731D42AE000BFBB
:10ED1000583E14080000964358651508A8C2022002
:10ED2000C84014081C3E1408ACE21308BCE21308E7
:10ED3000CCE21308543E1408273E1408208514081A
:10ED4000DCE2130800000000343E1408433E1408BF
:10ED5000D40F160804330220C4250220CC4915081C
:10ED60000833022004F5F054094A1D601C34146075
:10ED70000121074865F0A4F91AB0BDE8F08104A8A4
:10ED800064F0D4FF00283FF4B2AE4FF00C08B0E6B8
:10ED9000F4250220704700000020704700207047D3
:10EDA0000020704700207047002070477047000027
:10EDB000002070470020704784B001A804B080E8AC
:10EDC0000E000020704700000020704700207047B0
:10EDD000704700001020704700487047204E14080C
:10EDE00000487047304E14080020704770470000FC
:10EDF00001207047012070470020704700234360C6
:10EE00008360C360036143610023037670470000A1
:10EE100010B50446FFF7F2FF0023637610BD000033
:10EE2000027E531C00EB8202DBB2042B037682EDE0
:10EE3000010A84BF002303767047000010B5044622
:10EE4000FFF7EEFF9FED117AD4ED017A94ED020AFF
:10EE500077EE877A637E042B77EE807A94ED030A4F
:10EE600094BF0133052377EE807A94ED040A63762C
:10EE7000637E77EE807A94ED050A77EE807A00EE75
:10EE8000103AB8EEC00A87EE800A10BD00000000FC
:10EE900010B5044621F088FA204610BD05F0BEBA30
:10EEA00004F0CABB04F096BD03F060BD02F088B95F
:10EEB00001F00ABD01F0AEBE01F0F4BEFCF7CEBA1F
:10EEC000FBF780BD6B4B70B5044640F8043B8AF0FD
:10EED0007BFF002504F1100004F569561DF004FDC8
:10EEE00004F168006DF016F804F5907029F03AFA14
:10EEF00004F5AA601BF0C8FF04F2EC6021F0AAFA46
:10EF000004F6382034F0B0FB04F58E500436083097
:10EF100089F0A4FF04F59450183067F043F904F524
:10EF2000AA50083070F0A4FE04F5B2501C3092F0E4
:10EF3000CBFD04F5B350183082F056FF04F5B55000
:10EF400014301FF0DFFE04F5BB501030A2F076FC49
:10EF500004F5F050AEF0B4FE04F5F0501C306DF046
:10EF600099FB04F5F35010308CF010F904F5805340
:10EF700004F5F550404A83F8945E04F5F4530430E8
:10EF8000143313605FF008FF04F5F750294618307A
:10EF900017F0B4FD04F5175018308FF02DF904F573
:10EFA000185008309FF004FF04F53A501430A7F0D1
:10EFB000CFFC04F53E502C30A6F0CCFA04F53F50BF
:10EFC0001430A9F0E1FE04F541502030ADF0D2FF3D
:10EFD00004F543500430AEF007FC04F544501C30F7
:10EFE0009EF004FE04F54750043016F091FB04F542
:10EFF0004C503030A0F0D0FB04F54E500830AFF04C
:10F00000F7FF04F55B501D491C3065F065FC04F505
:10F010005B50343093F024FA04F55E503030AFF09A
:10F02000BBFE04F560500830C6F084F904F5405387
:10F0300083F8B45804F56355043528460C3574F04C
:10F04000C3FCAE42F9D104F569500D4D1030AFF05C
:10F0500023FF04F56950343073F0B2FF2B6813B10D
:10F060000848C6F019F92046074965F035FC2046E6
:10F070002C6070BD7042150880CD02205C16160809
:10F080000CC30220384E1408E84015082DE9F04F53
:10F0900004464FF000092DED028B9FB004F580452A
:10F0A000FFF710FFE14B04F56E5004F56A5823603A
:10F0B00004F5F757083004F5A046FFF71FFC04F5E8
:10F0C0009E4008F120081837183005F57E65B1F02C
:10F0D000B5FC04F56C5304F59E4004F59F4A2633B5
:10F0E00004F5AE4B78300AF1600A45F8A03C0623DF
:10F0F0000BF1440B05F89C3C82F00AFA04F5054339
:10F100002F6104F5A3407833C5F814803C30AB611F
:10F110000E934FF40063EB615A2386F87C304FF076
:10F120007E53C5F85C31C24BC5F86031C14BC5F8A0
:10F130006431C14BC5F86831C5F8CC3104F5A3453D
:10F1400074F042FC04F5A3407835483074F03CFC80
:10F15000BA4B0AF5FC7086F8F091C6F8D831FFF783
:10F160004DFEB74BB7495046C6F8D83186F8F191F5
:10F1700065F0B2FBB44B04F5A440C6F800A2C6E9A2
:10F180007E3700235030C6F82C32C6F834320123C3
:10F1900086F83C3220F014FCAC49284686F8609290
:10F1A00065F09AFB04F5A44041466430B2F00AF8D9
:10F1B00004F5A74041464830B1F05AFC04F5AA4096
:10F1C00041462C30B2F0DCFB2C22494606F2DC60D2
:10F1D0001AF180FF04F5AD4004F5AE499C492C308E
:10F1E00065F07AFB09F114099A4B09F10C00C6F895
:10F1F0001437C5F0B9F804F5AF43643358460F939C
:10F200000BF1140B79F094FE0F9B5B45F6D11E2396
:10F2100040F2CC60C6F814390023A6F8183921F062
:10F22000C1F8C6F8100904F5B2401C30C5F09CF8CE
:10F2300004F5B2406030C5F097F8874B1A680AB9F8
:10F24000C3F80090854B4FF48051C6F87C5904F503
:10F25000B340C6F8143704F5C0451DF047FC04F56B
:10F26000B44062F071F804F5B440B7EE008A04F5DA
:10F27000E24940304FF0FF3B66F062FC04F5B440D9
:10F2800009F11809543095F0ADFF04F5DE406C30FB
:10F2900006F02CF8724B04F5DF40C5F86C3F0830DF
:10F2A00006F024F86F4B04F5DF40C5F8883F2430A2
:10F2B00006F01CF86C4B04F5DF40C5F8A43F403065
:10F2C00006F014F8694B002204F5DF40C5F8C03F92
:10F2D00005F6E8737C30DA609A605A6083ED008A44
:10F2E00006F004F8624B04F5E040C5F8FC3F04F575
:10F2F000E045183005F0FAFF5E4B2846AB6134302C
:10F3000005F0F4FF5C4B28466B635C3005F0EEFFC4
:10F310005A4B2846EB65783005F0E8FF584B04F56A
:10F32000E140AB67243005F0E1FF564B04F5E140C6
:10F33000C5F8A430403005F0D9FF534B04F5E14047
:10F34000C5F8C0305C3005F0D1FF504B04F5E1400A
:10F35000C5F8DC30783005F0C9FF4D4B4846C5F89C
:10F36000F83005F0C3FF4B4B04F5E240C5F8183107
:10F37000343005F0BBFF484B04F5E240C5F83431AA
:10F38000503005F0B3FF454B04F5E240C5F850316D
:10F390006C3005F0ABFF424B04F5E340C5F86C312F
:10F3A000083005F0A3FF3F4B04F5E340C5F8883172
:10F3B000283005F09BFF3C4B04F5E340C5F8A8312D
:10F3C000443005F093FF394B04F5E340C5F8C431F0
:10F3D000643005F08BFF364B04F5E440C5F8E431AA
:10F3E00005F084FF334B04F5E440C5F800321C30CF
:10F3F00009F024FA04F5E440583005F077FF2E4B6D
:10F4000004F5E4402D49C5F858322D4B7430C5F849
:10F4100074324FF4C053A5F8C83265F05DFAFE238C
:10F4200004F5E7404FF400714CE000BFE0331408EE
:10F43000000080BF0000B4420000B4C2A44E140813
:10F44000B44E1408FC761608707416081874160862
:10F45000246D1608B466150880C70220B4F9130895
:10F460001C5B1408186214083865140894581408B2
:10F470002C5C1408B45C1408945B1408185A140823
:10F4800094591408A8611408A45D14089C5A14081F
:10F49000345D1408EC4E1408245E1408306114081E
:10F4A000245F140814601408945F1408AC601408F6
:10F4B000A45E140824581408B464140810A4160890
:10F4C000DC4E140885F8403305232246C5F86CB39A
:10F4D00085F864330830B54B85EDE18A1193B44B60
:10F4E0001094C5E9CD9900934FF00009AF4B1CF083
:10F4F000CFFB05F51663AF4A04F5F340C5F850B9E4
:10F50000DA6005F6CC13AC4A7830C5F8CC99C5F86A
:10F51000D099C5F8D499C5F8D899C5F8DC99C5F83B
:10F52000E0991A620F9320F04BFAA44A04F5F540D3
:10F530000F9BC5F80C9A283085F810BA04F5F449E9
:10F540009A640323C5F8403A05F65C2383ED008AEC
:10F550009B4BC5F8804AC5F8843A9A4BC5F8884A4F
:10F56000C5F88C3A984BC5F8904AC5F8943A20F003
:10F5700027FA04F5F540443020F022FA04F5F5406E
:10F58000603020F01DFA914B09F1FC00A5F8F8BAA3
:10F5900009F16409C5F8F43A20F012FA8C4B484698
:10F5A0008C49C5F8ACBCC3F8009065F095F94FF6EE
:10F5B000FF7304F5F94088493030A5F8A03A874B2D
:10F5C000A5F8BCBA186065F087F904F5F940503029
:10F5D0006EF038F9824B1EA9D6F87C29129404F5F6
:10F5E0000746CDE913347F4B3036CDE915347E4BD9
:10F5F000CDE917347D4BCDE919347D4BCDE91B3472
:10F600007C4B1D930CAB11E9030083E803000AABAC
:10F61000DDE91A0183E8030008ABDDE9180183E89E
:10F62000030006ABDDE9160183E8030004ABDDE966
:10F63000140183E80300DDE9120102AB83E8030053
:10F64000534649460E9804F50849CDE900283A4644
:10F6500009F1B809BFF0B0FC30469DF095F904F50A
:10F660000840314604F500466030B2F09BFF624B23
:10F6700009F13C00C6F860380B2386F8B4385F4BBC
:10F68000C6F8B83820F09CF95D49484665F024F981
:10F690005C4BD3F80080B8F1000F02D05A48C5F097
:10F6A000FBFDC3F8009004F50940584B04F50A49E6
:10F6B000443086F8BC88C6F8B83807F51B7386F85E
:10F6C000C18809F16409C6F8403986F8E58820F058
:10F6D00077F904F50940543020F072F904F5094037
:10F6E000643020F06DF91C22414606F674101AF1C0
:10F6F000F1FC04F50940E03082F0DAFC4846AFF056
:10F70000A1FC434B48464349C6F8643A65F0E4F827
:10F7100004F50A4340484FF0140C404AC8331060C7
:10F720001FFA88F108F101080CFB0102127C002A83
:10F73000F6D13B4A11803B4A11803B4AD2F8008007
:10F74000B8F1000F01D03948A9E704F50A40136069
:10F75000CC30AFF061FC364B04F50A403946C6F8B0
:10F76000CC3AD8300AF04CFC324B04F50D4032490B
:10F77000C6F8E03D6423E03086F8E43D2F4BC6F840
:10F78000183E2F4BC6F81C3E65F0A6F82D4B2046C0
:10F79000C6F8408EC6F8E03D012386F8488E85F80D
:10F7A00090391FB0BDEC028BBDE8F08F9DEE0108D3
:10F7B00068F613080000B442000080BF000080C05B
:10F7C000A1EE0108A5EE0108A9EE01080000FFFF67
:10F7D000E0C1022088F91408808B150888CD02202A
:10F7E000ADEE0108B1EE0108B5EE0108B9EE010871
:10F7F000BDEE0108C1EE0108985314088C4E1408A0
:10F8000004711608C4D502204C4E1408A8521408DE
:10F8100080ED130858ED13081C431408C8C20220D9
:10F82000C6C202209CC2022070C20220684E140888
:10F83000C4ED1308C44E14084C7515085081140803
:10F84000A88114082883140838B5037904463BB905
:10F8500005682DB1284632F06FFE284620F0A4FD41
:10F86000204638BD2D4B70B50360044600F5595055
:10F870003C3020F083F804F5405393F8B82042B9A7
:10F88000D3F8B4502DB1284632F056FE284620F069
:10F890008BFD04F5F05004F59255AEF025FA04F511
:10F8A000CC5004F58F560C350430FFF7CDFF04F52E
:10F8B000CB500C361C30FFF7C7FF04F5CB5014308B
:10F8C000FFF7C2FF04F5B350183082F0A5FAB54235
:10F8D00004D0183D284632F089FAF8E7104B04F6B8
:10F8E000046504F6D456C4F8383AAE4204D0083D54
:10F8F0002846FFF7A9FFF8E704F6983073F02CFDCF
:10F9000004F66C3073F028FD04F6CC2073F024FD6F
:10F9100004F52A6073F020FD204670BD7042150882
:10F920002CE8140838B5104B0446036000F500437A
:10F9300093F8542842B9D3F850582DB1284632F0E4
:10F94000FBFD284620F030FD04F5A043074AD3F81C
:10F950001009C3F8142708B120F02AFD2046FFF74C
:10F9600081FF204638BD00BFE0331408B466150897
:10F9700010B5C5F00BF8064C064B18602046FFF793
:10F9800085FB2046044A0549BDE8104016F126BC17
:10F99000103302200C330220902D032025F901089A
:10F9A0000069C0F3401070470F299DBF302303FB4F
:10F9B0000100B83000207047014B93F9250B7047C8
:10F9C00010630220014BD3F82C0F704710730220F4
:10F9D00008B503689B68984730B9044B93F84E0309
:10F9E000B0FA80F0400908BD0020FCE710A3022017
:10F9F00008B5044810F0CAF810B9034B93F848034F
:10FA000008BD00BF1033022010A30220022A10B547
:10FA10000C4605D135220A48BDE8104012F02CB939
:10FA2000084BD3F8340303685B689847A04205D1BC
:10FA30007EF0B8FCBDE810407EF02EBC10BD00BFCB
:10FA40001033022010A30220012910B50C4610D05B
:10FA5000022904D061B97CF057F9084A02E07CF031
:10FA600053F9074A062174F0EFFD064BC3F8704BBB
:10FA700010BD7CF049F9044AF4E700BF04501408B3
:10FA8000DC4F140810B30220F34F1408012910B5FD
:10FA90000C4614D0022907D0D1B90E4BC3F8401E32
:10FAA0007CF032F90C4A05E00A4BC3F8401E7CF0AA
:10FAB0002BF90A4A0621BDE8104074F0C5BD7CF060
:10FAC00023F9074A062174F0BFFD024BC3F8404EEC
:10FAD00010BD00BF10B30220435014081850140882
:10FAE0002C501408012903D0022914BF002102213F
:10FAF000014BC3F8341C704710730220012902D057
:10FB0000022900D011B9024BC3F8441E704700BF50
:10FB100010B302206C2910B400F3A6803F290FDC3B
:10FB2000162900F39980032940F39A8001247E4B23
:10FB30008C402340002B00F093805DF8044B70470D
:10FB4000A1F140032C2B00F28B8001A454F823F088
:10FB500009FD010861FC010861FC010861FC010864
:10FB600061FC010861FC010861FC010861FC0108FD
:10FB70003BFB010861FC010861FC010861FC010814
:10FB800061FC01083BFB010861FC010861FC010804
:10FB900061FC010861FC0108FFFC010861FC01082F
:10FBA000FFFC010861FC0108FFFC0108FFFC0108E3
:10FBB000FFFC01083BFB010861FC0108FFFC010898
:10FBC0003BFB010861FC010861FC01083BFB0108EB
:10FBD0003BFB010861FC01083BFB010861FC0108DB
:10FBE00061FC010861FC010861FC010861FC01087D
:10FBF00061FC010861FC010861FC01083BFB010894
:10FC00003BFB0108112B2BD801A454F823F000BFB3
:10FC10003BFB010861FC010861FC010861FC010873
:10FC20003BFB010861FC010861FC010861FC010863
:10FC300061FC010861FC010861FC010861FC01082C
:10FC40003BFB01083BFB010861FC010861FC01086A
:10FC50003BFB01083BFB0108A1F12703112BD1D984
:10FC60005DF8044B7FF010BCA0291FDC9529F7DD5F
:10FC7000A1F196030A2BF3D801A454F823F000BF96
:10FC80003BFB010861FC010861FC010861FC010803
:10FC90003BFB01083BFB010861FC01083BFB010841
:10FCA00061FC010861FC0108FFFC0108B52921DCA9
:10FCB000A929D5DDA1F1AA030B2BD1D801A454F8B1
:10FCC00023F000BF3BFB010861FC010861FC010857
:10FCD0003BFB010861FC010861FC01083BFB0108DA
:10FCE00061FC010861FC01083BFB010861FC0108A3
:10FCF0003BFB0108A1F1D003022BB1D81DE7002383
:10FD00005DF8044B7FF088BB084B012283F83C2E42
:10FD1000A3F58043D3F8280F00283FF40EAF6421E9
:10FD20005DF8044B7EF01CBC1000410010B30220B3
:10FD30006C2938B50346154600F3A2803F2912DC32
:10FD400038290ADC26296FDC102900F005811629E4
:10FD500000F08A81042900F016812A461846BDE881
:10FD600038407FF067B8A1F140022C2AF5D801A0F5
:10FD700050F822F031FF01085BFD01085BFD01082E
:10FD80005BFD01085BFD01085BFD01085BFD0108EF
:10FD90005BFD010861FF01085BFD01085BFD0108D7
:10FDA0005BFD01085BFD01088BFF01085BFD01089D
:10FDB0005BFD01085BFD01085BFD0108D3FF010845
:10FDC0005BFD0108270002085BFD0108DDFF01085B
:10FDD0001D000208C9FF01085F0002085BFD010861
:10FDE0004700020891FF01085BFD01085BFD010867
:10FDF0001FFF0108770002085BFD01086FFF010883
:10FE00005BFD01085BFD01085BFD01085BFD01086E
:10FE10005BFD01085BFD01085BFD01085BFD01085E
:10FE2000FF00020897FF0108A1F12702112A94D8C8
:10FE300001A050F822F000BF1FFF01085BFD010880
:10FE40005BFD01085BFD010823FF01085BFD010864
:10FE50005BFD01085BFD01085BFD01085BFD01081E
:10FE60005BFD01085BFD010881FF010869FF0108D6
:10FE70005BFD01085BFD01087BFF010875FF0108C0
:10FE8000A02921DC95297FF768AFA1F196020A2A03
:10FE90003FF663AF01A050F822F000BF81000208D6
:10FEA0005BFD01085BFD01085BFD0108870002089E
:10FEB000D90002085BFD0108E70002085BFD0108AC
:10FEC0005BFD0108A7000208B52923DCA9297FF7FB
:10FED00044AFA1F1AA020B2A3FF63FAF01A050F8B0
:10FEE00022F000BF9DFF01085BFD01085BFD0108DA
:10FEF000C70002085BFD01085BFD0108A3FF0108C4
:10FF00005BFD01085BFD01081FFF01085BFD0108A7
:10FF10001F010208A1F1D002022A3FF61EAF012400
:10FF20008FE0A91E864B4D424D4183F84153F6E7C1
:10FF3000AA1E844C5542554184F83B5E7BF0E4FE9A
:10FF4000814A94F83B1E814B002908BF1346804A22
:10FF5000062174F079FBE2E70A21FFF757FDDEE79F
:10FF60002A4601211846F8E72A460421FAE72A46DC
:10FF70000321F7E72A460C21F4E72A460F21F1E78F
:10FF80002A460021EEE70B21E7E72A460D21E9E7A3
:10FF90002A460521E6E72A461521E3E72A461121EC
:10FFA000E0E7AB1E5A425A41664B93F8D01B914290
:10FFB000B5D083F8D02B7BF0A7FE664A664B022DA6
:10FFC00008BF1346654AC3E729461846FFF78AFD6E
:10FFD000A5E729461846FFF737FDA0E7594CD5B1EC
:10FFE000022D0DD1012384F8383EA4F58053D3F8B7
:10FFF000340303685B6A984710B1594801F06CF804
:020000040802F0
:100000007BF082FE534A94F8381E534B002908BFF8
:100010001346544A9CE784F8385EE6E729461846BA
:10002000FFF734FD7BE7012445B1022D09D1454B93
:10003000C3F8284B002283F8182C02E0414BC3F888
:10004000285B204638BD01242DB1022DF9D1464B45
:1000500083F81843F5E7444B83F81853F1E7294632
:100060001846FFF74BFD5AE7022A7FF458AF3C4889
:1000700009F0DEFD53E77EF095F97EF00DF94EE7CD
:100080002A4607216EE7184629467EF043FD374889
:10009000AFF03AF8044600283FF441AF294B012263
:1000A000C3F8282BC6E7274BD3F8E83B002B3FF4D7
:1000B00036AF012425B1022DC3D183F82C40C0E70F
:1000C00083F82C50BDE7022D7FF429AF9FED280A5D
:1000D0002348FAF7E5FC22E7022D7FF420AF204801
:1000E0000FF060FC1BE701242DB1022DA9D1154BA7
:1000F00083F83A4EA5E7134B83F83A5EA1E7022D49
:1001000012D10F4DD5F834030368DB6B98470446D2
:1001100078B10121A5F5E04003F09CFE91E7294666
:100120001448C3F0C7FAFAE600210D4803F092FE26
:10013000F5E67BF0E9FD104A042174F085FAEEE65D
:1001400010A3022010B302203BAA1608D7361408C9
:1001500058501408618315083B831508685014082B
:1001600010330220745014081063022074BD022062
:100170000000000084A502208750140810B599B132
:1001800011680468416004B90160126801681B6865
:10019000521A9A4202D80021084610BD017A012362
:1001A00081F001010372F7E7037A3BB144682CB197
:1001B0001368029A1B1B12689342ECD90023C0E912
:1001C0000033EFE700238385037780F82830C0E908
:1001D0000533C0E908337047F0B504469F480E4622
:1001E0002DED028B87B0B0EE408AAEF097FF40B1A4
:1001F000236933B1206B00F5127012F067F80546E1
:1002000038B12046FFF7DEFF002007B0BDEC028BBF
:10021000F0BD236B93F94C22002A1EDD93F8B03217
:10022000DBB18F4BD3F8442E002AEAD12369D4EDF9
:10023000007A991EF5EEC07A48424841F1EE10FA74
:1002400084F82C0025D884F82D2084F828202277E3
:10025000C4E90822C4E90522D7E7824FD7F834035E
:1002600003689B6B984718B197F8383A002BD8D0A1
:1002700000217D480FF026FFDFED7C7AB4EEE70A1F
:10028000F1EE10FACDDA784804F0D2FB0028C8D19C
:10029000B7E76EB1F4EEC87AF1EE10FA3BDD236BEE
:1002A000D3F8D432DB0403D5714816F001FF0646BB
:1002B00084F82D60C5F01EF8D4ED027A9FED6D7ABA
:1002C000039067EE877AFCEEE77A17EE903ACDED71
:1002D000047A5B000593B4F90630002B1DDC002383
:1002E000C4E9083384F8283094F90430002B3CDC4E
:1002F0000023C4E90533237794F82C00002884D127
:1003000094F82D00002880D194F8280000287FF46C
:100310007CAF207F79E71646CAE70421524801F0F6
:1003200083FAB4F9063003AA04F1200007EE903AEC
:1003300005ABB0EE408AF8EEE77A009304ABF4EE3A
:10034000C07AF1EE10FACCBF01210021FFF716FFB1
:100350000028C9D07BF0D8FCB7EEC88A464A0421F1
:100360008DED008B74F070F9BEE7444E9FED447A3A
:10037000D6F8F02006F5D650B0EE476ADFED416AB8
:10038000D0ED007A82EAE27006F58051A0EBE270CF
:10039000A7EEA66A07EE900AF8EEE77AF4EEC67AC0
:1003A000F1EE10FA55D801F6C420D6ED3D7A90ED65
:1003B000006AF8EEE77AA6EE267AF4EEC77AF1EE56
:1003C00010FA46D501F6C8219FED2F7A91ED006A0B
:1003D000A6EE267AF4EEC77AF1EE10FACCBF01272A
:1003E0000027642113FB01F11E4BD3F8540A121AA3
:1003F000002AB8BF52428A422DDAD6F8F420D3F848
:10040000583AD31A002BB8BF5B428B42ACBF0023D3
:10041000012304F114000FB983F0010505AB03AA11
:100420002946009304ABFFF7A9FE00283FF464AF10
:100430007BF06AFCD6F8F4206423D6F8F01092FB27
:10044000F3F291FBF3F300920421104A74F0FCF8EC
:1004500052E70027C5E70023DBE700BF74BD022099
:1004600010B3022010A30220103302200000003439
:100470000852022000007A447852140810530220D7
:100480000000FA430000C8420000FAC38952140871
:1004900073B582890446036BD20766D493F94C2264
:1004A000002A03DD93F8B022002A5ED1544D05F5F1
:1004B000F272D5F83413914257D0A5F5A045B3F99F
:1004C00008606846D5ED3C7AB8EEE77AD5ED3D7A1E
:1004D000F8EEE77A8DED007ACDED017A3BF0B8F8D1
:1004E0007300B0EEC00A07EE903AF8EEE77AF4EE49
:1004F000C07AF1EE10FA40D4236B93F801232AB3AB
:1005000007EE906AF8EEE77AF4EEC07AF1EE10FAB0
:100510001CDB002183F80113236B586BB8F06EFECF
:10052000236B9FED387ADA6BD2ED067A67EE877A25
:1005300095EDBF7AF4EEC77AF1EE10FA06D5986B16
:10054000BBF0A2F9236B986BBAF02EFFA389226B44
:1005500013F0020302D192F8011399B9002382F833
:100560000233236B93F8010305E0002083F80103B5
:10057000236B83F8020302B070BD236B012283F862
:100580000123B9E7D5ED856AB0EEE67A9FED185BF9
:10059000B7EEC77AB4EEC57BF1EE10FADFDD95ED6C
:1005A000836AB0EEC67A9FED145BB7EEC77AB4EEFD
:1005B000C57BF1EE10FAD2DD95ED847AB0EEC77A04
:1005C000B7EEC77AB4EEC57BF1EE10FAC7DD66EE82
:1005D000866AF5EEC06AF1EE10FAC0D5D5F8F430AF
:1005E00009498B42ACBF00230123B8E7AFF3008079
:1005F000000000481857C63F0000003652C1E03FD7
:1006000010A302200AD7233C6CEEFFFF08B5036B52
:1006100093F802233AB1DA6A92F8A020022A03D0B2
:10062000002283F8022308BD0B4B15209FED0B0A17
:10063000D3ED857AF5EEC07ADFED097AF1EE10FAA6
:1006400030FE270A7FF0AEFC9FED060A1320BDE8BE
:1006500008407FF0A7BC00BF1053022000A08CC54B
:1006600000A08C450000000010B5084CD4F83403FD
:1006700003689B6B984738B9D4F8340304F59A742F
:10068000001B18BF012010BD0220FCE710A30220B0
:1006900005220249024811F01BBA00BF88A30220BC
:1006A0001033022010B50221032080F055F80221FA
:1006B000084680F051F80121042080F04DF8022115
:1006C000152080F049F81320022180F045F81D48DC
:1006D0000FF0F2FC50B30021462080F03DF80021DD
:1006E000492080F039F800214A20174C80F034F876
:1006F0000021012080F030F80021084680F02CF81D
:1007000094F8EC3BE3B1D4F8040B0368DB6A984738
:100710000E4B0146D4F8042B1B68B2F82821586A06
:1007200003689C6C2346BDE8104018470121462011
:1007300080F012F80121492080F00EF80121D3E762
:1007400010BD00BF1033022010B302200C33022072
:1007500038B5394C90F90A3094F8EC2BA4F50044E4
:1007600042B12B2B06D120460A223449BDE838403D
:1007700011F0AEB90125324A2B2B15700FD131483B
:10078000BEF0C2FE304810F0E5FE30480BF0F0FA43
:10079000012209212E48BDE83840F9F795BCD4ED77
:1007A000460A64219FED2B0A03207FF0EDFCD4ED77
:1007B000460A64219FED270A02207FF0E5FC9FEDA9
:1007C000260A03207FF0EEFB9FED230A02207FF034
:1007D000E9FB9FED220A04207FF0E4FB9FED1F0A56
:1007E00015207FF0DFFB13209FED1C0A7FF0DAFB62
:1007F00015480FF061FCA0B1002146207FF0DAFF20
:10080000002149207FF0D6FF00214A207FF0D2FF4F
:10081000002101207FF0CEFF002108467FF0CAFFB3
:10082000B0E7294646207FF0C5FF294649207FF0E2
:10083000C1FF2946E9E700BF10B30220B8A4022097
:1008400000C8022088B8022010330220E8BD022030
:1008500074BD0220000000000000C84200A08C45CA
:1008600000F5E040D0F8340303681B6C1847000023
:1008700000F56D5300F5004093ED017A0433B5EEB9
:10088000C07AF1EE10FA5DBFD0F84039DFED076AAB
:10089000D3ED017AD0F858095FBFF8EEE77AE7EEBA
:1008A000267AFDEEE77A17EE900A70470000C842FC
:1008B00000F5405090F8840B28B141F00101084246
:1008C00014BF01200020704710B54B6800F50044AC
:1008D0005168D4F874098B42D6BF0A461A461946A5
:1008E00036F01CF8C4F8740910BD000010B50446B9
:1008F000544891F00FFF10F008025FD0524B0122D4
:1009000013ED027AD3ED007A77EE877A9FED4F7A76
:1009100067EE877A10F0010353D04D4BD3ED036A95
:1009200093ED007A012337EE667ADFED486A27EE11
:10093000267A04F56D51D1ED036AF5EEC06AF1EE49
:1009400010FA41DD434A9FED416AD2ED006A01226F
:1009500066EE866AF4EE676AF1EE10FA58BFF0EEC2
:10096000667A04F5004090F87C1991B393B1D0F801
:10097000803906EE903AF8EEE66AF4EEC76AF1EED8
:1009800010FA58BFF0EE476AFDEEE66A16EE903AAE
:10099000C0F88039E2B1D0F8803907EE103AB8EEED
:1009A000C77AB4EEE77AF1EE10FA37FE277ABDEE99
:1009B000C77A17EE103AC0F8803909E0DFED267AE1
:1009C000A8E79FED257AB4E7002ACAD1002BC8D149
:1009D00010BDCBB1D0F84039D3ED016AD0F87439ED
:1009E000F8EEE66A76EE876A07EE103AB8EEC77A56
:1009F000F4EEC76AF1EE10FA37FE267ABDEEC77A3A
:100A000017EE103AC0F87439002AE1D0D0F8403916
:100A100093ED017AD0F87439B8EEC77A77EE277A79
:100A200007EE103AB8EEC77AF4EEC77AF1EE10FA94
:100A300058BFB0EE677ABDEEC77A17EE103AC0F82D
:100A40007439C5E7046A0220186A02200000C8420F
:100A50000C6A02205C6E02200000000000F50040DD
:100A60000023C0F8783970477FB51646002300226E
:100A700004463046CDE9022302AA1FF08FF848B1A0
:100A80009DED027B9FED2A6B27EE067BFDEEC77B7B
:100A900017EE900A04F50045C5F8780933785B072E
:100AA0001CD595F87C39CBB104F5F940012201A998
:100AB00050306DF04DF888B1D5F88039DDED016A20
:100AC00007EE903A9FED1C7AF8EEE77AE6EEC77AE9
:100AD000FDEEE77A17EE903AC5F8783904F5E04371
:100AE000D3F8403A042B1FD004F54054B4F97E2BC0
:100AF000002A16DDD5F878399FED107A83EAE37184
:100B0000A1EBE37107EE901AF8EEE77A67EE877AC9
:100B100007EE102AB8EEC77AF4EEC77AF1EE10FAB3
:100B200002D50023C5F8783904B070BDAFF300805A
:100B300000000000000059400000C8420AD7233CD2
:100B400037B50B7804460D465A071DD500F5F94018
:100B5000012201A950306CF0FBFFA8B1D5ED017A5C
:100B60002B78F8EEE77ADFED1B6ADB0767EEA67AF3
:100B70001BD59DED017AB4EEE77AF1EE10FACCBF09
:100B80000120002003B030BD2B7804F50044D5EDE2
:100B9000017A13F0010FF8EEE77A11D104F6581339
:100BA00093ED007AB8EEC77AE5E704F50044D4F88F
:100BB000403993ED017AB8EEC77AE7EE667AD8E766
:100BC000D4F8403993ED017AB8EEC77A77EE877A98
:100BD000E4E700BF0AD7233C00F54053B3F92E3BAE
:100BE00000EE103A00F5E0431A46D3F83413B8EE9D
:100BF000C00A783291420CD1D3F8402A042A02D09C
:100C000093F891392BB100F50540D0ED1E7A30EE06
:100C1000270A704710B50446FFF7DEFF9FED087AFC
:100C200004F5004404F65813D3ED007AF8EEE77AA1
:100C3000E0EE477AFDEEE77A17EE900A10BD00BFAE
:100C40000000C84237B500F50045044695F87C39E8
:100C5000FBB100F5F940012201A950306CF078FF9A
:100C6000B8B105F5186205F684139FED0D7AD2ED43
:100C7000007AD3ED006AF8EEE77AE6EE877ADDEDEA
:100C8000016AE6EEC77AFDEEE77A17EE900A03B046
:100C900030BD2046FFF7BEFFD5F87439181AF6E7C5
:100CA0000000C84210B50446FFF796FF04F509405E
:100CB000D0ED247A37EEC00ADFED047A20EE270A61
:100CC000FDEEC07A17EE900A10BD00BF0000C842CA
:100CD0002DE9F04100F5094700F509450446543770
:100CE000643504F5E04804F50946294638461FF006
:100CF0000FFAB7EEC00B08F6781344362A4638468A
:100D0000314683ED000A1FF009F908F67C13B7EEAF
:100D1000001ADFED210A762083ED000A35F034FD5C
:100D200004F59F43204683ED890AF9F74BFED8F876
:100D3000340303685B6898470B280DD008D80A284D
:100D400011D004F500440023C4F87839BDE8F081DF
:100D50000E38C0B20128F4D829462046FFF7F0FE2D
:100D60000028EED011E029462046FFF7E9FE30B911
:100D70004FF480410948FAF721FA0028E1D12046D2
:100D8000FFF790FFB0F5FA6FE6DD2A4631462046C0
:100D9000BDE8F041FFF768BE0000000010330220FC
:100DA00000F5004310B52DED028BD3F8682982B011
:100DB00093F86439044607EE902ADFED1A8ADA07C1
:100DC000B8EEE78A5CBF00F50052D2ED5A7A28EE01
:100DD000288A5CBFF8EEE77AA7EEE88A5B070FD5B2
:100DE00000F5F940012201A950306CF0B1FE38B194
:100DF0009DED010A30EE480A02B0BDEC028B10BD39
:100E0000204604F50054FFF705FF07EE900A94ED25
:100E10005A0AF8EEE77AB8EEC00A28EEC00AA7EE42
:100E2000A80AE7E70AD7233C70B500F5E046044678
:100E300033462DED028B1833D6F834239A424CD129
:100E400000F50053D3F8F85000F54053B3F97C3B5C
:100E5000002B65DD04F50B52F7EE007A92ED0F7A68
:100E6000B4EEE77AF1EE10FA5AD404F5A042F6EEA9
:100E7000006AD2ED027A67EEA67A87EE871AB5EE9F
:100E8000C01AF1EE10FA4BD907EE905A9FED278A5F
:100E900004F5F94004F50044B8EEE70A07EE903A8D
:100EA0005030F8EEE70A20EE080A6CF061FFD4F843
:100EB00078394FF429709FED1E1A002BDFED1D0AC3
:100EC000BEBF07EE903AF8EEE77AA7EE880ABDECCF
:100ED000028BBDE8704035F057BC08F019FDF8B939
:100EE00004F5A04306F67816D3F87C0903681B695D
:100EF000984704F540530546DFED0E0AB3F97C3BF5
:100F000040F27F2096ED000A01EE103AB8EEC11AC9
:100F100035F03AFCBDEEC00A10EE103A1BB297E76E
:100F2000BDEC028B9FED030A70BD00BF0AD7233CC6
:100F300000007A440000000010B50446C4F0DAF95D
:100F400004F58043D3F85C2F801A41F28832904236
:100F50000FD802212046FFF7ABFC50B104F5E04466
:100F6000D4F8402A042A04D103F5756393ED000AEE
:100F700010BD9FED010AFBE70000000030B500F551
:100F8000004504462DED028B95F87C3983B0DFEDEA
:100F9000278A7BB3D5F8803900F5F9409FED240A04
:100FA000012207EE903A01A95030F8EEE77A27EED9
:100FB000800A6CF005FEE8B1204605F68415FFF7BF
:100FC00033FFDDED017A85ED000A204637EE800A19
:100FD0008DED010AFFF7B0FFDDED017A30EE270A53
:100FE00020EE280ABDEEC00A10EE100A03B0BDECD8
:100FF000028B30BDD5F840292046D5F874395268A7
:101000009B1A08EE103AFFF7E7FD2046B8EEC88AB3
:10101000A0EE288AFFF790FFBDEEC88AB8EEC88A16
:10102000A0EE288ABDEEC80ADEE700BF0000C84275
:101030000AD7233C00F5E04310B50446D3F8340347
:1010400003685B6A984718B104F5004494F8380EB9
:1010500010BD000038B500F500440D46D4F87439D1
:101060000B44C4F8743994F87C393BB1FFF7E2FFC4
:1010700020B9D4F880192944C4F8801938BD00007B
:1010800000F5405030B5D0F8782BD3070FD40B20A3
:10109000084B1D785C688D4204D1224214BF0120A8
:1010A000002030BD013803F10803F2D1F9E7012037
:1010B000F7E700BFF852140800F5E04310B5044606
:1010C000D3F8340303685B68984701462046BDE8BF
:1010D0001040FFF7D5BF000037B500F500440546C6
:1010E000D4F85839C4F874390023C4F87839FFF7B4
:1010F000E3FFE0B105F5F940012201A950306CF0A1
:1011000027FDA0B12846FFF795FF80B9DDED017AF4
:1011100001239FED097A84F87C3967EE877AFDEE2A
:10112000E77A17EE903AC4F8803903B030BD002357
:1011300084F87C39F9E700BF0000C84238B504469E
:101140000D46FFF7B9FF30B1032128461EF002FD1E
:1011500080F00103D8B204F5004484F87D0938BD5D
:1011600073B500F500444A680D460646C4F8742974
:101170000B78D90741BFD4F840395B689B18C4F895
:10118000743994F87D3923B100F509416431FFF7D2
:10119000D5FF2B785B070FD506F5F940012201A991
:1011A00050306CF0D5FC38B1012384F87C396B6881
:1011B000C4F8803902B070BD002384F87C39F9E7A7
:1011C000F0B504460E462DED028B83B004F50045C4
:1011D00004F56E578DED010AFFF7C2FFB7EE001A56
:1011E00040F24310DFED330A9DED010A35F0CCFAF1
:1011F000D5F878392046B0EE408A5B4207EE903A47
:10120000F8EEE77A67EE807AFDEEE77A17EE901A4D
:10121000FFF720FFD7ED007AF5EEC07AF1EE10FA75
:1012200043DDD5F87839002B3FDD2046FFF70AFD76
:1012300007EE900ADFED206AB8EEE77AD7ED007A84
:1012400067EEA67AB4EEE77AF1EE10FA2DD53146C4
:101250002046FFF785FF04F5094132462046543108
:10126000FFF702FCD5F8783920465B4207EE903A4A
:10127000F8EEE77A67EE887AFDEEE77A17EE901AD5
:10128000FFF7E8FEB5EEC08AF1EE10FA0DDDD5F8F5
:10129000783907EE903AB8EEE77AC7EE087AFDEEB5
:1012A000E77A17EE903AC5F8783903B0BDEC028BB7
:1012B000F0BD00BF000000000000C8C2F0B500F59E
:1012C000004487B0074694F8643903F00503052B02
:1012D0000BD06DF0FDFE4FF4AE724FF480116DF047
:1012E000AFFE0025284607B0F0BD6A4603211D4821
:1012F0001EF040FC0028F4D001AA03211A481EF079
:1013000039FC05460028ECD0184BB7EE001A40F225
:101310006D10DFED170A93ED000A02AE35F034FAD6
:1013200004F66413B0EE401ADFED111AB7EE002A8E
:10133000DDED010A9DED000A0FCB86E80F0035F0C8
:1013400039F9DFED0C7A3046032220EE270AFDEE54
:10135000C07A17EE901A1EF039FB31463846FFF777
:10136000FFFEBFE754BC022074BC02208CAC0220FC
:10137000000000000000C842F7B50E4602210446F6
:10138000FFF796FA70B304F5E045D5F8403A042B20
:1013900028D12046FFF790FE20B304F5F94704F565
:1013A000094101236A465037543138466CF0BAFA85
:1013B000C0B104F50941012301AA384664316CF03B
:1013C000B1FA78B19DED017A05F69C15DDED007A54
:1013D00077EEC77A96ED007A37EE277A86ED007AB7
:1013E000C5ED007A03B0F0BDF0B500F5945600F5F8
:1013F0008044054618362DED048B89B094F8121FF1
:101400003046039164F09EFF07460399304664F02E
:10141000ABFF042FB0EE408A039921D1002305A829
:101420008DED050A069307933AF0A2FC05F50850E6
:1014300005A9183036F04AFCDFEDAB7A8DED050AD0
:10144000B4EEE71ACDED060A8DED071AF1EE10FAAB
:1014500006DB05F5005393F8747117F001070CD102
:10146000002294F8483F62F3000384F8602F84F868
:10147000483F09B0BDEC048BF0BD94F8483F05F53A
:101480009E4128469A0701F164015FBF43F00203C1
:1014900084F8483F04F64C7383ED008A04F66473C5
:1014A00083ED001AFFF768FF94F8603F092B00F204
:1014B000898004F66873B0EE480A9FED8C9AD3EDEC
:1014C000000A34F0FBFF00BB04F64C7394F8121FC3
:1014D0003046D3ED008A64F071FF07EE900A9FED6D
:1014E000847A78EEC88AF8EEE77AF0EEE88A67EE5A
:1014F000877A67EE897AF4EEE78AF1EE10FAC2BFD6
:1015000094F8603F013384F8603F04F6687394F800
:10151000121F3046D3ED008A64F050FF07EE900AA8
:101520009FED747A78EEC88AF8EEE77AF0EEE88AF2
:1015300067EE897A67EE877AF4EEE78AF1EE10FAC1
:1015400002DD002384F8603F04F6687383ED008AAF
:1015500094F8483FDA078CD5284605F50046FFF792
:101560001FFC04F6647393ED008A96F87C3930EE24
:10157000488A002B6ED005F5F940012205A95030AC
:101580006CF0E6FA00286BD1C3F0B4FED4F85C2FFF
:1015900041F288310346821A8A4204F5756204F6E4
:1015A000547166D982ED008A284681ED008A0221B5
:1015B000FFF77EF918B106F5AF66F268B260C4F8BD
:1015C0005C3F56E794F8483F43F0010384F8483FF6
:1015D00005F5E043D3F8406AD3F8342305F5E34337
:1015E000301F2833464246419A4212D005F5E34364
:1015F00044339A420DD005F5E04378339A4209D13D
:101600003D4B05F50A40B3F8A21AD8300AF04AFC5F
:1016100000B13E4694F8483F590795D4002E93D028
:1016200002212846FFF744F900288DD043F0040337
:1016300005F5AE40314A062184F8483F04F664734C
:10164000143093ED007AB7EEC77A8DED007B72F01F
:10165000FBFF79E72846FFF72FFD00288BD193E7A2
:1016600004F664739DED058A93ED000A38EE408A16
:101670008AE79FED200A92ED007A28EE008ADFEDDE
:10168000207AA7EE278A82ED008AC4F85C0FD1ED9C
:10169000007A38EE678AF3EE0E7AB0EEC88AB4EEBE
:1016A000E78AF1EE10FA7FF7E4AE94F8483F5B0763
:1016B0000ED504F6647405F5AE40124A062194ED89
:1016C000007A1430B7EEC77A8DED007B72F0BCFF64
:1016D00005F59E4024220021483009B0BDEC048B62
:1016E000BDE8F04018F1F6BC000000340AD7233CF6
:1016F000CDCC4C3DCDCC4C3E10A30220B8521408AA
:10170000CDCC4C3FD552140838B50B4D0C460A6869
:1017100005F66C731A60C3F0EDFD9FED087AC5F80D
:10172000700FD4ED027A67EE877AFCEEE77A17EE57
:10173000903AC5F8743F38BD1073022000007A4417
:1017400038B50C4C0D46D4F8700F88B1C3F0D2FDFB
:10175000D4F8703FC01AD4F8743F984297BF04F68B
:101760006C740020012023688CBFC4F8700F2B60BC
:1017700038BD00BF1073022073B50D46694604469C
:101780001646FFF7DDFF18B19DED000A02B070BDEF
:1017900029462046FFF78CF878B966BB04F50A4560
:1017A000D83528460AF0B0FFB8B328460AF05EFBE9
:1017B00098BB2046FFF7F4FAE8E704F5804595F872
:1017C000483FDB0704D505F6647595ED000ADDE7B3
:1017D00004F50A40D8300AF0B9FF0028DDD004F53E
:1017E000945095F8121F183064F0ACFD0228D4D143
:1017F0009FED0C0ACAE704F5004393F87435022BF9
:10180000CCD104F5F940012201A950306CF0A0F9C7
:101810000028C3D09DED010AB8E704F5094494ED12
:10182000240AB3E70000000000F5004393F87C2988
:10183000FFF7A2BF73B50D4601A90446FFF780FF6D
:10184000064648B1002304F5F3449DED010AE36127
:1018500001232B7002B070BD2046FFF7A1FA20468D
:101860002E708DED010AFFF767FBDDED017A022195
:10187000204637EEC00A8DED010AFFF719F828B1AE
:1018800004F5804494F8480F00F001002870E1E767
:1018900070B50B7805460C46164603F00503042B7D
:1018A00015D105F500456DF013FCB2B24FF480116F
:1018B0006DF0C6FBD5F84029636852689B1A13F592
:1018C000FA7FC8BF6360237843F00103237070BDC3
:1018D000F8B500F5005300F5E0470446D3F8686119
:1018E000D7F8A059B54219D00E4A1268D26A92F8B8
:1018F0009C209AB100F50941751B25226431FFF740
:10190000C7FF07EE905A04F59F40B8EEE70ADFEDF7
:10191000067A603020EE270AB3F07EFDC7F8A06992
:10192000F8BD00BF0C3302200AD7233C70B51C4D14
:1019300006460C4695F849338BB3002385F84933A6
:10194000A5F580457AF0E0F92346164A062172F0A3
:101950007BFE95F8B4380E2B21D1032C19D8DFE883
:1019600004F01E020A1196F854100F220E48BDE82A
:10197000704010F081B90F220C490B48BDE870404F
:1019800010F0A6B896F854300A2B02D10F2208495D
:10199000F3E708490448BDE8704000F0C5B970BDE0
:1019A00010A302205053140810330220B4A30220C5
:1019B00088A3022064BC022010B5044600F507404D
:1019C00030309BF039FB04F50840BDE81040603032
:1019D000B1F07CB938B50A4C04F1DC0549B1D4F852
:1019E0003433AB4205D00E222946A4F5E04010F076
:1019F0006FF8D4F83403431B5842584138BD00BF38
:101A000010A3022070B50E4611461D46FFF7E2FFF7
:101A1000044658B1114B3269D3F858198A4207DA93
:101A2000002201F57A7128461DF0D0FF204670BDD6
:101A30000B4A9FED0C7AD2ED007A67EE877A07EEBB
:101A4000101AB8EEC77AB4EEE77AF1EE10FA03DDB9
:101A50000022A1F57A71E6E70024E7E710B302203F
:101A6000546E02200000C8422DE9FF41884611460D
:101A700007461E46FFF7AEFF044658B1002501AAEF
:101A800041463846019502950395B1F02BFA04467C
:101A900020B90024204604B0BDE8F081DDED017AD4
:101AA0009FED147AF0EEE77A0395F4EEC77AF1EE43
:101AB00010FA08D5DDED027AF0EEE77AF4EEC77A97
:101AC000F1EE10FAE5D401A83AF086FC01A83AF04C
:101AD00069F89FED090A01A83AF050F89DED021A45
:101AE0009DED010A3046B7EEC11AB7EEC00A1EF0EE
:101AF00083FBCFE70000003400401C462DE9F04393
:101B0000484F85B00646884697F849331446EBB9E6
:101B1000D7F83403012587F8495303685B68984771
:101B200086F85400D7F834233F4B9A420CD0BC3B84
:101B30009A4202D197F8903933B1D7F8403A042B42
:101B400002D03A4B9A4256D1002450E00025E9E7F2
:101B5000002D4CD00E22364936480FF0B9FF7AF0EE
:101B6000D3F82346344A012172F06EFD3FE0002D88
:101B70003DD0324808F088FE0E2208B13049EBE72C
:101B80003049E9E7304B6F460FCB87E80F003B4603
:101B90002A4641463046FFF735FF10BB044624E095
:101BA000294B6F460FCB87E80F003B462A4641463C
:101BB0003046FFF759FFF0E7234B6F460FCB87E81E
:101BC0000F003B462A4641463046FFF71BFF814641
:101BD0003B462A4641463046FFF746FFB9F1000F23
:101BE000DBD03946134800F09FF8002DB7D12046CE
:101BF00005B0BDE8F08303F5A6739A42A4D0062C85
:101C0000F3D801A353F824F0EF1B0208EB1B0208E2
:101C1000851B0208A11B0208B91B0208511B020800
:101C20006F1B020810A3022044A402206CA3022010
:101C3000B4A302201033022070531408E8BD022020
:101C400098A40220D0A3022074BC022000F5E04C2E
:101C5000F8B500F500449CF893E905460F4604F6F4
:101C60004416BEF1000F53D004F664130FCB86E880
:101C70000F0001238CF8943904F6641697E80F00DE
:101C800086E80F0005F50946D4F86C39643693B937
:101C9000D4F870397BB9D4F85C39D4F86829C4F821
:101CA0006C39D4F86039C4F8703922B9D4F85819AD
:101CB00030461DF08BFE314628222846FFF7E8FD0E
:101CC00094F8641911F0040102D130461DF042FF6E
:101CD00005F5094105F509403246443154301EF0FE
:101CE00053F938B104F6441604F6541494E80F007E
:101CF00086E80F00284607F057F92846FEF7E8FF68
:101D0000284607F0C5FD2846BDE8F840FEF7A8BD07
:101D100004F654130FCB86E80F0001238CF894E9E6
:101D20008CF89339A8E70000F8B500F54053044655
:101D30000D46B3F9D63A002B36DB0B7813F0020FC1
:101D400014BF4FF0FF33012304F5004686F81C3919
:101D500006F6541306F644170FCB87E80F0006F675
:101D6000641795E80F0087E80F0004F50941572232
:101D7000204600256431FFF78BFD2046FFF7ACF9C4
:101D80002046FEF7A5FF204607F082FD04F5E0435C
:101D9000204683F89459C6F8205983F8995907F0DA
:101DA00003F986F81A5CF8BD4FF0FF33CCE700006A
:101DB000364B1B682DE9F043054685B0D86AF7F726
:101DC0004BFE002860D105F5804393F9483C5A1C2E
:101DD00053D0002B05F5AA6711DD95F861254C213C
:101DE00007EE903A01FB0272F8EEE77A92ED0B7A79
:101DF000B0EEC77AB4EEE77AF1EE10FA3DDC05F505
:101E0000005305F5F75693F87431183613F00104B2
:101E100029D0C3F340089B0732D495F814144FF02F
:101E2000B00995F8A94409FB015191F8F1314CBB77
:101E3000022B18D968461DF0C3FD6946304616F0DE
:101E400011FA044678B195F814344246684609FB05
:101E50000353D3F800121DF0B9FD16F0EBFC6946F0
:101E600016F0C8F80446384619F0F4F8304615F074
:101E7000CFFF2846F9F774F9204605B0BDE8F08396
:101E80000024F0E74446EEE70020F6E70C3302209A
:101E900038B50C4B05460C461B68D86AF7F7DCFDD5
:101EA00010B10024204638BD16F0C4FC214616F0BF
:101EB000A1F804460028F4D005F5F44064303AF067
:101EC00019FEEFE70C330220F0B500F5E04300F512
:101ED0000046002287B0044606F6441583F893298D
:101EE00000EE101A83F8942906F65413B8EEC00ACF
:101EF00006F664170FCB85E80F0002AD04F5094222
:101F000016492846543263F03BFF95E80F0087E8F6
:101F10000F0004F5094140F2571220466431019147
:101F2000FFF7B6FC01992046FFF708F90199204612
:101F3000FFF716F904F540532046B3F9D63A002BC3
:101F4000B4BF4FF0FF33012386F81C39FEF7C0FE03
:101F5000204607B0BDE8F04007F09ABC508D022043
:101F600010B50446024963F00BFF204610BD00BFC8
:101F7000508D0220F8B500F5004504460E4605F6E2
:101F8000541305F644170FCB87E80F0006F108013C
:101F90002046FFF75BFEB28804F5E04302EB8202C5
:101FA00002EB8202920012B2002AD8BF4FF4C8722C
:101FB000A3F88E29D5F84029D5F868195068091A70
:101FC0004C20C3F8601991680A31C5F86C190021DA
:101FD000D2680A32C5F870290022C3F8742983F840
:101FE000902983F8A429C3F8642903F6581203F64C
:101FF000881311604FF0FF3243F8382C04F5AA62C1
:1020000094F8611500FB0122D26A1A60F8BD000045
:1020100070B50E4608310446FFF718FEB38804F584
:10202000E04543B3642213FB02F3C5F86039B5F908
:102030008E3904F59E4024220021002B00F1480037
:10204000DCBF4FF47A73A5F88E3918F143F804F524
:10205000094304F50540314693ED240A7830BDF07C
:102060001BF9D5F8403A072B0CD120460421BDE8D6
:102070007040F8F757BCD5F86039002BD7DC40F634
:10208000B833D2E770BD000030B5083185B00446E2
:102090006D460FC985E80F0004F509412846543103
:1020A0001DF004FE2046294604F5E044FFF7CEFD6E
:1020B0000123C4F85C3305B030BD00000B7A00F595
:1020C000004013F0020F14BF4FF0FF33012380F8DC
:1020D0001C3970477FB501F1080305466C460E4672
:1020E0000FCB84E80F0005F50941204654311DF05F
:1020F000DDFD21462846FFF7A9FD31462846FFF7BA
:10210000DDFF04B070BD00007FB501F10803044697
:102110000E466D460FCB85E80F0004F509412846B1
:1021200054311DF0C3FD29462046FFF78FFD2046A0
:10213000314604F50044FFF7C1FF337907EE903ACA
:10214000337E9B07F8EE677A44BF9FED097A67EE0E
:10215000877A9FED087A67EE877AFCEEE77A17EECA
:10216000903AC4F814390123C4F8343904B070BD6E
:102170000000803B00A00C477FB501F10803044636
:102180000E466D460FCB85E80F0004F50941284641
:1021900054311DF08BFD29462046FFF757FD2046A0
:1021A00031464FF47A72FFF789FFB38804F5004493
:1021B0005343C4F82C390123C4F8343904B070BD3A
:1021C0002DE9F34100F50945044600F509400E46A6
:1021D000643504F5E047443029461DF023FDD0B9AD
:1021E0004FF0FF33C7F8503906F1080738461DF0A5
:1021F00017FC032802463AD1F16828461DF0E6FB99
:1022000004F50043B2882046C3F8342902B0BDE883
:10221000F041FEF723BC27F041FFF8F7B1F80128A1
:1022200014D94FF0FF33C7F8503927F037FFB022E9
:1022300090F8F43202FB030090ED3C0AB7EEC00ABE
:1022400028469FED111B1EF011F8CDE704F500584C
:10225000D8F8F80034F066FAC7F8500998ED3E0A4D
:10226000DFED0B7AB8EEC00A20EE270AE6E701AAF6
:10227000002138461DF0E0FB0028C1D00022019962
:10228000BBE700BFAFF300800000000000408F40BC
:102290000AD7233C7FB501F1080304466D460E467C
:1022A0000FCB85E80F0004F50941284654311DF095
:1022B000FDFC29462046FFF7C9FC2046314604F5BF
:1022C0000044FFF7FBFE0023C4F8343904B070BDAE
:1022D00037B504460D46C3F00DF82062D5ED027AFD
:1022E000F5EEC07AF1EE10FA15DD9FED127A67EE89
:1022F000877AFCEEE77AC4ED077A79F005FDE269AA
:102300004FF47A730621B2FBF3F30B4A03B0BDE836
:10231000304072F099B990F00DF8002395F90D2036
:10232000009395F90C1095F90E308FF057FFE0618E
:10233000E3E700BF00007A44A0531408F0B5044658
:102340002DED028B85B004F5E04616F073FA15F01A
:102350000BF904F5005393F8F0330BB900287CD047
:10236000D6F85039013378D1D6F87439002B50D0D3
:10237000C2F0C0FFD6F87439C01AB0F5FA6F6CD34A
:1023800094F81434B02506F658179FED628A05FBC1
:10239000034393ED847A9FED5D0BB7EEC77A27EE8A
:1023A000000B34F0D9F997ED007AB7EEC77A30EE2A
:1023B000470BB7EEC00BB7EEC00A34F0CDF9B7EE5D
:1023C000C00BDFED557A20EE080A20EE270A34F024
:1023D0005DF9FDEEC07A04F5AE40062117EE903AA5
:1023E0001430C6F8503997ED007A27EE087AB7EE28
:1023F000C77A8DED027B94F8142405FB024292ED1E
:10240000837A464AB7EEC77A8DED007B72F01CF9ED
:1024100023E004F59070F7F7B3FF02281DD994F874
:102420001434B022F1EE047A02FB034393ED837A75
:10243000B4EEE77AF1EE10FA0FDD394B1B68D86A7B
:102440000368DB699847012803D0C2F053FFC6F840
:102450007409D6F87439002B8AD104F5A043D6F854
:102460005019D3F87C094A1C036844D01B6B984769
:102470002C4811F00FFC20B104F5F44064303CF01E
:10248000EFF82046FEF70EFCD6F860390546834289
:1024900034DA07EE905A04F5AE40234A0621B8EE2E
:1024A000E77ADFED227A143004F50044012527EEA7
:1024B000277A04F64417B7EEC77A8DED007B72F0E9
:1024C000C3F84FF0FF3386F89059C6F8503904F638
:1024D000541304F664140FCB87E80F0084E80F0050
:1024E000134890F0E1F80023284686F8933905B0A8
:1024F000BDEC028BF0BD5B6B9847B9E7094811F062
:10250000A9FB0028C5D1F2E7AFF30080000000A0CE
:1025100046DF913FE02E65420000C842B0531408E8
:102520000C33022010330220D45314080AD7233C62
:10253000046A0220F8B500F5094600F5094504468D
:102540004436643504F5A047294630461DF06AFB41
:1025500050B304F5E043D3F850194B1C24D0D7F8FE
:102560007C0903681B6B984704F50045D5F834399E
:10257000012B49D0D5F83439022B06D12046FEF77D
:1025800049FBD5F86839984245DD2046FEF742FB05
:10259000D5F86839C01A0028B8BF4042B0F5FA7FB4
:1025A000CCBF0020012037E004F509402946543013
:1025B0001DF0AEFD9FED197BB4EEC70BF1EE10FAE6
:1025C00018D5304629461DF03DFCB6EE007B284666
:1025D0009FED146B9FED151BA0EE067BBDEEC70BA8
:1025E0009FED147AB8EEC00A20EE070AB7EEC00AD3
:1025F0001DF03CFED7F87C092A469FED0F0A3146B4
:1026000003689B6A9847AFE72046FEF703FBD5F8BF
:1026100068399842AEDB0120F8BD00BF0000000021
:1026200000006940000000009461B6400000000016
:1026300000C072400AD7233C0000000073B5384C3C
:102640000546D1ED026A0E46D4F858399FED357A29
:1026500007EE903AF8EEE77AD7EE876AF5EEC06AB1
:10266000F1EE10FA08DD79F04FFB2F4A062171F0E8
:10267000EBFF012002B070BDD1ED037AA4F5D26466
:10268000F5EEC07A94ED006AF1EE10FA11DDF4EE89
:10269000C67AF1EE10FA0CD579F036FB94ED007A9B
:1026A000224A0621B7EEC77A8DED007B71F0CCFF90
:1026B000DFE7DFED1F7A337CB4EEE76AF1EE10FA64
:1026C00054BFB0EE677AB0EE467A0BB90020D1E77E
:1026D000B5EEC06AF1EE10FA0CDC86EE876A03EB09
:1026E000830307EE903AF8EEE77AF4EEC67AF1EE5D
:1026F00010FAEBD595F82440002CE7D1C2F0FAFD92
:10270000AB6A4FF47A72C01A337C53439842DDD9D6
:10271000012385F82430C2F0EDFDA8622046A9E728
:1027200010B302200AD7233CF053140801541408B4
:102730000AD723BC38B50546AEF07AF9ACF0EEFC0A
:10274000044640B9C2F0D6FD2B6AC01AEB69984224
:1027500084BFEC610124204638BD000038B5044632
:102760000D46C2F0C7FD9FED087A04F50043C3F89B
:102770003809D5ED027A67EE877AFDEEE77A17EE33
:10278000902AC3F8342938BD00007A4410B50446B5
:10279000C2F0B0FD04F50043D3F83829801AD3F80D
:1027A000342990424FF0000084BFC3F8340901205F
:1027B00010BD000000F5004300F5F2410020D3F801
:1027C000342991ED1E7A22EAE27207EE902AF8EEA1
:1027D000E77AB4EEE77AF1EE10FA44BFC3F83409B1
:1027E0000120704700F5405300F5004010B5B3F9E3
:1027F000D63A00F6641400F65410002BB4BF4FF024
:10280000FF33012300F8383C0FC884E80F0010BDE7
:1028100038B504462DED028BF0EE408AB0EE608AAA
:1028200009B301295CD0B5EEC08AF1EE10FA67DD7C
:10283000DFED347AB4EEE78AF1EE10FA60D8FCEE00
:10284000C87A04F5AE40304A0621143004F54054ED
:1028500017EE903A71F0F8FEFDEEC87A17EE903A56
:1028600084F8A33A3AE0F8EE000A33F027FE40B1CC
:1028700004F5E0444FF0FF33C4F86C33BDEC028B39
:1028800038BD04F54053B3F9AC2A07EE902AF8EEB0
:10289000E77AF4EEE87AF1EE10FAC4D8B3F9AE3A7A
:1028A00007EE903AF8EEE77AF4EEE87AF1EE10FAF5
:1028B000B9DBDFED147A04F5E04304F5AE40134ACA
:1028C00068EEA77A06211430FDEEE77AC3EDDB7AD5
:1028D000FCEEE87A17EE903A71F0B6FE0120CDE7F3
:1028E000FCEEC07A00F5AE4004F56A54084A0621B1
:1028F000143017EE903A71F0A7FEC4ED0E8AEDE7A2
:102900000020BBE70000C8424754140820541408B4
:1029100034541408D1F80D3000EE903AD1F8093053
:10292000097A00EE103AFFF773BF000070B58B888C
:1029300004460D46012B11D100F590763046F7F78D
:102940001FFD02280AD994F81414B023204603FB73
:102950000161BDE87040DC31FFF79ABA15F06AFFFB
:1029600005F10801BDE8704015F044BB00F5E042F8
:10297000134610B57833D2F8342304469A420ED168
:1029800000F5E141082224310FF0A2F804F5AE4031
:10299000034A06211430BDE8104071F055BE10BD49
:1029A000585414082DE9F04F00F50048DFEDD97AAE
:1029B00000F5E045044608F658330E462DED068B2B
:1029C00093ED008A99B0B0EEC87AB4EEE77ADFED05
:1029D000D27AF1EE10FA41BF00F54053B3F9D63A7E
:1029E00008EE103AB8EEC88AB4EEE78AF0EEC88A6C
:1029F000F1EE10FA94BF4FF0FF37012788F81C79E9
:102A0000D5F85C33052B16D8DFE813F006002C0050
:102A100064008500C100600100F5A044B0EE680AC2
:102A20003A460831D4F87C090368DB6A9847BB480A
:102A300006F06EFF08B9002049E1B94C6422D4F8D1
:102A40004039A4F50040B4F9981B5B6801FB0231E2
:102A5000FFF73AFAA4F5004006F0A6FA0123C5F8FC
:102A60005C33E8E700F5A043B0EE680A3A46083167
:102A7000D3F87C090368DB6A9847D8F81839002B2B
:102A8000B8BF5B42012BD6DD98F81D391BB998F809
:102A90001E39002BCFD004F50053D3ED980A93EDE7
:102AA000990AF1EE600AB1EE400A14F135FCDFED4F
:102AB0009D7A04F5AE409C4A20EE270A0621143088
:102AC00085EDD80AB7EEC00A8DED000B71F0BCFDA4
:102AD0000223C4E700F5094901F1080A09F1540984
:102AE000504649461DF014FBB7EEE89AB1EE047B60
:102AF00030EE490BB0EEC00BB4EEC70BF1EE10FA9E
:102B000000F3EA80D8F818390133022B40F2EE8046
:102B10000323C5F85C3304F5A04306F10808B0EEC2
:102B2000480A3A46D3F87C0941460368DB6A98476D
:102B3000012FD5EDD87A04F5F753DFED7C6A9FEDD0
:102B40007C7A93ED890A07FE267A77EE877A9FEDE5
:102B5000797AA7EEC70AB7EEC00A33F0FDFDB0EEF2
:102B6000C00B9FED687BB4EEC70BF1EE10FA7FF55A
:102B700062AF04F5AE4006216F4A143071F064FD77
:102B8000042341462046C5F85C33FFF75FF804F59F
:102B9000E0489FED6AAA06F1080508AF98EDD80A4B
:102BA0000DF130099FED668A04F50A4A30EE0A0AF3
:102BB0000DF1400B0AF1D80A95E80F00B7EEC00AF4
:102BC00087E80F0089E80F009FED501B38461DF085
:102BD0004DFB98EDD80A4846B7EEC00A9FED4B1B57
:102BE0001DF044FB04F5A0434A463946D3F87C095E
:102BF000B0EE480A04F50949036809F154099B6AD3
:102C0000984798EDD89A39EE0A9A95E80F00B7EEF2
:102C1000C99A8BE80F00504608F00EFC5846B7EEF4
:102C2000C01AB0EE490B1DF021FB5A463946484602
:102C30001DF0AAF998EDD80A14AF834630EE0A0ABF
:102C4000B7EEE81A95E80F00B7EEC00A87E80F0064
:102C500038461DF00BFB394648462A461DF05EF902
:102C600004F5F75005A9F0EE408A18308DED058A7D
:102C70008DED068A8DED078A15F0DEFB002869D000
:102C8000294648461DF01EF903A905A8CDED040A02
:102C90008DED030A38F0F8FCDFED227A20EE270AEA
:102CA00033F0D6FCB0EEC00ABBF1000F3FF4C3AE68
:102CB000F3EE0E7AB4EEE70AF1EE10FA42D50523F0
:102CC00031465046C8F85C3308F082FC012019B048
:102CD000BDEC068BBDE8F08F494650461DF018FA52
:102CE000B4EEC09BF1EE10FA7FF70CAF04F5A044F0
:102CF000B0EE680A3A465146D4F87C090368DB6AAC
:102D0000984798E6000000481857B63F00000000BA
:102D100000408F4000000034000000B41033022057
:102D200010B30220E02E6542805414080000B44223
:102D30000000874335FA8E3CA25414080000344347
:102D400000000000F6EE007AF4EEE78AF1EE10FAE9
:102D5000B5DC70E6BBF1000F3FF46DAEAFE700BF2E
:102D6000F0B5044600F50A408FB00F46D83009F0A0
:102D7000BDF8054648BB09AE30461CF021FE04F5FF
:102D8000E0434FF6FF7204F5F440B3F8A03A643024
:102D9000934208BF002307AA013399B23BF07AFFA0
:102DA000B0B104F500440FB1C4F8185901AD04F6F0
:102DB000641496E80F0085E80F00E3680548009367
:102DC00094E80E0003F010FF054628460FB0F0BD52
:102DD0000125FAE7D0A3022070B50546002106F0D0
:102DE00099FE05F50046D6F820497CB9284606F03C
:102DF0008FFD10B90024204670BDD6F81839012B7C
:102E0000F8DDC2F077FAC6F82009F4E7D6F83419ED
:102E100061B1C2F06FFAD6F82039C01AD6F82C3951
:102E20009842E7D900230121C6F834392846FFF734
:102E300097FF04460028DDD005F5AE40054A06217F
:102E400005F5E045143071F0FFFB002385F8993952
:102E5000D1E700BFC454140838B50A468B8804462D
:102E60000025190A137EDB0744BF01EB81014900ED
:102E700006F050FE04F5E043204683F8995906F029
:102E800047FD10B90025284638BD04F50043D3F8A6
:102E9000341951B1D3F81829D3F814198A42F1DD45
:102EA000012AEFDD0121C3F834592046FFF758FF0E
:102EB00005460028E6D004F5AE40034A062114304A
:102EC00071F0C2FBDFE700BFDC54140838B50546DB
:102ED000898806F01FFE05F50044D4F8343983BB19
:102EE000D4F81839002BB8BF5B42012B02DC002458
:102EF000204638BD94F81D2994F81E3972B9002B6C
:102F0000F5D0D4F8582905F5AE40642306211430D5
:102F100092FBF3F30C4A71F097FB01E0002BF0D128
:102F20000121C4F834192846FFF71AFF0446002887
:102F3000DDD005F5AE40054A0621143071F084FB62
:102F4000D6E70021EFE700BFF45414081255140827
:102F500010B504460B4809F0A1FD48B10A4BDFED5E
:102F60000B7AD3F8143B93ED090A20EE270A10BD23
:102F700004F54054B4F9043B00EE103AB8EEC00A30
:102F8000F5E700BFE8BD022010B302200AD7233CBA
:102F900000F5405310B52DED028BB3F9081B00F579
:102FA000004304460029ACBF01224FF0FF32002944
:102FB00083F81C29B8BF494289B206F0ABFD04F57D
:102FC000F243204693ED1E8AFFF7C2FFB5EEC00A1A
:102FD000F1EE10FAD8BF9FED0E0ABCEEC00AB8EEB3
:102FE000400AB4EEC08AF1EE10FA0AD804F5AE40F9
:102FF000084A0621143071F027FB0120BDEC028B3A
:1030000010BD204606F084FC0028EFD1F6E700BF93
:10301000000000002C5514082DE9F04F4FF0FF334D
:103020000F4600F5E04900F5004A05462DED028BFC
:10303000C9F8503989B00AF66413BC8804AE97F811
:103040000480240A0FCB86E80F0025D005F5094738
:103050003146443738461DF05BF8B0EE408B3146C0
:1030600038461CF0EFFEDFED5B7AB7EEC88BB4EEAE
:10307000E78AF1EE10FA0FDBB7EEC00BDFED567A00
:10308000E3B2304620EE270A01EE103AB8EE411BBB
:10309000B7EEC00A1DF0EAF805F5A04B05F50947A3
:1030A00099F89429DBF87C0954379FED4C0A0368A2
:1030B0009B6A32B305F5094132464431984705F51C
:1030C0004053B3F9063B002B1EDD07EE903A09F69C
:1030D0007812F8EEE77A92ED007AB4EEE77AF1EE44
:1030E00010FA11DD05F509413246384644311CF02D
:1030F0004BFFF8B90024204609B0BDEC028BBDE8B7
:10310000F08F32463946D9E7B8F1000F1CD1002CB8
:103110003ED1DBF87C4928462368D3F82080FFF7AE
:1031200017FF09F66C132046D3ED000AC047B0EE36
:10313000408A0DE0002CDDD10AF654130AF644153E
:103140000FCB85E80F00D6E707EE908AB8EE678AC6
:10315000314638461CF0DCFFB7EEC00BB4EEC08A37
:10316000F1EE10FA17DBB9F8A03A314638460124DF
:1031700003931CF0CDFFBCEEC00B05F5AE40039BE6
:103180000621174A14308DED000A71F05DFAB2E79E
:103190009FED128ADCE705F5094132463846443195
:1031A0001CF0F2FE04460028A4D0B9F8A03A31463B
:1031B000384603931CF0ACFFBCEEC00B05F5AE40E7
:1031C000039B0621074A14308DED000A71F03CFA8A
:1031D00091E700BF00000034E02E654200000000CF
:1031E000445514086255140838B500F5E04401232D
:1031F000054684F8A839B4F8AA3905F50055013315
:10320000A4F8AA39C2F076F8114B04F6AC12C4F84F
:10321000BC0903F5A04103F5AA43C4F8C009462040
:10322000D1F898131B68116004F51B629FED097AB1
:10323000136004F6B413D5ED857A04F6B81467EE7E
:10324000877AC3ED007A7CF0C1FE84ED000A38BDB8
:1032500010330220E02E6542F0B500F5E04700246F
:10326000C34B89B0054687F8994908460E4683F84E
:103270007D4939F00DFB002836D0012387F89039BD
:1032800005F5A043D3F87C090368DB6B984705F587
:10329000004387F8974903A8C3F820491CF090FB26
:1032A000B7F8A01A4FF6FF7305F5F44001AA99424A
:1032B00008BF21466430013189B23BF0EBFCF0B12C
:1032C000BDF80630A3F115025342534187F89139F6
:1032D00050B105F50A40BDF80610D83008F0E2FDFF
:1032E00010B1002387F8913974885E2C78D8522C5D
:1032F00032D8103CA3B20F2B4CD9002491E00346E6
:10330000E4E7C33C112CF8D801A353F824F000BF24
:10331000AD350208FB320208AD350208FB32020867
:10332000FB320208FB320208AD350208FB3202080C
:10333000FB320208FB320208EB350208FB320208BE
:10334000FB320208FB320208FB3202087D3502081C
:10335000FB3202089D350208533C0B2CCDD801A34B
:1033600053F824F01D3502082535020835350208CA
:10337000FB320208FB320208FB320208FB32020871
:10338000FB320208FB320208FB3202082136020837
:10339000353502080F2CB0D801A353F824F000BF34
:1033A000A1340208DB340208E5340208EF340208D5
:1033B00003350208AD34020873340208FB320208F8
:1033C000FB320208FB320208FB320208FB32020821
:1033D000FB320208FB32020813350208F9340208F6
:1033E000D42C21D8C22C8CD8B22C00F0B78010D8A5
:1033F000702C00F0AE80722C7FF47FAFD6ED027A95
:1034000005F50045FDEEE77A17EE903AC5F8343938
:1034100044E0B32C00F0A780BC3C012C8CBF0024FE
:103420000124204609B0F0BD40F6B8339C4200F0BC
:10343000ED804AF2CE639C4200F0ED80DF2C7FF4F9
:103440005CAF73899FED4B1A07EE903A737A317B2C
:1034500000EE903A337AF8EEE77A474800EE103AF9
:10346000F8EE600A27EE811AB8EE400A85F0FAFFFE
:1034700014E005F50A440023D83487F8293A718806
:10348000204607F0B3FF314628B1204609B0BDE819
:10349000F04008F09BB92846FEF76CFD0124C0E718
:1034A00006F108012846FEF7D1FBF7E705F50A44C7
:1034B0001521D834204608F0F5FC48B100233146E8
:1034C000204687F8293A09B0BDE8F04008F080B8F6
:1034D00031462846FEF79CFDE0E731462846FEF7D8
:1034E000F9FDDBE731462846FEF70EFED6E731460A
:1034F0002846FEF741FED1E731462846FEF7CAFED0
:10350000CCE705F5E1412922284624310EF0E0FA06
:10351000C4E731462846FEF753FEBFE7012487F88B
:1035200097497EE7002305F50A403146D83087F8F1
:10353000293AABE705F50A47D837384608F096FC34
:103540003146044618B12846FEF79EFD69E7384625
:10355000B9E731462846FFF701F99FE7314628468B
:10356000FFF7D8F99AE731462846FFF7DFF995E7E4
:1035700010B302200AD7233C9C6E0220B388012B93
:103580008CD803F0010305F5AE40294A062187F8DF
:1035900092391430B38871F057F87FE7B188284624
:1035A000003918BF012100F055FC77E705F5094403
:1035B000F36805F50045E03495F8591A7BB933698D
:1035C0006BB973695BB920467EF0A0FD04287FF4D7
:1035D00065AF95F8591A20467EF0A2FD5EE706F128
:1035E000080220467EF02AFF58E705F5004305F55E
:1035F0000940002296ED041AD6ED020AE03096ED5D
:10360000030A93F8591A7EF0ADFD47E7317A09486D
:1036100007F0E0FA42E731462846FFF7E5FD3DE7CF
:1036200005F5E04031467830FEF752FE36E700BF40
:1036300080551408E8BD022000F5E0421346D2F898
:10364000342378339A4201D1FFF706BE0120704738
:1036500070B54B7A05460E4600F5E044DBB1C1F08B
:1036600049FED4F8BC394FF47A72C01A737A5343C6
:10367000984210D905F5AE40094A0621143070F081
:10368000E3FF0023002284F8A83904F6C4131A606B
:10369000012384F8C83994F8A80980F0010070BDAE
:1036A000905514082DE9F0474B888AB004460D4622
:1036B0001F2B6BD80F2B41D804F5AE40C34A042111
:1036C000143070F0C1FF94E0A3F1BC02182AF3D8C3
:1036D00001A151F822F000BFF3370208F3370208C6
:1036E000B9360208B9360208B9360208B9360208F6
:1036F000B9360208F3370208B9360208F337020870
:10370000B9360208B9360208B9360208F33702089A
:10371000B9360208B9360208B9360208F33702088A
:10372000F3370208F3370208B9360208B93602083F
:10373000F3370208B9360208F3370208A3F1100282
:103740000F2AB9D801A151F822F000BF3D38020874
:103750001F39020829390208353902084B39020895
:103760004938020813380208B9360208B936020887
:10377000B9360208B9360208B9360208B936020865
:10378000B9360208553902083F390208702B00F09B
:10379000048121D8A3F1530291B20B298CD80B2AB2
:1037A0008AD801A151F822F05F3902087139020864
:1037B0007B390208B9360208B9360208B936020860
:1037C000B9360208B9360208B9360208B936020815
:1037D000B93902087B390208D42B0CD8BB2B3FF631
:1037E00073AF722B00F0DE80A3F1B202012A3FF624
:1037F00063AF012057E04AF2CE62934200F0D780D7
:103800003FF65AAFDF2BF4D040F6B8329342F0D0F7
:1038100052E700F50A461621D836304607F0E6FD95
:1038200030B1294630460AB0BDE8F04708F0C0B8CC
:1038300020460AB0BDE8F047FEF780BD29460AB031
:10384000BDE8F047FFF7E8BB00F50A451521D8357C
:10385000284608F027FB28B128460AB0BDE8F04703
:103860000BF014BE04F5E04504F5054604F50947E0
:1038700004F50948D5F8403A04F509497836443743
:10388000072B08F1640809F154090FD104F5F44439
:1038900042463946304638340194D5F860390093B1
:1038A0004B46BBF0D9FD0AB0BDE8F0870DF127010A
:1038B0008DF827004648FDF7BDFF05F69C1304F57B
:1038C0000A40D5F880A9D3ED007A05F51763643076
:1038D000D3ED000A05F67C1330EE670A93ED001A6B
:1038E000CDED060A8DED070A8DED051AABF00CFC47
:1038F0000546204601F09CF89DF827309DED051AFD
:103900004246DDED060A39469DED070ACDE9020380
:10391000CDE900A54B463046BBF0E0FCC3E7A988E3
:1039200006F0F8F80020BEE729460AB0BDE8F047E7
:10393000FFF792BA0AB0BDE8F047FFF74DBA294643
:103940000AB0BDE8F047FFF7C1BA0AB0BDE8F047DA
:10395000FFF71EBB0AB0BDE8F047FEF7EBBD04F56C
:10396000E040294678300AB0BDE8F047FEF766BE71
:1039700004F50A402946D83055E704F50A46D836FA
:10398000304608F073FA08B9304666E72946204603
:10399000FFF708F80028F7D185E70AB0BDE8F0473F
:1039A000FEF7F4BE0AB0BDE8F047FEF703BF0AB069
:1039B000BDE8F047FFF74CBE04F5E04029467830FB
:1039C0000AB0BDE8F047FEF7B5BE00BFA855140821
:1039D0001033022000F5E042134670B57833D2F878
:1039E000342305460E469A4202D00024204670BD7C
:1039F000FFF758FE04460028F7D005F5AE403188A1
:103A0000143075F077FAF1E738B500F5E044054673
:103A100094F8A839D3B1C1F06DFCD4F8C039C01AFC
:103A2000B0F57A7F12D90023002205F5AE400621B9
:103A300084F8A839C4F8C03904F6C41314301A60E5
:103A400001230C4A84F8C83970F0FEFD05F5E04505
:103A5000D4F834337835AB4208D14AF2CE63B4F8A7
:103A6000A22A9A421CBF002384F8A83994F8A80916
:103A700038BD00BFC45514082DE9F84304468946F3
:103A800090461F46FFF7C0FF054600B304F5E04629
:103A900004F5F544B6F8AA3904F12A00A9F8003073
:103AA00096F8A83A88F800301CF084FC04F12C0049
:103AB00087ED000A1CF07EFC089B83ED000A099B41
:103AC000B6F9AE2A1A800A9BB6F9B02A1A8028469F
:103AD000BDE8F88300F5E040B0F8AA398B4204BF96
:103AE000002380F8A839704738B500F540550446E2
:103AF00040F20F5004F5E0442DED048BB5F9303B56
:103B0000B0EE408AB0EE600A5A4207EE903AB0EE4C
:103B1000419A00EE902AB8EEE71AF0EE618AF8EECC
:103B2000E00A32F031FE04F6AC134FF4A26083EDEC
:103B3000000AB0EE490AB5F9323B5A4207EE903A14
:103B400000EE902AB8EEE71AF8EEE00A32F01CFE1A
:103B500004F51B6340F2115083ED000AB0EE680AD1
:103B6000B5F9343B5A4207EE903A00EE902AB8EE8F
:103B7000E71AF8EEE00A32F007FE04F6B41340F25A
:103B8000125083ED000AB0EE480A95F9A13A01EE11
:103B9000103A95F9A03A00EE903AB8EEC11AF8EE54
:103BA000E00A32F0F1FD04F6B81383ED000AC1F02B
:103BB000A1FBC4F8C009BDEC048B38BD00F5E040A2
:103BC00000F6C41383ED000A80F8C819704700009E
:103BD00038B500F5E0440D46D4F8340303685B685B
:103BE0009847A84211D10C280FD8012341F2F602C0
:103BF00003FA00F0104208D084F8A839C1F07AFB2B
:103C0000C4F8C00994F8A80938BD002384F8A8397D
:103C1000F8E7000021F04003152B04D0A1F15E036A
:103C200058425841704701207047000000F5E042BB
:103C30001346D2F834037833984205D1B2F8A23A49
:103C40005B1A58425841704700207047192965D8BF
:103C5000DFE801F00D1115191D2125292C643034E0
:103C600037593A3D4043474A4D5164555D6100F52F
:103C7000E2403430704700F5DE406C30704700F5AC
:103C8000DF400830704700F5DF402430704700F512
:103C9000DF404030704700F5DF407C30704700F572
:103CA000E0401830704700F5E040E2E700F5E04002
:103CB0005C30704700F5E0407830704700F5E14037
:103CC000E3E700F5E140E4E700F5E140F0E700F567
:103CD000E140F1E700F5E240E3E700F5E240503073
:103CE000704700F5E240C8E700F5E340C9E700F59A
:103CF000E3402830704700F5E3404430704700F55A
:103D0000E3406430704700F5E4401C30704700F534
:103D1000E4405830704700F5E44070470020704799
:103D200000290DDB0748CBB290F8442F9A4207D305
:103D3000D0F8403F0122A0F58040595C0DF09CBFB7
:103D4000704700BF1073022000F580432DE9F34156
:103D500093F8103F00F5AE45044603F0010603F06A
:103D6000020803F004075B0705F1140535D01F4A6C
:103D70000621284670F068FC26B104F5A4406430A2
:103D8000ADF07CFCB8F1000F04D004F5A74048303A
:103D9000ADF0E6F927B104F5AA402C30AEF0AEF84C
:103DA00004F500440123124A284684F8393E11499B
:103DB000114BB8F1000F08BF1A46002F08BF194673
:103DC000CDE900210D4A0621002E18BF13460C4AEA
:103DD00070F03AFC02B0BDE8F0810A4A062128469C
:103DE00002B0BDE8F04170F02FBC00BFE5551408EB
:103DF000DE5514085CB216087C941508D8551408D2
:103E0000F65514080856140810B5044600F5A440E9
:103E10006430ADF05FFC04F5A7404830ADF0CCF95C
:103E200004F5AA402C30AEF0A3F804F5004393F853
:103E3000392E5AB1002204F5AE40062183F8392EFE
:103E40001430034ABDE8104070F0FEBB10BD00BF47
:103E50002856140809B1FFF777BFFFF7D5BF000058
:103E600000F5E0420848D2F83413814209D092F8B4
:103E7000410338B913467833994203D192F8920935
:103E800070470020704700BF44A4022010B50446CC
:103E9000C1F030FA054BD3F85433C01A642804D863
:103EA0002046BDE810407AF0E7B910BD10A302200B
:103EB00010B500F59E448AB00023D4ED007AF5EEEB
:103EC000C07AF1EE10FA45D9079300F5F750089340
:103ED00003AA099306AB04A91830019307AB00931A
:103EE00005AB14F00DF930B3DDED087A9DED077ADE
:103EF00087FE277ADDED097A87FE277AD4ED007AEE
:103F0000B4EEE77A9DED047A77EEA76AF1EE10FA47
:103F1000F4EEC76AACBF01200020F1EE10FA0CD815
:103F200002309DED037AF4EEC77AF1EE10FA0CD868
:103F3000003818BF01200AB010BDF4EEC77AF1EEC8
:103F400010FA9CBF0130C0B2EBE7012894BF0020FB
:103F50000120F0E70020EEE738B5124B04461A7A4C
:103F6000FAB901251D726CF05FFF2A4604F50A4577
:103F70001121D8356CF008FD284607F0F7FF80B115
:103F8000284607F0B3FF062238B104F5E341283193
:103F90000548BDE838400DF09BBD04F5E2416C31A9
:103FA000F6E738BD60C1022010330220074B10B580
:103FB0001A7A4AB100241C726CF036FF2246112195
:103FC000BDE810406CF0E0BC10BD00BF60C1022035
:103FD0002DE9FF41054668461BF0F2FC694605F5F0
:103FE000F75808F11808404614F01AFA0646E8B1E6
:103FF0003748ABF089F850B105F59E43D3ED007A10
:10400000F5EEC07AF1EE10FA94BF0126002605F510
:104010000A40304C304FD83007F0A8FF00B146B10D
:10402000002328462380FB73FFF7C0FF04B0BDE8E0
:10403000F0812846FFF73CFFA0B363787BBB237871
:104040000133DBB2082B237002D1404614F0DEF8B6
:104050002378092B02D1404614F0D0F82378092B9D
:104060001DD94FF4857323806CF0DEFE02221021EF
:104070006CF08AFCC1F03EF96368C01A47F2305315
:10408000984209D905F5AE40144A0221143070F067
:10409000DBFAC1F02FF960602846FFF75DFF637817
:1040A000FB73C3E72378002BF9D0013B6278DBB2C6
:1040B0002370002AF3D0002BF1D166706CF0B4FEAF
:1040C000324610216CF060FC2846FFF76FFFE6E7F0
:1040D00074BD022060C102200DC202203C561408AB
:1040E00010B500F5E044D4F8403A042B01D101208A
:1040F00010BD00F50A40D83008F0B6FC0028F6D113
:1041000094F86C0AF4E7000073B500F5E0450192FD
:104110000446A5F84C13C1F0EDF8C5F85003D5F8E6
:10412000340303685B68984785F84A03D5F834037D
:1041300003685B689847019A182818D8DFE800F0F0
:104140000D170D0D0D0D0D0D0D1751175817585852
:1041500017404040171717405800334B93F83A3E2A
:10416000FBB104F5DF417C3120460DF0B1FCD5F800
:10417000340304F5AE4495F84A63036814345B686D
:104180009847864247D0D5F8340303689B68984720
:10419000264A03460421204602B0BDE8704070F074
:1041A00053BA04F5405393F9183B022BD9D0042B92
:1041B0000BBF04F5E04104F5DE4118316C31D3E763
:1041C00004F50043D3F8AC3DD90203D504F5E14131
:1041D0002431C9E704F5E3419B064CBF4431283143
:1041E000C2E720460192FFF77BFF019A0028BED16B
:1041F00004F54056019296F9183B002BB7D0D5F83C
:10420000340303685B68984785F84A0396F9183BBE
:10421000019A022BCAE7064A0421204602B0BDE8F3
:10422000704070F011BA00BF10B302204C56140851
:104230006E561408F0B5044685B00F46154604F5D1
:10424000E04679F09FFFD6F83403A6F84C73036874
:104250005B68984718281ED8DFE800F00D0D0D0D9B
:104260000D0D0D0D0D1D65820D0D71711D535353F7
:104270001D1D1D530D003E4BD3F8402A012A21D1AC
:1042800004F5405393F8193B023B012B1AD904F56E
:10429000A04383F81027D6F8340304F5AE44354A1A
:1042A000354B1434052D18BF1346026803939268EA
:1042B0009047039B00900421304A204670F0C4F9D7
:1042C00005B0F0BD2E4B93F83A3E3BB104F5DF410B
:1042D0002A467C3120460DF0FBFBDCE704F5405319
:1042E00093F9193B032B03D1204605F07BFCD2E761
:1042F000022BEBD0042B2ED104F5E0412A46783175
:10430000E8E704F50043D3F8AC3DDA0223D49B067A
:1043100004D504F5E3412A464431DBE704F5E341E3
:104320002A462831D6E72046FFF7DAFE0028B2D128
:1043300004F50A40D83007F041FE0028EED104F51C
:10434000405393F9193B032BCED0022BBED0042B44
:10435000D2D0012B9FD104F5E1412A462431B9E79F
:1043600004F5405393F9193B042B94D1C4E700BFE3
:1043700010A3022084561408793814088C561408A7
:1043800010B3022070B500F5AE450446124A042170
:10439000143504F5E046284670F056F90023A6F8D7
:1043A0004C3304F5405393F8B438032B12D196F8EC
:1043B0004A13302220460DF05FFCD6F83403036820
:1043C0009B689847054A034606212846BDE8704089
:1043D00070F03AB970BD00BFA0561408B756140863
:1043E00000F5A043002205294FF0040110B5044652
:1043F00000F5AE4083F8102700F114000CBF054A09
:10440000054A04F5E04470F01FF90023A4F84C338A
:1044100010BD00BFD0561408E156140830B50B4645
:1044200087B00446062A3CD8DFE802F03B4A1C84E9
:104430001291040000F5004393F8EC3B43B10422D1
:1044400000F5E441444807B0BDE830400DF040BB02
:1044500004F5004393F8EC3B23B104F5E341042257
:104460002831EFE704F5E04204F5E343D2F83413D2
:104470002833994224D004F5E443994220D0D2F85D
:10448000403A042B1CD0354D95F86533C3B13449FF
:1044900005F664203BF008F828B1304B012283F880
:1044A0006C2A07B030BD2E4905F664203BF068F950
:1044B00030B104F5E0410422A5F5E0407831C2E7CF
:1044C00004F5E04204F5E343D2F83413283399426B
:1044D000E7D004F5E4439942E3D004F50A40D2F86A
:1044E000405AD83008F0C0FA0028DAD1042DD8D0CC
:1044F00004F5405393F9E33A022B0ED004F5E14161
:104500000422204624310DF0E3FA04F56A502330EA
:1045100007B0BDE8304060F0ABBA104890F86533A2
:10452000002BEBD00E4900F664203AF0BDFF0028C6
:10453000B3D1E3E70B4A112101A8BFF0CBFF04F58B
:10454000084001AA0121B830ADF0C4FDA9E707B0C9
:10455000BDE8304005F046BB1033022010A3022016
:1045600064BC0220FC56140870B52DED048B044683
:10457000C0F0B8FE4F4B0546B4F8BE101A884E4E38
:104580008A424E4A06D01980002330601370BDEC79
:10459000048B70BD33684A49C31A8B4275D9012315
:1045A000137079F0FFFE79F0A7FD356079F0FAFE1F
:1045B00079F0A2FD04F5A04393F80F3723B104F579
:1045C0000840B830ADF0DAFC79F0BEFD0428DED941
:1045D00079F0D8FD0021204604F508450BF09AFB40
:1045E00000212046F0EE409A0BF09EFB0121204670
:1045F000B0EE409A0BF066FD00212046B0EE408AF6
:104600000BF09CFB04F50A40F0EE408AB8356430AC
:10461000AAF084FDDFED2B7A0028B0EE690A4FF096
:10462000040007FE888A7BF0BDFCB0EE490A132027
:104630007BF0B8FCB0EE680A15207BF0B3FCB0EE5E
:10464000680A1A207BF0AEFC4620B0EE480A7BF0E8
:10465000A9FC2846ADF020FD08BB012108467CF0EE
:1046600051F89FED180A02207BF09CFC9FED150A83
:1046700003207BF097FC20460BF066FF2046BDEC44
:10468000048BBDE870400CF065BF1278002A3FF43F
:104690007EAF44F6206293427FF679AF81E72846E9
:1046A000FCF756F804F5004393F9C2382B2BD4D00D
:1046B0006DE700BF6CC1022070C102206EC10220F4
:1046C000400D03000000000000F5E0431846D3F859
:1046D00034237830824202D193F86C0AE8B10F4B50
:1046E00093F8B40803F5A043A0F1270293F8483EDD
:1046F000012A0FD92C2809D00A2809D0A0F13102AB
:10470000504250410A2B18BF002070470120F9E7A2
:10471000012070470A3B58425841704710630220FD
:1047200008B500F5405393F8F42642B193F83037BA
:104730002BB1FFF7C9FF80F00100C0B208BD012016
:10474000FCE700002DE9F04700F54055044600F570
:104750000A40B14F8AB095F830876430AAF0D4FC93
:10476000D7F8403A0646042B42D1012104F55B57A5
:10477000DFF8B8A2343738468EF0FEFA9AF8483E91
:1047800081460A2B04D1002E54D100238AF8483EDA
:1047900095F8F436002B59D195F9FA369F4D012B37
:1047A00003D0063BDBB2012B11D895F8B4380A2BA5
:1047B0000DD104F5E046D6F8340303681B6A984728
:1047C00028B12B22D6F8381320460DF081F99AF83B
:1047D000483E0A2B04BF37238AF8483E95F8B43880
:1047E0000A2B02D1372385F8B4380AB0BDE8F08728
:1047F0000028BAD004F5E043B7F8A29AD3F83403FE
:1048000003685B6898471428AFD004F50A40D83095
:1048100007F07AFF0028A8D14946A7F5E040FFF746
:10482000F9F901460028A1D097F8681A4B1E5942A1
:1048300059419BE740EA0803DBB2002BA8D1AAF557
:10484000004000F0F5F800289FD0A1E7002ECCD062
:1048500004F505407830BAF081FC0028C5D1204627
:10486000FFF732FF0028C0D1B9F1000F00F0C3807C
:104870004A466B4938468DF055FE95F9FA86B8F1EF
:10488000010F06D040F38380A8F10603DBB2012BB1
:104890007DD85FFA88F8B8F1010F4BD104F5E042FA
:1048A0001346D2F834137833994207D192F86C3A10
:1048B00023B195F8E33A013B012B96D904F5E14188
:1048C0000A22243106AE20460DF002F930461BF0D4
:1048D00077F895F90D2792BBB8F1010F2FD004F5A9
:1048E0000048B5F90E37DFED4F5AD8F84019002BC4
:1048F000D1ED017AF8EEE77A52DD07EE103AF8EEE4
:10490000C76AE6EEA57AFDEEE77A304617EE901A12
:104910001BF05CF800233846CDE904338EF0C8FA6A
:1049200004A98FF019F800285FD0049B0893059B19
:10493000099317E004F5E1410A227831C2E72046E5
:104940006F46FBF795FF04F5094207EE900A2146F2
:1049500054323846B8EEE70AFDF702FB97E80F003D
:1049600086E80F0095F9FA36012B10D03146204623
:10497000FCF7E4FB31462046FDF7D6F995F9FA3607
:10498000072B04D104F5A044012384F80E376CF002
:104990004BFA4A4609210AB0BDE8F0476BF0F4BF74
:1049A00005F5E16393ED005A04F55C5393ED007A4D
:1049B00005F2FC63D3ED006A35EE076A36EEC57A80
:1049C000B4EEC67AF1EE10FA8BBF37EE067A05F632
:1049D0004433F6EE006A93ED007A8ABF27EE257A1B
:1049E000E7EE257AE7EE267A8DE7D8F840399A681F
:1049F000DB6808929CE7B8F1000F3FF4F6AE95F83B
:104A00003037002B7FF4F1AE04F5AE40064A0521A5
:104A100014306FF019FEBAE710A3022010630220D1
:104A2000085714080000C8421157140810B3022098
:104A300010B5044600F50A406430AAF06FFB98B147
:104A400004F50A40D83008F003FD60B904F5F444D9
:104A5000DFED097A94ED117AB4EEE77AF1EE10FA0F
:104A6000ACBF0120002010BD04F5F444DFED037A53
:104A700094ED117AF0E700BFCDCCCC3D6666663F81
:104A800038B500F5E04500F5E44304461C33D5F89D
:104A900034239A4202D195F8380AD8B904F50A406D
:104AA000B5F8A21AD83006F0A1FCA0B904F5E0448C
:104AB000D5F834337834A3420CD195F8383A4BB159
:104AC000D5F8403A032B05D1B5F8A20AA0F1160398
:104AD0005842584138BD0020FCE700002DE9F74F4F
:104AE00000F5E04A04465246DAF83413783291422F
:104AF00004D100F5405999F9BC2A3AB90022CAF804
:104B00002C2A8AF8292A03B0BDE8F08FC0F0F2FB06
:104B1000DAF88459804635B1451B40F6C3129542F8
:104B200094BF002501252046FFF782FF834620B170
:104B300000278AF8287A002640E004F50A4064300D
:104B4000AAF0E2FA01900028F2D004F50546783682
:104B50003046BAF003FB0746002840D09AF8286A8E
:104B6000C6BB3DB304F5005041F27071D0F8F0209F
:104B7000002AB8BF52428A4206DCD0F8F420002A4C
:104B8000B8BF52428A4228DD04F5F54104F50940D8
:104B9000283154301BF0BCFA0022CAF82C8ACAF81B
:104BA000302A9FED427BB4EEC70BF1EE10FA4CBFFA
:104BB0000126002601222F468AF8282A04F5907043
:104BC000F5F7DEFB022832D9002F42D10022CAF8C5
:104BD0002C2A98E75D465E46ECE73546EAE7304624
:104BE000BAF09EFA064640B1002DA4D04FF4FA72F6
:104BF0000026019FCAF8302AE0E7DAF8402A012AA5
:104C000007D0032ADAD12046FFF73AFF002892D1D5
:104C1000EAE709F65C32D2ED007AF5EEC07AF1EE01
:104C200010FA88DD9AF8382A002A84D1DEE704F5E4
:104C3000475599F81A130435284611F0E7F800286B
:104C4000C4D099F81A13284611F0DEF90028BBD118
:104C5000BCE7DAF82C0A10B9CAF82C8A53E7A8EB9B
:104C60000008DAF8302A9045FFF44DAF9AF8292A67
:104C7000002A7FF448AF01228AF8292A99F8BC3A21
:104C8000DB0705D504F50A400C216430F5F71CFA62
:104C900004F5AE40143036B1064A022103B0BDE837
:104CA000F04F6FF0D1BC044A3146F7E70000000036
:104CB00000C05240285714083E5714082DE9F04F01
:104CC000064600232DED028B06F5405985B006F50A
:104CD000907B0393C0F00EFB09F6B823804658463C
:104CE000D3ED007AF5EEC07AF1EE10FAC9BF9FED70
:104CF000C67A962767EE877AFCEEE77AC8BF17EE8A
:104D0000907AF5F73DFB022840F20D8196F81434B5
:104D1000B0229FEDBE7A02FB0363D3ED837A67EE88
:104D2000877AFCEEE77A17EE903A9F428CBF002715
:104D30000127B9F9AC3A06F5F75003A9022B00F1A7
:104D40001800B8BF022307EE903AB8EEE78AF6EEF5
:104D5000087A28EE278A13F035FB054640B1DDEDD1
:104D6000037AF4EEC87AF1EE10FAACBF0125002503
:104D7000584606F5E044F5F703FB01281AD806F576
:104D80000A406430AAF0C0F9A0B19DB904F64423EA
:104D9000DFED9F7A93ED007AB4EEE77AF1EE10FA48
:104DA00008DDDDED037AF4EEC87AF1EE10FAACBF5F
:104DB0000125002506F50A40D83005F065FD82463C
:104DC000002840F0018106F50A406430AAF09CF901
:104DD000002800F0078196F8143406EB0313D3F88B
:104DE000C0317BB158460193F5F7CAFA012800F2A9
:104DF0009C80019BA8EB030041F2873398428CBF53
:104E000000230123D4F8802902B11BB9002D40F002
:104E10008E803D4606F5E043D4F8342378339A4239
:104E20001AD199F9E43A002B40F08980002384F8E4
:104E30002A3AD4F8403A042B00F0B280072B00F055
:104E4000C580032B08D13046FFF71AFE20B100259C
:104E500084F8295AC4F8845994F82A3A03B18DB9D0
:104E600007EE905A9FED6B7A04F64423F8EE677ACA
:104E7000D3ED006A67EE877A9FED677AE6EE877A70
:104E8000C3ED007A3046FFF7D3FD054698B194F89C
:104E9000482AC4F880890AB9C4F84C8A06F5E04368
:104EA000D4F834137833994205D1D4F8843903B156
:104EB0000AB9C4F8848906F5004384F8485A83F88F
:104EC000ED5794F8C43C65F3C30384F8C43C9AF0EE
:104ED00067FD29469AF040FD504B30465D71FFF763
:104EE000FDFD3046F9F7EAFB35B199F8B6381BB944
:104EF000C0F000FAC9F8B808304689F8B658FFF78C
:104F000097FD002840F08E8006F50A406430AAF034
:104F100005F980F00100C0B284F8500A05B0BDEC7C
:104F2000028BBDE8F08F002703E753466AE730F0B5
:104F3000F5FD2FF027FC00287FF46BAF6AE75B429A
:104F400007EE903A06F58453F8EEE77A93ED027A8D
:104F5000F4EEC77AF1EE10FA13DD0123DFED307ABB
:104F6000C4F8348A84F82A3A04F6442393ED007A8C
:104F7000B4EEE77AF1EE10FA7FF75BAFC3ED007A9B
:104F800057E794F82A3A002B3FF453AFD4F8343A59
:104F900040F6B832A8EB030393423FF647AF48E729
:104FA00006F505407830BAF0BBF800283FF454AF5E
:104FB00004F51763DFED1A7A93ED007AB4EEE77A21
:104FC000F1EE10FA7FF748AF012545E704F51763C6
:104FD000FEEE007A93ED007AB4EEE77AF1EE10FA85
:104FE000F2D439E7002DD4F8403A18BF3D46012BE2
:104FF00001D1002530E706F505407830BAF086F893
:105000000028F6D128E700BF0000B4420000C842E3
:105010009A99993E9A99193E9A99593F0DC2022040
:10502000CDCC4C3E002077E7002070470020704731
:1050300001207047034BD3F8400A431E58425841A1
:10504000704700BF10A3022030B587B002A81AF045
:10505000B7FC3B48BAF05AF820B13A493A48FCF755
:105060007FF81FE03648BAF05BF8E8B1374C04F13E
:105070002405234604F11002A4F11001A4F5777071
:105080000095BAF08BF8A4F6DC7204F110033049F5
:10509000A4F57770CDE9004592ED000AA4F1100265
:1050A000BAF01CF807B030BD02A92548BAF08EF856
:1050B00008B102A9D2E7274CD4F8303C002B0CDD14
:1050C00094F8D03B4BB1A4F580402049FCF748F858
:1050D000A4F58040FBF7C2FCE4E71B4804F018FC91
:1050E0000028BAD11C4C94F864395B0720D4D4F85A
:1050F0007839002BB1D0134AA2F12001A2F110009F
:105100001AF042FF0028A8D1144CB7EE000A0E484E
:10511000D4ED007A04F6E87130EE670AFCF750F837
:1051200004F6C87204F6E8710748FBF7CDFBB9E74F
:10513000A4F50040FCF7C2F80028B3D1D7E700BFC0
:1051400088B8022074BC02201033022064BC022004
:10515000588202201073022010B302208CAC02206F
:105160000A4808B590F8553B013B012B03D8A0F540
:105170004050F6F7F5FC0648F6F7B6FB0448F6F79C
:10518000AFFC0348BDE80840F7F78CB81063022075
:105190001033022010B5044607480DF0B9FB50B19A
:1051A000064B93F8190C30B1236820469B6B984747
:1051B00080F00100C0B210BD30C0022010B3022048
:1051C00010B504461448FEF71FFC08B1002010BDBE
:1051D000124B9C42FAD003F11C029442F6D003F128
:1051E00038029442F2D003F174029442EED0D433E8
:1051F0009C42EBD0236820461B6A984720B1084B9D
:1052000093F80E37002BE1D1206907F047FC80F0BE
:105210000100C0B2DBE700BF1033022098A20220D9
:105220001083022010B504461948FEF7EDFB08B1C3
:10523000002010BD174B9C420ED003F11C0294427B
:105240000AD003F13802944206D003F1740294426A
:1052500002D0D4339C4206D10F4B93F90D0BB0FA18
:1052600080F04009E5E7236820461B6A984720B193
:105270000A4B93F80E37002BDAD1206907F00EFCA9
:1052800020B12069BDE8104009F0A2BF0120D0E79D
:105290001033022098A20220106302201083022003
:1052A00073B50F4E0D46114696F9A42B1AB9012479
:1052B000204602B070BD036801915B6998470446BF
:1052C0000028F4D1D6F8AC3D019913F4802FEED02C
:1052D00004482A46044B0068C06A2DF0C7F8E7E787
:1052E00010B302200C33022050571408084A026001
:1052F000084A111F4260816002F10801C160A2F1F9
:10530000380102F59C7201614261034A8261704773
:105310009C57140820BE02200852022008B50368DA
:105320001B6E9847064800F15C03D0F834239A427C
:1053300005D0A0F5E040BDE80840FEF765BD08BD1A
:1053400010A302202DE9F341684C0027684A00258C
:1053500004F6581306464FF0FF3104F6F8101F60AC
:1053600004F6142384F8A859A4F500581A6004F62A
:10537000EC13604A84F83C591A602A46A4F8925902
:1053800084F8965984F8545984F8295A84F82A5A8A
:10539000C4F8E059C4F8DC59C4F8D859C4F8E8593D
:1053A00084F8205AC4F80C5A1AF010FB04F1780360
:1053B000F21A5342534188F8F03904F668131F601B
:1053C00004F58057B36907F6441CD3F8FC3184F820
:1053D0009559A4F88C3907F6541384F8A459C7F8E2
:1053E00020590FCB8CE80F00BFF084FFC4F83C03BA
:1053F000336830465B6998474FF0FF3384F899591A
:10540000C4F86C3388F8105784F89809306906F0AE
:10541000E5FC87F87D5984F8975930463368DB6D91
:105420009847054600285DD0336830469B6B984707
:1054300084F8380A336830465B6B984787F8EE0784
:10544000D8F87C090368DB6B984708F2AC60ACF0D5
:1054500087FAA4F5E0400AF0ADFB27488DF0F2FC96
:1054600094F86C3ACBB1A4F5E040FFF7E1FAA0B9AB
:1054700007F66420A9F052FE78B9D4F83403036823
:105480005B6B984748B976F03FFC1C4A06216FF0E9
:10549000DBF804F6642039F0E3F81948F5F792FADE
:1054A000336993F9CC206AB101A9586812F08AFFD8
:1054B000376901469DED010A07F18800FAF78CFE75
:1054C00087F84101336830465B69984750B13369CA
:1054D00093F94C22002A02DD93F8B03213B900236D
:1054E00084F84133284602B0BDE8F08110A30220C1
:1054F000000080C0000080BF046A02205C571408CE
:105500001033022070B503680E4615465B6E98474F
:10551000044650B995F900303BB905483246054B71
:1055200029460068C06A2CF0A1FF204670BD00BF6C
:105530000C3302208057140810B50E4C2046ACF0F6
:1055400001F804F5B270ABF06FFD04F53270ACF009
:10555000BDFC094B002103F5E04203F5A04382F8AE
:10556000541902F6581200211160012283F8B0216B
:1055700010BD00BF748502201033022008B52DED48
:10558000028BB0EE408A15207AF00CFD1A20B0EEA6
:10559000480ABDEC028BBDE808407AF003BD00006C
:1055A0000848012108B590F90D3BA0F5405033B1F2
:1055B0000AF088FD4620BDE808407AF0F3BC0AF006
:1055C000A9FDF7E710630220012070470120704712
:1055D0000120704701207047012070471920704753
:1055E00000487047045814080048704714581408BD
:1055F00084B038B505AC05460D4884E80E0014218A
:10560000FBF73EFD2A696423B2F9C01068B103229A
:10561000594320461AF0DAF921460548FCF784FB85
:105620000120BDE8384004B070470122F0E700BF18
:105630001033022013B511496A46A1F110001AF087
:10564000ADFA40B19FED0B7B9DED006BB4EEC76BE7
:10565000F1EE10FA0CD80A4CD4F87C0903689B6B65
:10566000984728B12E220749A4F5A0400CF030FA43
:1056700002B010BD00000000000080BE74BC02201B
:1056800010830220B8A4022030B51D4C054687B017
:10569000D4F8380303685B69984738B12F22194959
:1056A00019480CF015FA012007B030BD174807F073
:1056B000F5F90028F2D1A4F50054D4F87C09036868
:1056C0009B6B984728B1D4F87C0903681B6C9847FA
:1056D00098B10F4B02AC0FCB84E80F00284601F0C5
:1056E000CFF92868059B009394E80E00446C284687
:1056F000A0472846FFF79EFFD5E7064BEAE700BF25
:1057000010A30220B8A4022010330220E8BD02201A
:1057100064BC022074BC022010B50446FFF78AFF67
:105720002046BDE8104001F0F7B9000004207047A2
:10573000004870478D5E1408004870478D5E14085D
:10574000037F73B1D0ED087AFDEEE77A17EE903A59
:10575000084AC2F8543A437F3BB1436AC2F8583A08
:1057600070478369D3F8F831F2E78369D3F8FC31E5
:10577000F4E700BF10A3022008B5002300F12801C0
:105780008383806912F040FE012008BDF8B56D4E9C
:105790000446012106F5E047304606F540552DED5B
:1057A000048B97EDE19A0AF0B5FAB0EE408ADFED8E
:1057B000669A012130460AF0B7FAB5F9303BC8EED7
:1057C000297A04F1280108EE903AB5F9323BA06934
:1057D00008EE103AF8EEE88AB8EEC88A68EEA78AB2
:1057E000C0EE297A28EE278A12F00EFE95F9363B94
:1057F0005BB3F0EEE87A9FED557AF4EEC77AF1EEFE
:1058000010FA22D5227FA369002A54D101222277DF
:105810000022226294ED087AB0EE490ADFED4C7A5C
:105820000122D3F8F83167EEC77A9FED4A7A4A48E9
:1058300067EE877AFDEEE77A17EE901A0B44C7F809
:10584000543A0023ABF00EFE08E00023F0EE490AC4
:10585000B0EE680A40482377ABF000FE04207AF0EF
:10586000A1FB95F9363B43B1F0EEC87A9FED377A4C
:10587000F4EEC77AF1EE10FA28D40023F0EE490ACC
:10588000B0EE480A35486377ABF036FA13207AF069
:1058900089FBB5F9343B002B03DD314E96F94235D7
:1058A0005BBB20212748F5F789FC002842D1254819
:1058B0000AF04CF841E0D3EDC56A96ED467AD4ED96
:1058C000087AE6EE877AC4ED087AA3E7637F2BB9FE
:1058D00001236377A369D3F8FC316362616AB0EE98
:1058E000490AC7F8581AA369D3F8FC010023091A1A
:1058F0001A461A48ABF0E8FAC8E70121A6F5A0401D
:105900000AF01CFA80EE297AB5F9343B002106F240
:105910002C5007EE903AF8EEE77AF0EE490A27EEBF
:10592000870AACF0C7F92046BDEC048BBDE8F8400F
:10593000FFF724BE0348F6F721FB07EE900AB8EE06
:10594000E70AF0E71033022000A08C450000003485
:10595000E02E65420000C84274850220D8860220ED
:10596000108302202DE9F04FDFF89CA300F12805F9
:10597000044601210AF5E04B50460AF540562DED4C
:105980000C8B97B09BEDE1BA0AF0C4F901215046A7
:10599000F0EE408A0AF0C8F901215046B0EE408A84
:1059A0000AF0CCF9DFEDCD7AB6F9303B01A888EEEC
:1059B000A77A9FEDCBDA0AEE903AB6F9323B9FED2B
:1059C000C99A0AEE103AB6F9343BDFEDC78AF8EE11
:1059D000EAAA09EE903AB8EECAAAF8EEE99A6AEE97
:1059E00087AA88EE277A9FEDC18AF0EEEACAF4EE24
:1059F000C8CAF1EE10FA54BF4FF001094FF0000988
:105A00002AEE07AA80EE277A9AED460AB0EECACAB5
:105A10006AEE8D7AB4EEC8CACDED017A6AEE0D7ADF
:105A2000F1EE10FACDED027A54BF4FF001084FF0BD
:105A3000000869EE879AF0EEE9BA69EE8D7AF4EE25
:105A4000C8BACDED037AF1EE10FA54BF0127002752
:105A500036F094F801A9284634F01EFD284634F0AB
:105A600023FE284634F08AFD20EE090A284620EE5F
:105A7000280ABDEEC00A10EE103ACBF8543A34F0C2
:105A800097FD20EE090A20EE280ADFED998ACDED78
:105A90000D8ABDEEC00ACDED0C8ACDED0B8A10EE5D
:105AA000103ACBF8583A0DF1280B4FF07E53A0690D
:105AB00059460A9312F0A8FC002150460AF002FB56
:105AC000B0EEC00AB4EEC80AF1EE10FA16D5504690
:105AD000FEF7AEFF90B9F4EEC8CAF1EE10FA0DD59C
:105AE000B4EEC8CAF1EE10FA08D5F4EEC8BAF1EE79
:105AF00010FA44BF9BE80F0085E80F000AA80DF1DB
:105B0000100A34F025FE294612A88DED141A8DEDE9
:105B1000120ACDED130ACDED151A34F03FFE5146B1
:105B20000EA88DED101ACDED048ACDED058ACDEDD0
:105B3000068A8DED0E0ACDED0F0ACDED111A34F067
:105B4000DFFBB6F9303BF4EEC8CADFED6A7A01EE4E
:105B5000103AB6F9323BF1EE10FA09EE103AB6F906
:105B6000343BB8EEC11A08EE903AB8EEC99AF8EE96
:105B7000E88A21EE271A29EE279A68EEA78A21EEF5
:105B80000D1A29EE0D9A68EE8D8A06D594F83830F4
:105B9000DFED577A002B01FE271AB4EEC8CAF1EEEA
:105BA00010FA06D594F83930DFED517A002B09FE52
:105BB000279AF4EEC8BAF1EE10FA06D594F83A3006
:105BC000DFED4B7A002B48FEA78A9AE8070007AE64
:105BD000F1EE410A86E80700C2209DED070A30F089
:105BE000D3FDB0EE491AF1EE490AC3208DED070A44
:105BF0009DED080A30F0C8FDB0EE681AF1EE680AB3
:105C0000C4208DED080A9DED090A30F0BDFD514616
:105C100030468DED090A35F047FF12A928468DED73
:105C2000120ACDED130A8DED141A34F035FC284616
:105C300034F03AFD304BDDED076A304693ED9A7A49
:105C40009FED280AC6EE877ADDED086ACDED077A6A
:105C5000D3EDF37A86EEA77ADDED096A8DED087A49
